:020000040000FA
:080000000002040000000000F2
:020000040000FA
:100400004F5F21000E7F22000E01880000000000D7
:100410000C000700A04D2A00010020001100070079
:10042000000020000000E000020032000000020096
:1004300000000000F2BE0200000000000040DA00F0
:100440000000FE004440A900206F21000000E000F1
:100450000300320000002000A00188004440A800F2
:100460000000060091018800800078000000EB0089
:1004700015003700E280400032A0B4009101BA00BC
:10048000E280400032A0B4009102BA00E280400055
:1004900032A0B4000002EB00472BDE00F507B200EB
:1004A000602CE10004003A000059EB008301E900F0
:1004B000FDFF3E00040037006128E100010032002A
:1004C0000082EB00040007001101BA000200E00006
:1004D000E8FF3A00000006003159BA008301E90044
:1004E0000C0032002159BA008301E90008003200F3
:1004F0000400E00003003A00E280400032A0B400B3
:10050000F5FF370011D9BA008301E900FAFF3A007C
:100510008100E800E180400032A0B4000000060045
:100520000EDF04000000000068DF0400000000008F
:10053000B6DF0400000000006CD5040000000000DD
:10054000ECD50400000000003AD6040000000000D2
:10055000D081040000000000D281040000000000EF
:10056000DE810400000000002EC80400000000002E
:100570009CC8040000000000F4C804000000000053
:1005800082B30400000000009CB3040000000000DF
:10059000A6B3040000000000B0B304000000000097
:1005A000B8B3040000000000C8B30400000000005D
:1005B0004CB404000000000026B504000000000058
:1005C00040B50400000000005EB50400000000001B
:1005D00086B5040000000000C2B504000000000061
:1005E000EAB5040000000000C0B3040000000000F1
:1005F000ECB50400000000001AB604000000000082
:100600000AB4040000000000FCC504000000000063
:100610000CC604000000000044C6040000000000F6
:100620004AC604000000000056C604000000000096
:1006300066C60400000000006EC604000000000052
:100640009CC6040000000000CAC6040000000000B0
:10065000F8C604000000000022C7040000000000EB
:100660003EC704000000000044C704000000000072
:1006700052C704000000000088C70400000000000A
:1006800004C604000000000092C70400000000003F
:100690000040DA000000FE001004B1000300350045
:1006A0009001B10001003C001000050000000500B1
:1006B000800078001104B100030035009101B10001
:1006C00001003C000050A000000006001004B10032
:1006D000070035009001B100040034007000B10043
:1006E000030035009001B10001003C00100005003E
:1006F000000005006900E100040035006D00E10024
:10070000030034000002B1000100320000000500C7
:10071000100005002002E20004003D002342AB006F
:10072000020032002302AB00FEFF32000040DA007C
:10073000FEFF37000A00FA0080017800E20F500047
:1007400028003E0080AB8000E10F5000080032001E
:10075000802320000000E000050032000423200078
:100760002523200046232000800178000400370064
:10077000042220002522200046222000832220007F
:10078000144090000004E000040035008009EB00F4
:10079000144090000074A000104298001540900092
:1007A0000028A30003003A00154090000024A00098
:1007B000904298008001EB00070037001540900040
:1007C0000008A300FDFF320063C078000000FB00BA
:1007D000000B78008301E800828F5100F7FF3A0098
:1007E0000800370030002000B0BF9F00C3BF9F004B
:1007F000D1BF9F00E2BF9F006A80570000C0DA00AF
:100800006FB99700020078000080FA00000006002F
:100810000A00FA0011002000B1BF9F00C0BF9F0076
:100820006A80570000C0DA004FB897000080FA00D5
:10083000000006000A00FA0051002000B1BF9F002E
:10084000C0BF9F006A80570000C0DA005FB8970001
:100850000080FA00000006000A00FA00881F7800F5
:10086000800178000000E00029003A0080AB8000A1
:10087000E10F500008003200802320000000E0005B
:1008800005003200042320002523200067232000D8
:100890008001780004003700042220002522200077
:1008A0006722200083222000144090000004E00012
:1008B000040035008009EB00144090000074A00093
:1008C000104298000002EB000C003700130A2000D1
:1008D000154478006140640002003A008301E90099
:1008E000FBFF3A000402E8009541780061C0610016
:1008F000050032001700780080587800040351008A
:10090000820F5200F1FF3A00060051000800370044
:1009100020002000A0BF9F00B3BF9F00C1BF9F0069
:10092000D2BF9F006C80570000C0DA005FB897000C
:100930004F0478000080FA0000000600889FBE0087
:100940008004780090AB80000000E00003003A00D3
:10095000100007000000E0000A00350090AB8000A6
:100960000900E00002003A000004780006003700A9
:100970000004780009004000060007000000E000C5
:1009800001003D000084EB00080078004F04BE0029
:1009900000000600800078000000E00004003A003B
:1009A0004057210090AB8800010178000600370015
:1009B0000081EB00405F2100808F500002003E006C
:1009C00091AB88000001EB000200780000000600F7
:1009D000020AB900001BB9000200B8008100420001
:1009E0008100430000000600F4FF2F008B02370057
:1009F00004002000890237000001BE00A2020700A7
:100A00000470A70003F0A10003F8A30013003A004C
:100A10006509B10010003200090035006928E100C5
:100A20000200350001002800000005000000400021
:100A3000818048008502E900FCFF3A0000000600C2
:100A4000F88F4200050035008100D1000080D300FE
:100A50008502E800FCFF3A00000006008000EB0081
:100A6000000005000001BE00870207000470A70017
:100A700003F0A1006509B100160032000D00350039
:100A80006828E10006003500F0FF2F00F1FF270085
:100A90000300E00013003B000100280000000500F7
:100AA00000004000818048008502E900FCFF3A0018
:100AB00008003700F88F420002003C008000EB0085
:100AC000000005008100D1000080D3008502E8000D
:100AD000FCFF3A000300E00002003B006000100051
:100AE000E0801800000006006022B8000602200026
:100AF0000000D0008180D2000482D2008582D20022
:100B00000000A0000202520083825A00030031005C
:100B10000202420083824A000000A1000603E900AD
:100B2000F3FF3A000000060003F0A200889FBE0019
:100B30008A9FBE008C1F7800680207006F02330096
:100B40006450E1004F0032006420E10052003200A6
:100B500003826C0007003B000905D0000306D000AB
:100B6000820F54000C065D000200390002003200C2
:100B700089017800030678008582550004003D0055
:100B80000003FD008103FD008502EA008B85420021
:100B9000840F720002003B0060001000E08018002B
:100BA0006011B8000005EB007A28E1000A00390066
:100BB00006007800C75DDD00F707B200878075008A
:100BC0002D003700828171000A0178006105600004
:100BD0008180D1000080D3008502E900F9FF3B004D
:100BE000060440008784480002003B0060041400B3
:100BF000E0841C000988A300070032008A8171008C
:100C000082817100610164008904D1000884D300ED
:100C10008B05E800170037000978A30013003A009D
:100C20000B00E000130034008B05E90008044400C9
:100C300089844C000A4474000978A3000D003A002E
:100C40000B00E000070034008B05E90008044400B5
:100C500089844C0001003A000B0020000978A300B1
:100C6000F7FF32000001EB000200370082817100C3
:100C70000A017800310207000CF0A70001F0A00083
:100C8000270237006420E10002003A00838F6C00E5
:100C9000270233000801BE000200BE002002370018
:100CA000889FBE008A9FBE008C1F78000B02070041
:100CB0001202330003866C006450E100240032000D
:100CC0006420E100270032006150E1002200320080
:100CD0006120E100210032008B854200EB07B1006A
:100CE0000134B800003AB8000804420089844A0080
:100CF000013AB8000030B8008880400009014A007D
:100D000004003300000040008180480002014900D7
:100D10008B05E900C909DD00830170000100320084
:100D200013002000C814DE004814DD004709DE006F
:100D30001200B200C808DE0008847000FF0107003E
:100D400001F0A1000CF0A70001F0A000F4013700B1
:100D50006120E100F60132000801BE000200BE0081
:100D6000F7FF37006150E100FCFF3A00F001370067
:100D7000889FBE008A9FBE008C1F7800D7010700A5
:100D8000DE01330003866C006450E1002E00320067
:100D90006420E100330032006150E1002F00320096
:100DA0006120E1003100320085855500EB07B0007D
:100DB0000900200008042000050037000804440052
:100DC00089844C000A0031000603430087834B00EE
:100DD0000001530081815B00F8FF33000203BE0075
:100DE0000800A0000804440089844C00F6FF390084
:100DF000C639DD00830173000100320013002000BA
:100E00008904D1000884D3000998A30005003200AA
:100E10000800A7000300A0008904D1000884D300C3
:100E20008B05E8008904D1000884D3000001EB00A1
:100E30000281D200C101070001F0A1000CF0A7005F
:100E400001F0A000B60137006420E100B8013200D3
:100E50000801BE000200BE00F7FF37006120E1007C
:100E6000B30132006000B800F3FF3700000020003B
:100E700001F82700F0FF3700889FBE008A9FBE0060
:100E8000010578000100E0000400350008003C0086
:100E90000000E00020003200050037006000100074
:100EA000E080180002003B0001F02C001A0037001F
:100EB0000004BE006011B8006B0920000982CF0059
:100EC000020039000882CF000441B000694252009C
:100ED0000E00320008003B00828171006101640055
:100EE0008904D1000884D3008B05E8000442E8009F
:100EF000F9FF3A00050037000804440089844C00DB
:100F00008B05E9000442E900FBFF3A008B01070072
:100F10000AF0A70001F0A0004F05BE004F04BE007C
:100F200000000600140020003C013700EEFE070020
:100F30000400BE0000000600889FBE008A9FBE001D
:100F40008C1F78000205BE000004BE000006EB0006
:100F5000E00F5000E08F5800E00F5900E08F59007B
:100F600007003D006000B8006011B80008045000A0
:100F7000898458000A0559008B8559001C002000FF
:100F8000E00F5200E08F5A00E00F5B00E08F5B0043
:100F900002003D000F0007000C00A2000800BE0088
:100FA0000A01BE008B0107000203BE000002BE0062
:100FB0000C00E00001003200060007000400BE0043
:100FC0000601BE004F0678004F05BE004F04BE006C
:100FD000000006006000B8006011B8000402500074
:100FE00085825800060359008783590000000600D7
:100FF000881F7800000478005001BE004000BE0049
:1010000004004000858048000601490087814900AE
:10101000009CBE000294BE000400E1000588E100CF
:101020000690E1000798E1000200310068004400EA
:101030001008E8004F04780000000600F48747001D
:10104000889FBE008A9FBE008C9FBE008E1F7800C6
:101050000205BE000004BE00D4B79F00E5B79F00A4
:10106000F6B79F0087BF9F000000EB00C0B79F004E
:10107000B0B79F00A0B79F0090B79F0080B79F00B8
:101080000D042000BFB097004FB097000001400052
:101090000000E0000F003D004F08DE00000071007E
:1010A000C0B79F009E00070001003D001200200015
:1010B000A100070001003D0012002000A60007006B
:1010C000B1000700B60007000F004000C8FF07008E
:1010D000220037004F08DE0000067100CCB79F00E9
:1010E0008F00070001003D00120020009200070061
:1010F00001003D001200200097000700A200070039
:101100000FB297009FB297002FB39700BFB397001D
:10111000A90007000000520081805A0002015B0014
:1011200083815B0080B79F0091B79F00A2B79F00AB
:10113000B3B79F000007EB009F0007000020E1000D
:1011400001A8E10002B0E10003B8E10001003100B4
:101150001E0020000E005600C0B79F004FB297003F
:101160000400E0000700350010002000010020000E
:101170006011B80008047000898470000A057100CD
:101180008B8571008D06E900BEFF3A000400E00087
:1011900003003D00820007000F00400094FF07009D
:1011A0004FA897000000E00004003A000FB4970039
:1011B0009FB497002FB59700BFB597009400070024
:1011C0004F0778004F06BE004F05BE004F04BE001B
:1011D0004F01B10000000600881F780018002000B1
:1011E000881F780095FF07008F87E9004F0478007B
:1011F00000000600801FEB0090FF07008F87E900CA
:1012000000000600889FBE008A9FBE008C1F7800E9
:101210006E00070007003D0073000700E00F5B0051
:10122000E08F5B0007003D00320007000006EB0086
:10123000040037003400070002003D002A000700C8
:101240001C00200072000700E3FF07000203BE003D
:101250000002BE000C00E000010032002200070086
:101260000400BE000601BE004F0678004F05BE0018
:101270004F04BE0000000600889FBE008A9FBE008B
:101280008C1F78005100070005003D005600070044
:10129000E00F5B00E08F5B0006003D0004003700BC
:1012A0001900070003003D006000B8006011B8009D
:1012B0001000070056000700CEFF07000203BE0023
:1012C0000002BE000C00E000010032000600070032
:1012D0000400BE000601BE004F0678004F05BE00A8
:1012E0004F04BE00000006006000B8006011B800A6
:1012F00000003700040250008582580006035900A0
:1013000087835900000006000006EB00E00F520042
:10131000E08F5A00E00F5B00E08F5B0000000600EA
:101320000180400090B79F000001EB008FB0970054
:101330000100E000000006000200700090B79F006E
:101340000180400080B79F000001EB00FFA89700DC
:101350000100E000000006000200700080B79F005E
:10136000018040006FAA9700CF20DE0001007000CE
:10137000F0AF9F0004024200250007004F18DE0076
:101380000002720000000600E4AF9F000804440061
:1013900089844C000A054D008B854D000000060035
:1013A0003FB29700CFB297005FB39700EFB39700BB
:1013B00000FE2F00000006003FB09700CFB097005E
:1013C0005FB19700EFB19700000006000205BE0074
:1013D0000004BE00E00F5000E08F5800E00F5900FD
:1013E000E08F5900000006006000B8006011B800EE
:1013F00008045000898458000A0559008B8559005B
:101400001C002000E00F5200E08F5A000000060090
:101410000800BE000A01BE0000000600889FBE0052
:101420008A9FBE00841F78002C0007004F007800C0
:1014300011003300F0FF2F00838F6C0006003B008B
:10144000040565000A00A7000800370009F0A6009F
:101450001000200008003700820F5400838F5C00CA
:10146000030039001000200001003E0000002000B1
:1014700009F0A7000000EA004F05BE004F04BE00BF
:101480000000E00000000600C70ADE00F107B2001D
:10149000F50FB20008003200E1CF42000200320036
:1014A0000170A00024000500810F700001003200CF
:1014B0000408050044000500810F700002003A0096
:1014C000140005008502E9000000400081C04800CA
:1014D000FCFF3B000170A000240005000004BE00DA
:1014E000E9FF07000003BE000405BE000200BE00C5
:1014F000E5FF0700844F7500000006000200BE00F3
:101500006450E100050036006420E100020036006E
:101510000968A30001003A000800BE000160A000B5
:101520004F0678004F05BE004F04BE0000000600C5
:10153000F0FF2F00F1FF2700F9FF370081002000A6
:10154000618055000B003D000B00200061FE2F0064
:101550000100E1001D00340082817100610164001E
:101560008904D1000884D3000000E800FAFF3A00A3
:101570007100200061006400030070000200600040
:101580000900320061044400E0844C000988A50091
:10159000050032008B05E8006808E10002003A000F
:1015A0008904D1000884D300F20F20000258E10022
:1015B00005003D00C75DDD00F907B20089807500B8
:1015C00008007800000006000BF827008B00780068
:1015D00000000500889FBE008A9FBE008C9FBE0051
:1015E0000404B8000506B8008904460060854E0072
:1015F0000606B8000A054600E0854E000706B8005A
:101600008B054600040EB800890446000A854E008A
:10161000E0854D00050EB8000A0546008B854E009A
:10162000060EB8008B0546000416B8000A054600F1
:101630008B854E000516B8008B054600041EB800C9
:101640008B0546000800BE000A01BE004F06BE0022
:101650004F05BE004F04BE00000006002800FA003F
:10166000889FBE008A9FBE008C9FBE0003866B00D1
:101670000F0207000028A30064003A000128A3001D
:1016800067003A000008A30062003A000108A300C6
:1016900065003A001E009000BE08900081064000E0
:1016A000ED3FB100F4805700EE019000111AB80030
:1016B0008E099000311BB8009E099000311CB800C3
:1016C000511DB800F485570046000700FE01900048
:1016D0003A0007008B85E8003E0007008E09900065
:1016E00040000700EE019000340007008B85E80001
:1016F000380007008E099000400007009E09900006
:101700001B18B800890440000A854800FE019000BB
:10171000340007008B85E80038000700EE019000D8
:10172000300007008E0990001B18B80089044000A3
:101730000A8548000A98A30008003A000402420003
:1017400085824A0006034B0087834B0008044C0047
:1017500089844C000A054D008D06E90084827200E0
:10176000850273004C3ADD008502720001003200F0
:1017700015002000443ADE001400B2004538DE00B7
:10178000CB45DD000B007000C540DE00CB4DDD0019
:101790008B8070004549DE00CB55DD000B017100E8
:1017A000C551DE000D037800DA01070003F0A10047
:1017B0000CF0A70003F0A000D10137001B18B800FF
:1017C0008502400006834800E0834B0060044C0023
:1017D000070037001B18B800060340008783480045
:1017E000FAFF37001B18B800870340000884480040
:1017F000E0844C0060054D00000006001B18B80096
:101800000804400089844800FAFF37000108A3005B
:10181000B8013A005800BE005801BE00E3FF37008F
:101820000008A300B3013A0009047800F9FF37006B
:101830008103780014FF07000001BE006000B800BB
:101840000478A30013003A006220E10015003E0076
:101850000D0039008301D1000281D3008180D300C3
:101860008301D1000281D3008180D3008301D100A4
:101870000281D3008180D3000538B000C42ADD0086
:10188000F300B2008381720007F0A70003F0A0000C
:1018900000000600F3FF2700F2FF2F006110B900DF
:1018A000FBFF370003FF2700F7FF37008F1FD10032
:1018B000C40107008F87E9000000E0000000060077
:1018C000801FEB00BF0107008F87E9000000E000E8
:1018D000000006001400FA00889FBE008A9FBE0028
:1018E0008C9FBE000005BE000206BE0068004700D7
:1018F0000C90BE000A90BE00DB0107006400E1000E
:101900001A00320016003E006100E1001A003200A9
:101910006E049000FE0490000E0B90009E0B900051
:101920006011B8009E0590000B38B100D501200071
:1019300082817100610164008703D1000683D300B6
:101940008984D3000884D3008502E900F8FF3A00B7
:10195000FAFE07000DF0A70001F0A00068013700B3
:10196000F1FF2700F0FF2F006501370001F8270085
:1019700000002000F7FF37006000B800F5FF3700D7
:10198000E00107000509780000000600809FEB00D9
:101990008C0107008F87E9000000E00000000600CE
:1019A0002800FA00889FBE008A9FBE008C9FBE0060
:1019B00007067800878669000C003B000304780066
:1019C0008704780008F0A10009F0A100840F5000FE
:1019D000858F5800860F5900890F5C000300330083
:1019E0000CF0A20001003A000CF0A1003001070049
:1019F0006400E1005F003200780147006408E10004
:101A0000610032006C014700748557003200BE004F
:101A10001201BE003A04BE001A05BE001E0390006B
:101A2000BE0A90008503530006003D000004FD003F
:101A30008104FD000205FD008305FD008703EA0027
:101A4000050378000DF8A3000400320060041400C0
:101A5000E0841C0060051D00E0851D006022B800C8
:101A60007D0320000D38E1008006EB000B003900FB
:101A70004433DD00F300B200830173003900370006
:101A8000848272000D027800E10664008B85D1002B
:101A90000A85D3008984D3000884D3008703E90032
:101AA000F7FF3B0008004000898048000A01490018
:101AB0008B81490004003B0060001000E0801800AA
:101AC00060011900E08119000358A30009003200E9
:101AD0008D82720084827200610260008301D100F5
:101AE0000281D3008180D3000080D3000603E80088
:101AF0001B0037000348A30017003A000600E0006F
:101B0000170034000603E9000D00A30000004800A0
:101B10008180480002014900838149000348A300F5
:101B20000F003A000600E000090034000603E90057
:101B30000000400081804800020149008381490083
:101B400001003A000003EB000348A300F5FF320058
:101B50006022B80002003700848272006182660051
:101B6000EC00070003F0A1000CF0A70003F0A000B8
:101B7000E3003700640147006408E10002003A0016
:101B80000DF8A300DB003A003200BE001201BE00D7
:101B9000DB0037001400FA00889FBE008A9FBE0059
:101BA0008C9FBE000004BE000205BE006800470016
:101BB0000A90BE000890BE002B0107000070A7002D
:101BC0000BF0A1000BF8A30020003A009E09900042
:101BD0000E099000FE0090006E0090009E029000A2
:101BE0003443200084825200C50032000A003C00C9
:101BF000B4FC2F000428E100140034008301D1005C
:101C00000281D3008180D3000080D3008502E800E8
:101C1000FAFF3A00BA003700B40020000428E100BF
:101C200007003C000000400081804800020149009C
:101C3000838149008502E900FAFF3A00B0003700CD
:101C40000300280002002000010037006011B800E6
:101C50006000B800AA0037002800FA00889FBE0084
:101C60008A9FBE008C9FBE0003866B009000070019
:101C70006400E100440032006408E1004A003200E0
:101C80006100E100460032006108E10049003200D5
:101C9000EC0647006000B8003D02BE003D03BE00F8
:101CA000F48657006011B8003D04BE003D05BE003B
:101CB0007D0320000B0037000000A0008D06E90026
:101CC000130032000402420085824A0006034B00E2
:101CD00087834B00000040008180480002014900DA
:101CE000838149000802520089825A000A035B007E
:101CF0008B835B00F0FF3B000802420089824A00B0
:101D00000A034B008B834B008D06E900EDFF3A0080
:101D10008482720086827200F707B20087827200A6
:101D200001003200150020001E0490003E0B9000C0
:101D300006035400E63FB0000368A300070032002A
:101D40000000A7000500A0008301D1000281D3009C
:101D50008180D3000080D3000603E8008301D10016
:101D60000281D3008180D3000080D3000002EB0009
:101D70000482D2006700070003F0A1000CF0A70066
:101D800003F0A0005E003700640247006408E10031
:101D9000580032003400BE003401BE00F6FF3700A8
:101DA0006108E100530032006011B8006000B80023
:101DB000F1FF370003FF270002002000FBFF370080
:101DC000889FBE00830478000300E0002C003500EB
:101DD00003003C0000827000040271002600320003
:101DE00036432000C50020008383CF000A0039005D
:101DF0000541B1008283CF00070039000541B100E1
:101E00008183CF00040039000541B1008083CF00F9
:101E1000010039000541B10085C353006022B800BC
:101E2000120032000A003B008482720061026000EE
:101E30008301D1000281D3008180D3000080D300D0
:101E40000603E8008743E800F7FF3A000700370081
:101E50000000400081804800020149008381490060
:101E60000603E9008743E900F9FF3A00290007006B
:101E700009F0A70003F0A0004F04BE000000060018
:101E800060001000E080180060011900E081190076
:101E9000D3FF3B00033E2C00F7FF370007F0A20002
:101EA000BFFE37004F89DE0082017800C4FF370093
:101EB000680447000294BE000094BE00FC04470082
:101EC0008694BE008494BE00090078006600070076
:101ED000080078006400070099007800814F7000C6
:101EE0000B003B000800BE00930007004F00B1004C
:101EF00003003700F3FF2700F2FF2F006110B90045
:101F00004F06BE004F05BE004F04BE000080FA0021
:101F100000000600180020005700200008045300AD
:101F20000D003D000600200097FC2F000740E10057
:101F30001E00340084827200610260008301D100BF
:101F40000281D3008180D3000080D3000804E80020
:101F5000F8FF3A00470020006104600005047400A7
:101F6000040464000D00320061004000E08048007D
:101F700060014900E081490003B8A5000700320074
:101F80000603E8006538E10004003A008301D1004F
:101F90000281D3008180D3000080D300F87F20002D
:101FA0000830E10003003500080378006000B80045
:101FB0006011B8004433DD00F300B2008301730008
:101FC00000000600889FBE008A9FBE008C9FBE0056
:101FD0000404BE000605BE00809FBE00829FBE00B6
:101FE00063000700040678000800BE000A01BE0076
:101FF0005F000700840678004F03BE004F02BE005A
:102000008D4F76007FB0970013003300F0FF2F0054
:102010008B8F6B0006003B000D0666000C00A700CE
:102020000A00370007F0A600100020000A00370061
:10203000880F5200898F5A008A0F5B008B8F5B00DC
:10204000030039001000200001003E0000002000C5
:1020500007F0A7000000EA004F06BE004F05BE00D3
:102060004F04BE0000000600800078005002BE0051
:102070005003BE004439DE00F700B200F37F2000B9
:1020800003016100090032000218E10016003A0065
:1020900085017200830173008381730000082000B2
:1020A00015003A004000200013003700850172003F
:1020B000830173008381730005003A0004A8BE0009
:1020C00006A8BE00100020000B0037000201E90046
:1020D0000402420085824A0006034B0087834B00BE
:1020E0000748A300F9FF32000740A00004A8BE0083
:1020F00006A8BE00200020008000980092009800F2
:10210000000006000003BE00DFFC07006220E100C3
:10211000020032000600BE0005000500E507B10020
:10212000F107B20004F023008480700007F0A700DC
:1021300001F0A00024000500E48240001078A30014
:1021400007003200640240001178A3003400BE0092
:102150001401BE00040032000330A7000000060096
:102160003500BE001501BE000330A00000000600CF
:1021700005FF270005826100070032000428E10006
:1021800001003200240005000600070001003A00AB
:10219000440005000408050002000700F9FF3A00AA
:1021A000140005006F8261008102700085027100D9
:1021B00085027200000006000400FA00E0BF9F00E4
:1021C000E4815700812978000002EB000F003700FE
:1021D0006FB89700904078007FB897001040780063
:1021E0000402E80080CF5000040032008180FB0030
:1021F0000080FB0000805000070037006FB8970098
:102200000000E800E0BF9F009309E800820F520041
:10221000EFFF3A000000EB000080FA00000006002B
:1022200010417800B141510003003A000000E8007D
:102230000204E000FAFF3A000300FB000000060081
:102240008001780000017800314078000059780062
:102250000004E000FCFF3A000300780000000600E4
:102260008001EB0002003700817178008301E800F3
:10227000828F5100FCFF3A00000006000000FA00C7
:10228000CFB89700688157006E0407000080FA00FD
:1022900000000600810178000000E9000081EB00E9
:1022A000E50F500004003E00800040002055210052
:1022B0006081780003B0780002007800000006001A
:1022C000000178000000E900E50F50000F003E001B
:1022D0008000400020552100E08078000100E000EF
:1022E00002003A0010002000B4000700E18F400017
:1022F000060032000000EB00E18F500004003200C5
:102300000200780001000100000005000080EB00E1
:102310000000060010002000E9FF07001000200068
:10232000A6000700800278008001780001003700D5
:102330008301E8001304E000FDFF3A000002EB0017
:10234000820F52000600320064C078008059780085
:102350000402E8000004E00002003200F8FF370049
:102360008049EB000500780000000600810178003C
:102370000002EB000B003700E44078000104E000AD
:10238000030032000402E80093CF50000400320042
:102390008180FB001380FB000080500000000600DD
:1023A0008301E800820F5200F3FF3A0000000500AD
:1023B0000C00FA00A0BF9F00C0BF9F000A000700EA
:1023C000B0BF9F00F0BF9F00100C2000D0BF9F0047
:1023D00074815700EFB097006C805700F40107003C
:1023E0000080FA0000000600800078003004E00061
:1023F000FEFF3A00010050000000E9000000060066
:1024000010417800814F5100040032000000E800C4
:102410000204E000FAFF3A000000EB0000000600B2
:102420008001EB000200370061F079008301E800D1
:10243000828F5100FCFF3A0000000600889FBE001A
:102440008A9FBE008000780000C2B3000100370000
:10245000890078008104780039447800804F540066
:10246000FBFF3200E94F5400F9FF3200D0C2B30045
:10247000804F540004003A00194478008184E80039
:102480001AC0B300060037000045EB00B0C2B3002D
:10249000804F540002003A00194478008184E8001B
:1024A0006022B8000A003700A200200003002000CC
:1024B0000400BE0046F907000B4144000281FB0006
:1024C0000300200000024100818249003944780065
:1024D0000880FB000BFD2F000B004000E90F5000AF
:1024E000F1FF36000A04E000020032006002120030
:1024F000E0821A000400BE004F05BE004F04BE007B
:1025000000000600000378008002780002027800D4
:102510008001EB00080037000402E90063C0780086
:10252000805A78008301E8000004E00002003A00CD
:102530008000EB0006003700828F5100F6FF3A0062
:10254000FBFF37000040EB0080F07A008100E800DC
:10255000848F5000FBFF3A00060078000000060060
:102560000C00FA00889FBE0000047800CFB09700EE
:10257000F0FF2700D0BF9F008004EB0099BF9F00B1
:1025800088BF9F00A8BF9F00200C2000B0BF9F0005
:102590007881570070805700AA0307000FB8970092
:1025A000094878000FB89700080450000800780028
:1025B0004F04BE000080FA0000000600000478000E
:1025C000E50807000800780052F80700889FBE0061
:1025D000000478008144780000FD2F0000004400D2
:1025E000E90F500002003E00000178000D003700A6
:1025F0000800780028F807000000E000030032001F
:10260000080078002AF80700000478000800780025
:102610002EF807000000E0000700320090FA2F00BB
:10262000000144000980FB00800F510002003D00C2
:102630000280FB0001003700F00F20004F04BE00B5
:1026400000000600881F780020AB8000D00807003B
:102650000004780027F807000000E000FAFF3A00C5
:10266000E10F44000300320021AB80000800780035
:10267000FB0807004F04780000000600EC874700C5
:10268000889FBE008A9FBE008C9FBE008E1F780070
:1026900081BF9F000207780020AB88008046EB00D6
:1026A000040137008884FB000900780011F8070056
:1026B000800078000000E00002003200E1FF070027
:1026C000FC00370050C2B300804F5400F0003A00C5
:1026D0000FBD970020C0B300C0EF9F00D1EF9F0057
:1026E00081EF9F000300370040C0B300C0EF9F00A0
:1026F0000FBD97000FB99700B240780082BF9F00CE
:102700008184FB0090C6B30080CF500035003200BA
:1027100017003E006640500080CF5000620032003B
:102720000C003E007740500080CF5000280032005F
:1027300006003E000104E0009B003200A0C2B3008E
:1027400080CF50006E003A001D00370080C5B300F6
:102750001600370040C6B30080CF50002100320081
:102760006440400080CF500065003A0012003700FE
:1027700030C7B30080CF50001E00320007003E007B
:102780006740500080CF500011003200634040008D
:1027900080CF50005A003A001400370050C7B300F1
:1027A00080CF50000F0032006340400080CF5000C7
:1027B00053003A006500370020C0B300CBFF37005C
:1027C000DFE897008140E800D1EF9F00C8FF3700A5
:1027D0004FE9970080C0B300E24F5100C3FF3A00B9
:1027E000C1FF3700ACC0B300590037008CC0B30044
:1027F0005700370093FF0700DFE897000104E0006F
:1028000002003A004E017800D2B79F0020AB800052
:102810005F08070000047800E10F4000A2003200CA
:102820008FEC9700120037000A85E8008ABF9F00EE
:10283000160037008FB897001100FB00800F54007E
:10284000F9FF32005FE997000204E00003003A005C
:102850005FB0970008587800D0B79F008944E9001E
:102860000A00320020AB800049080700000478000D
:102870000800E800E10F500004003600080078006E
:102880009CF707000000E000EAFF3200DFE8970055
:102890000104E00087003A008D46E8005FB1970030
:1028A00001497800830037005FE897000004E000EA
:1028B00003003A008D46E800CE007800D1B79F00B3
:1028C00020AB800032080700E10F400076003200A4
:1028D0005FE997000204E00003003A00DFB09700D0
:1028E00080587800D1B79F000FE997000241E900B6
:1028F00082EF9F004240A9006E003400F0FF3700D5
:102900000180FB0008FD2F0008004000E90F500087
:102910005F003E000A0078006E08070080EF9F000D
:1029200088007800030037000FB897000000E80027
:1029300080BF9F000FB997001200FB00010040000C
:10294000E90F5000F8FF360069FF37000CC1B300F3
:102950003CFF070020AB80000D0807000005780051
:102960000040EB00E0EF9F00D0022000800F5500F8
:1029700005003A0020AB800005080700000578003C
:1029800011C0B300E1EF9F008C4078000A0078008E
:102990000EFF0700E14F40000A003A0021AB800023
:1029A0000A0078002E0807000D04E0004B003A00F2
:1029B00020AB8000300090000048A30043003200AC
:1029C000480037008FED97006044B8000C81FB0091
:1029D000030020000800BE00FDF707000004BE0051
:1029E0008C4078000A007800F8FE07000080FB00A9
:1029F0000100200008044000898448008B45E9005C
:102A00000700320020AB8000E107070000057800D6
:102A10008C407800EDFE0700E14F4000EBFF3A00EC
:102A20008C4078000A007800E8FE0700E14F400083
:102A300003003A0021AB80000A0078000808070074
:102A40006FE997000204E000020032006004140005
:102A5000E0841C005FE897000004E00015003A00E5
:102A60008D46E800CFE89700E4CF500003003A001D
:102A70004E0078000888BE000E0037000E81E90085
:102A80000207780012007800080878000900370073
:102A900020AB8000BE070700808F54000500320085
:102AA000E10F40000B003A000D04E0000D00320081
:102AB0000A0037008FB897003144780081BF9F002B
:102AC0000804E000F7FE3A00040037000000EB00C5
:102AD0000500370021AB8000E10707000D80FB00F7
:102AE000010037000080EB004F0778004F06BE0062
:102AF0004F05BE004F04BE00CF00B100000006002D
:102B0000889FBE00000478008144780000FD2F00FB
:102B100000004400E90F500002003E000001780070
:102B20000D00370008007800DBF607000000E00029
:102B30000300320008007800DDF60700000478008A
:102B400008007800E1F607000000E000070032000E
:102B500090FA2F00000144000980FB00800F510013
:102B600002003D000280FB0001003700F00F200052
:102B70004F04BE0000000600881F780030AB8000C4
:102B80008307070000047800DAF607000000E00081
:102B9000FAFF3A00E10F44000300320031AB80003D
:102BA00008007800AE0707004F0478000000060018
:102BB0008F04B000889FBE008A9FBE008C9FBE001D
:102BC0008E1F780081BF9F008206780030AB88009E
:102BD0000040EB00E0EF9F00AF0137008884FB006E
:102BE00009007800C3F60700800078000000E000CC
:102BF00002003200E0FF0700A701370050C2B30017
:102C0000804F540092013A000FBD970022C0B300DC
:102C1000C2EF9F00D1EF9F0001477800030037000B
:102C200041C0B300C1EF9F000FBD97000FB99700DF
:102C3000B240780082BF9F008184FB0070C6B30061
:102C400080CF50001D003E0000C0E90080CF500042
:102C50003A0031007940500080CF5000B600320079
:102C60000E003E006740500080CF5000330032001D
:102C700006003E000104E000280032007B405000C6
:102C800080CF5000FB003A002800370070C4B3002A
:102C900080CF5000F7003A002800370030C6B3005C
:102CA00080CF5000DD003200A9003E006B40500094
:102CB00080CF5000EF003A0011013700F0C6B3009A
:102CC00080CF5000A400320008003E006640500053
:102CD00080CF50009E0032000E003900634040005B
:102CE00080CF5000E3003A009300370050C7B30094
:102CF00080CF5000960032006340400080CF5000EB
:102D0000FF0032006540500080CF5000D9003A00EB
:102D10009300370020C0B3008B003700EFE8970026
:102D20000104E000F3003A000F0137005FE997006B
:102D30000241E800D2EF9F00BBFF37008EFF070083
:102D40000E04E00001003A00BEC3B30030AB8000C7
:102D50000F07070000017800D0022000800F51000B
:102D600005003200C0FA2F000F004000D0B79F00CE
:102D70000044EB0014003700C1FA2F008F804000A0
:102D800082587800D1B79F0030AB80000007070061
:102D9000000178000E47E900F5FF37005FB09700AB
:102DA00002587800D0B79F00E0022000800F510049
:102DB00001003A000844E80030AB8000F406070048
:102DC000000178000E47E9000E04E0000400320024
:102DD00000FD2F0000004100E90F5000EFFF36001A
:102DE0000804E00003003A00E0022000800F5100D8
:102DF000EAFF32000E04E0002D00320050062000F1
:102E0000800F51000300320050042000800F510059
:102E100027003A005FB49700025C780030AB800076
:102E2000DB060700000178008E44E90002003A004A
:102E3000D8B79F001E003700D0022000800F51003D
:102E4000050032000080E900800F510002003200CE
:102E5000D8B79F0012003700024C7800DFB097000F
:102E60008180E800D1B79F0030AB8000C806070022
:102E7000000178008EC4E900070037005FB09700BA
:102E800002587800D0B79F0030AB8000C006070022
:102E9000000178008944E9000904E00004003200E0
:102EA00000FD2F0000004100E90F5000F3FF360045
:102EB000DFB097008048EB00E10F410003003200D3
:102EC00031AB800002007800E50607005FB1970093
:102ED000C0FA2F000F004000800F510004003A009C
:102EE000EFE897000104E000F5003A009E0037008B
:102EF0005FE997000204E000E7003A006FE89700FE
:102F00000040E800E0EF9F000D81E900CFE8970066
:102F1000E2CF5000D8003E0082067800120478000C
:102F20008000EB00C0FA2F000F0040000D070700E3
:102F3000008CBE00D80037004FE99700E24F5100E7
:102F400037FF320080C0B300C0EF9F0036FF37006C
:102F5000ACC0B3006B0037008CC0B3006900370011
:102F600005FF0700DFE897000104E00002003A00D7
:102F70004D017800D2B79F0030AB80008406070077
:102F800000047800E10F4000530032008E447800C6
:102F9000120037000A85E8008ABF9F00160037003C
:102FA0000FB997001200FB00800F5400F9FF3200A8
:102FB0005FE897000004E00003003A00DFB09700EC
:102FC00088587800D1B79F008944E9000A00320090
:102FD00030AB80006E060700000478000800E800AF
:102FE000E10F50000400360008007800C1F507002A
:102FF0000000E000EAFF32005FE997000204E00011
:10300000A5003A006FE897000040E800E0EF9F005D
:10301000DFB09700824878009F0037005FE9970093
:103020000204E00005003A006FE897000040E80065
:10303000E0EF9F00CD007800D1B79F0030AB80005B
:1030400053060700E10F400087003200DFE89700D9
:103050000104E00003003A005FB1970000597800D6
:10306000D2B79F000E47E9004240A9008A00340011
:10307000F2FF37000180FB0008FD2F000800400030
:10308000E90F50000E003E000A007800910607008C
:103090000047780088007800030037000FB89700D9
:1030A0000000E80080BF9F000FB997001200FB00EE
:1030B00001004000E90F5000F8FF3600DAFE37004B
:1030C00030AB800032060700808F5400720032005F
:1030D000E10F400005003A006FE897000004E000AF
:1030E0007A003200804078007600370031AB8000F3
:1030F0005B0607006FE997000280FB007400370051
:103100000CC1B3009CFE070030AB80002006070016
:10311000000578000040EB0080EF9F00D002200007
:10312000800F550005003A0030AB800018060700FC
:103130000005780011C0B30081EF9F008C4078003B
:103140000A0078006EFE0700E14F40000B003A00D5
:1031500031AB80000A007800410607006FE9970054
:103160000204E000E3FF3A0030AB80003000900042
:103170000048A3004E003200540037008E4578000E
:103180006044B8000C81FB00030020000800BE0072
:103190000FF607000004BE008C4078000A0078009B
:1031A00057FE07000080FB000100200008044000DB
:1031B000898448008B45E9000700320030AB80006D
:1031C000F3050700000578008C4078004CFE0700EE
:1031D000E14F4000EBFF3A008C4078000A00780095
:1031E00047FE0700E14F400003003A0031AB80008A
:1031F0000A0078001A0607000FE897000004E000B4
:103200000200320060041400E0841C00DFE8970034
:103210000104E00020003A006FE997000241E80055
:10322000E2EF9F004FE89700E44F500003003A00A0
:103230004D0078000888BE00170037000D81E900B6
:103240008206780012007800080878001200370023
:1032500030AB8000CE050700808F54000E00320096
:10326000E10F400014003A006FE997000204E0000B
:1032700016003200A0FF37008206780012047800A2
:103280008000EB00C0FA2F000F0040002907070064
:10329000009CBE000294BE000FB897003044780036
:1032A00080BF9F000804E0004CFE3A000400370095
:1032B0000000EB000600370031AB8000E805070096
:1032C000EFE897000180FB00010037000080EB0071
:1032D0004F0778004F06BE004F05BE004F04BE00EA
:1032E0008F04B10000000600889FBE008A1F78008E
:1032F000804078000004E00021003D008040EA00AA
:10330000D0C6B30080CF5000090034008104FB0018
:1033100042062000110009008204D8000001780054
:10332000010078004311DD002A3021001F00370022
:103330000100FB002330210039003700A2002000EB
:10334000110009000200D800000178000100780097
:103350004311DD00030141004300DD000300400094
:103360003002BE002003BE0042209000D220900018
:10337000F221900062219000B8F807002E0037007B
:10338000D0C6B30080CF5000230034008104FB007E
:1033900042062000110009008204D80000017800D4
:1033A000010078004311DD002A3B21000A014100A1
:1033B000A8002000110009000800D8004300DD002B
:1033C0000A00400040229000D0229000602390002C
:1033D000F02390000288900092889000B2899000BB
:1033E000228990009DF80700801F78000102780074
:1033F000110009008804D8000102FD004F00780088
:103400000402FB004322DD000A0242005403BE0016
:103410004402BE00D8FF37000100FB00233B21001F
:10342000EACF5000C5FF3C004300DD000300400030
:103430005001BE004000BE004F0578004F04BE00A2
:10344000000006008F03B000889FBE008A9FBE0068
:103450008C9FBE008E1F7800E0B79F00F1B79F00E1
:1034600082BF9F000000EB00A0B79F00E60437007A
:103470008001EB0050C2B30080CF50000900320041
:103480000100FB00EFB09700EC040700E10F4000E3
:10349000DD043200AFB097008100E800A1B79F00C3
:1034A000D90437007FB1970092407800D0C2B300B2
:1034B00080CF50000C00320007003C006D405000EF
:1034C00080CF50000D0032006B40400080CF500094
:1034D00019003A000E00370000C3B30080CF50003F
:1034E00015003A000F0037000330A0007FB29700AC
:1034F0000402E800F4B79F00EAFF37000300A000D1
:10350000FFB297008502E800F5B79F00E5FF37009E
:103510000310A0007FB697000C06E800FCB79F00E0
:10352000E0FF37000320A0007FB097000000E80014
:10353000F0B79F00DBFF37000318A3000100320043
:103540000300A1000338A300010032000320A10002
:103550000100FB0002FD2F0002004000E90F5000B7
:1035600010003E008000EB00C1B79F00020278000F
:103570004FB197006A10B900FFB297001501FB0028
:103580000001410004014100C2B79F005500FB004B
:10359000F5B79F0004004000E90F50000D003E0009
:1035A000F3FF37000006EB00CCB79F00A0C2B300CA
:1035B00080CF500007003A000FB89700C000780095
:1035C00080BF9F00C1B79F007FB197000201E80054
:1035D000F2B79F00E0C2B3007FB29700944F100093
:1035E00021003A00830678000DE0A0008400E80086
:1035F00064405000914F100004003200F1B79F006A
:103600008002EB00B5B79F00100037000FBE970097
:103610004C0078008CBF9F00B0B79F00FFB09700B0
:103620008180E800F1B79F00130037003FB2970098
:103630006A20B9000000410003004000B0B79F00BD
:10364000FFB297008502E800F5B79F007FB69700AC
:103650001C01FB0003FD2F0003004100E90F500097
:10366000F2FF360004003700830678000DC0A0008A
:103670000000EB00B0B79F007FB19700B240780028
:10368000F2B79F00C17F9F00C0C6B30080CF50003B
:103690002700320014003C006840500080CF5000EA
:1036A0009D00320009003C006C40500080CF50006B
:1036B000290032006B40400080CF50007200320081
:1036C0000104E000560432008E00370060C6B300EB
:1036D00080CF50001C0032006340400080CF50007B
:1036E00088003A008C00370030C7B30080CF50000C
:1036F0001C00320007003C006440500080CF5000A6
:10370000130032000040E80080CF50007D003A00F6
:103710001100370050C7B30080CF50007D00320049
:103720006340400080CF500076003A000B00370025
:10373000000028000D48A30001003A00000120000D
:1037400080867600CCFF37000DA0A0007200370005
:103750000D60A000700037000D50A0000D70A0009B
:103760006D0037008FB997004300780083BF9F003A
:10377000000478000000E00001003A002850210019
:103780008004EB00010037008104E8008900780024
:10379000088044001004E000FBFF3A003FB29700AD
:1037A0000400E00003003200890F520001003100E4
:1037B000840478000007EB00CFB29700898F520095
:1037C00001003600098752004368DE00E106600010
:1037D00019003A000D06780009003700EFB0970095
:1037E0000002200015040700E10F40000300320032
:1037F0002FB097000000E800A0B79F000C06E8007B
:103800008E0F5600F5FF3A000087EB000A003700E4
:10381000880078003100FB0001047800EFB09700C9
:1038200006040700E10F400003003200AFB097002C
:103830008100E800A1B79F000900E900800478003A
:10384000E10F4000F2FF3A000006EB000D00E0003F
:103850000A003A00EC033700EFB0970000022000A6
:10386000F6030700E10F4000030032002FB197007C
:103870000201E800A2B79F000C06E8008E0F560078
:10388000F5FF3A00E00337008FB997004300780056
:1038900083BF9F00CF80DE000101780082017800A5
:1038A0000205BE000004BE000203BE000002BE000E
:1038B0004822DE00482EDD0004027600C47F9F000F
:1038C0000D48A3000A0032000404E00008003200A2
:1038D000E14F420006003200D1FB2F00018047007B
:1038E00004487800184098002900200002003700A2
:1038F000D07F9F0019002000D2FB2F0002844700D8
:10390000A6FF3700C3FB2F000384470019002000E7
:10391000A2FF37000D0CB30000702000008266008B
:10392000270232000DC8A30002003200640020000C
:10393000B4B79F000D48A300050032000FBA9700EE
:103940004401BE004400BE0084BF9F000400370055
:103950008FBA97004500BE0085BF9F00B4F70700EF
:10396000E0AF9F00F1AF9F0082B79F0093B79F0029
:103970006022B8006033B8006FA89700FFA89700D6
:103980000FB197009FB19700C8F707000000E00053
:103990000A003D006FA89700FFA897000FB197009D
:1039A0009FB1970003F0A200E0AF9F00F1AF9F002E
:1039B00082B79F0093B79F003D00B3000000EB006B
:1039C00080A79F006022B8006033B8006FA89700FE
:1039D000FFA897000FB197009FB19700B8F70700B5
:1039E0000000E000340032006FA89700FFA89700A5
:1039F0000FB197009FB19700B6F7070003FC2F00A7
:103A000003814700DEF707000FA097000000E900E0
:103A10006300B900A2002000110009000200D800D4
:103A20008000FD0081A79F000100E00002003D0032
:103A30000100E90080A79F000FA497000840EA005A
:103A400029FE07006FAA9700FFAA97000FB39700FF
:103A50009FB3970001F70700A0AF9F00B1AF9F0091
:103A6000C2AF9F00D3AF9F006022B80006002000C5
:103A700007FF23008DF707000000E00002003D0073
:103A80000800E9000B0037006022B80006002000A3
:103A9000470224002FA89700BFA897004FA99700BE
:103AA000DFA99700B9F707000000E0000200350029
:103AB0000800E80080A79F003FB29700F80F52006F
:103AC00057003C00D0C6B300804F5200290036009A
:103AD0000485FB0042062000110009000285D80081
:103AE00000017800010478004311DD002B30210033
:103AF0000B0141006022B8000600200007FE2300F1
:103B00000288900092889000B289900022899000EB
:103B1000D2F60700A9002000809FBE001100090016
:103B20000984D800000478004F00BE004344DD0043
:103B30000B04440048229000D82290006823900093
:103B4000F8239000C5F60700801F78000102780076
:103B5000110009000985D8000102FD004F0078001E
:103B60004322DD000B0242005403BE004402BE00AB
:103B70001F0037000480FB0029302100EA4F52006B
:103B800014003600A2002000110009000280D800B5
:103B900000017800010478004311DD0009014100B3
:103BA0006022B8000600200007FE2300422090009B
:103BB000D2209000F221900062219000A7F6070029
:103BC0004344DD00090444003802BE002803BE005F
:103BD000070037004300DD00090040006022B80004
:103BE0000600200007FE23005001BE004000BE007A
:103BF0009AF607000002BE000203BE006FA89700FD
:103C0000FFA897000FB197009FB1970064F70700D6
:103C1000E0AF9F00F1AF9F0082B79F0093B79F0076
:103C20000FA49700E90F540015003C006022B80073
:103C30006033B8006FA89700FFA897000FB19700F6
:103C40009FB197001EF707000000E000320032002D
:103C50006FA89700FFA897000FB197009FB197003A
:103C6000CCF70700E00F5000E08F5800E00F59003C
:103C7000E08F590028003A00E10F5400260034007C
:103C80000400200005002E00B6E0220017012400E9
:103C90002FA89700BFA897004FA99700DFA997000A
:103CA00002F707000000E00002003D00730054002E
:103CB000010037007200540080A79F000FC09700DA
:103CC00089FD0700A0AF9F00B1AF9F00C2AF9F006A
:103CD000D3AF9F000002BE000203BE006FA8970092
:103CE000FFA897000FB197009FB19700DAF7070080
:103CF000A8F707000205BE000004BE006000B8007F
:103D00006011B800A0A79F00B1A79F00C2A79F00A5
:103D1000D3A79F002E0037006FA89700FFA8970039
:103D20000FB197009FB197009AF707000205BE00F8
:103D30000004BE00E00F5000E08F5800E00F590073
:103D4000E08F5900020035001DF80700130037000E
:103D500010002000010020006011B8000800600081
:103D6000898060000A0161008B8161008B03D100B2
:103D70000A83D3008982D3000882D3000000720036
:103D80008180720002017300838173000CF80700C8
:103D90000002BE000203BE0001F707000002BE00E1
:103DA0000203BE006FA89700FFA897000FB197000D
:103DB0009FB1970039F80700A0A79F00B1A79F0007
:103DC000C2A79F00D3A79F000000EB0080A79F0021
:103DD00014C0B300254621000B0037000400FB008F
:103DE0004300DD00050040005001BE004000BE0061
:103DF0000040E10001C8E10002D0E10003D8E10089
:103E0000030039000442E800F44F5200F3FF3A0087
:103E1000C47F9F000400FB00BFB0970000804000FB
:103E20008FA09700010040004FB19700000751009C
:103E3000BFB197000300E000010032000E07E90067
:103E400063806600010032000E07E9000D28A30020
:103E500026003200E18066000D18A3000C0032003D
:103E6000D00220000100E00001003A000080E900DB
:103E7000EFB0970071020700E10F40001800320018
:103E80002FB297000402E800A4B79F001400370087
:103E90000100E00012003200EFB0970000022000A5
:103EA00066020700E10F40000D003200AFB297003C
:103EB0008502E800A5B79F0009003700EFB0970022
:103EC000000320005D020700E10F40000300320004
:103ED0002FB697000C06E800ACB79F000E07E9006C
:103EE0000E00E000F5FF3C003D0037000D38A30058
:103EF0000A0032000B003700EFB0970000022000EC
:103F00004E020700E10F4000030032002FB097007F
:103F10000000E800A0B79F000E07E9000E00E000D7
:103F2000F5FF3C00E18066000D18A3000C00320094
:103F3000D00220000100E00001003A000080E9000A
:103F4000EFB097003D020700E10F4000240032006F
:103F5000AFB097008100E800A1B79F0020003700B4
:103F60000100E0001E003200EFB0970000022000C8
:103F700032020700E10F4000190032002FB1970014
:103F80000201E800A2B79F00150037000000FB0007
:103F90004300DD0021462100010040003002BE0048
:103FA0002003BE000800BE000A01BE008AF407001C
:103FB000A4002000050020006033B8008DF4070045
:103FC0000003B000EFB097001C020700E10F4000B3
:103FD00003003200AFB197008301E800A3B79F0050
:103FE0004F7A97000440E900C07F9F00E14F4000F6
:103FF000E6FF3A000B003700EFB097000003200007
:104000000E020700E10F400003003200AFB297003C
:104010008502E800A5B79F000FA097000000E90007
:1040200080A79F000FA097000000E000F2FF3C0077
:104030003FB6970020C1B300F20F560001003C00CC
:104040006FE09700C07F9F00CF7897000100FB00D2
:104050003FB1970000005100E0A79F000104E0007D
:1040600008003200EFB09700E0022000F3010700E3
:10407000E10F400003003200AFB197008301E80078
:10408000A3B79F004F78970097FC07000002BE007F
:104090000203BE002FA09700BFA097004FA197007A
:1040A000DFA197006DF50700BAF607001E00370084
:1040B0000000FB004300DD002C4621000C00400006
:1040C0003002BE002003BE000800BE000A01BE0090
:1040D00041F40700A4002000050020006033B80070
:1040E00044F407000003B000EFB09700D3010700CD
:1040F000E10F4000030032002FB297000402E800F5
:10410000A4B79F00CF7A97000500FB004300DD00B5
:104110000C0040003002BE002003BE000800BE00BC
:104120000A01BE0033F407000205BE000004BE0011
:104130004F7E97000C40E900C07F9F00E14F400098
:10414000DBFF3A000006EB0009003700EFB09700F4
:1041500000032000B9010700E10F40000300320016
:104160002FB097000000E800A0B79F000C06E80001
:10417000EFA09700810F5600F4FF3A000D38A3001E
:10418000A10132000E00E0009F0134000006EB00A8
:10419000EFB0970000022000A8010700E10F4000E7
:1041A000030032002FB197000201E800A2B79F0080
:1041B0000C06E8008E0F560093013200F4FF370022
:1041C0000D007800000CB20028003A000D00E0005D
:1041D00005003D008FB997004305BE004304BE00B3
:1041E00083BF9F00140037000D48A3000B0032006E
:1041F0000FBA97004400BE0084BF9F004F89DE00C5
:10420000CF91DE000002BE00020378008203780036
:104210000605BE000404BE00070037008FBA9700F1
:104220004500780085BF9F0000047800CFC4DE0001
:10423000090578008A057800E00F5400E08F5C00E3
:10424000E00F5D00E08F5D0020003D003D00B30009
:104250006000B8006011B80008045000898458005C
:104260000A0559008B855900180037000D00E00041
:1042700005003D000FBE97004C05BE004C04BE007B
:104280008CBF9F00110037000D48A30008003200CA
:104290008FBA97004500BE0085BF9F0004017800DB
:1042A000840178000205BE000004BE00070037004C
:1042B0000FBE97004C0078008CBF9F000004780070
:1042C000090020000A0020000B0020003FB09700EA
:1042D0000000E00007003A00E00F5400E08F5C00AF
:1042E000E00F5D00E08F5D0002003A001100200049
:1042F000B1B79F000D0778000E0CB200000420003B
:10430000800F57002F00320003003C000E00E00039
:10431000070032003F00370000082000800F5700E0
:1043200014003200000C2000800F570039003A00C2
:1043300014C0B300254621000B0037000400FB0029
:104340004300DD00050040005001BE004000BE00FB
:104350000040E10001C8E10002D0E10003D8E10023
:104360002B0039000442E800F44F5200F3FF3A00FA
:104370002700370000012000010020006011B80074
:1043800014C0B3000040E10001C8E10002D0E10028
:1043900003D8E1001E003900450020000000D000D5
:1043A0008180D2000281D2008381D2008502E9009F
:1043B000FAFF3A000442E800F04F5200F1FF3A00E1
:1043C0001300370080002000010020006011B800B9
:1043D00014C0B3000040E10001C8E10002D0E100D8
:1043E00003D8E1000A0039003C0020000000D000A2
:1043F0008180D2000281D2008381D2000C06E900C4
:10440000FAFF3A000442E800F54F5200F1FF3A008B
:10441000C47F9F00CF7897000100FB003FB1970059
:10442000820F500002003D00C27F9F000400370051
:10443000BFB19700808F510001003D00B0B79F00D1
:104440004FB297000400E000040032006380660071
:10445000020032000402E900C4B79F000DE8A30087
:104460000B003200CFB297003FB697008C8F5200FE
:1044700003003C000000EB00C0B79F0004003700C1
:10448000CFB097003FB1970082805000C1B79F0026
:10449000CF7997000300FB000002EB0094A79F0078
:1044A000CFB29700808F520002003400008052008B
:1044B00090A79F000D28A30037003200E18066001E
:1044C0000D18A3000C003200D00220000100E00013
:1044D00001003A000080E900EFB09700D700070024
:1044E000E10F40000E0032002FB697000C06E800E6
:1044F000ACB79F000A0037000100E000080032005E
:10450000EFB0970000022000CC000700E10F400050
:10451000030032002FB097000000E800A0B79F0012
:104520009FA097000100E0000F0032000006EB00A2
:10453000EFB0970000032000C0000700E10F40002B
:10454000030032002FB197000201E800A2B79F00DC
:104550000C06E8009FA19700830F5600F4FF3A0075
:104560000002EB0094A79F00BFB29700C328DD00B4
:10457000A04521008080400091AF9F004228DD00CF
:104580006400500080AF9F006328B900F0A79F002F
:1045900063065000820037001FA697000C00E00061
:1045A00011003200688066000F003A0000067800B3
:1045B000EFB0970000022000A0000700E10F4000CC
:1045C000030032002FB097000000E800A0B79F0062
:1045D0000C06E8009FA09700810F5600F4FF3A00F8
:1045E0000001EB0092A79F00E18066000D18A30078
:1045F0000C003200D00220000100E00001003A006F
:104600000080E900EFB097008C000700E10F400048
:10461000D5FF3200AFB197008301E800A3B79F0038
:10462000D1FF37000100E000CFFF3200EFB097006C
:104630000002200081000700E10F4000CAFF3200A5
:104640002FB297000402E800A4B79F00C6FF37000E
:1046500000042000800F57003000320003003C00AF
:104660000E00E000070032003D0037000008200087
:10467000800F570011003200000C2000800F5700FF
:1046800037003A001FA897003002BE002003BE008A
:104690000800BE000A01BE00CFF20700A4002000FF
:1046A000050020006033B800D2F2070004C3B30055
:1046B00004424000C47F9F0029003700955021002C
:1046C000D5B79F000D58A30002003A00A051210069
:1046D000D0B79F0014002000050020006033B80010
:1046E0008FA897008100E900050033000402D00084
:1046F0008582D2000683D2008783D200F9FF37007B
:104700000800BE000A01BE00B3F207006F0060009F
:104710005FB197006240780010003700140020005D
:10472000050020006033B8008C0178008301E900A7
:10473000050033000402D0008582D2000683D20037
:104740008783D200F9FF37000800BE000A01BE00CF
:10475000A1F20700674060000043B000C07F9F00E7
:104760004F7A97000400FB00EFB09700330007007A
:10477000E10F400003003200AFB297008502E8006D
:10478000A5B79F001FA897006800500090AF9F003A
:104790008FA89700E480500081AF9F006306560009
:1047A000D0FF2F003FB197000090B900FFA1970004
:1047B0000080410063005000800F5600A4FF3A00C3
:1047C0000D38A300100032001FA297000400E00083
:1047D0000D0034000006EB00EFB09700000220004F
:1047E00016000700E10F400003003200AFB297004F
:1047F0008502E800A5B79F000C06E8001FA09700FF
:10480000800F5600F4FF3A007FB19700B240780065
:10481000F2B79F00C17F9F000104E00014FB3A0043
:104820002FB097004F0778004F06BE004F05BE001F
:104830004F04BE008F03B10000000600889FBE0039
:104840000001780001047800B10090000118A30075
:104850003D0032000198A30003003A0018009000C8
:104860000000E00038003A000190A00031049800F8
:1048700082047800F90FB200180090000000E000F8
:1048800002003A0028009000000C7800EA8F5400E3
:1048900006003A00380090000078A30003003A00B8
:1048A00088007800D0002000E4FF07009800900006
:1048B00058009000808F50000B0032000100E8008B
:1048C000100498001800780009587800000C78004F
:1048D00011C0B3002056210001487800EA8F54002F
:1048E000060032001900370088007800094078007F
:1048F000F4020700800478001400370038009000AC
:104900000088A3001100320018019000A800900058
:104910004800900087EF070098009000810F50003A
:1049200004003200380090000003B3003004980007
:104930008084EB000000EB00100498002800900039
:10494000000C7800010037008084EB00090078003B
:104950004F04BE0000000600881F780040AB8000B6
:104960000000E0000100320000000100E8522100D8
:1049700008007800160307006C044400205521004D
:10498000800F5400FAFF3A004F0478000000060040
:10499000881F780000047800B00090000148A30050
:1049A00007003A000108A300050032000198A300A7
:1049B00008003200100090000000E0000500320006
:1049C000380090000040A000300498008080EB0088
:1049D000200037000190A1003104980018009000D9
:1049E0000000E000060034000000E9001004980018
:1049F00018007800B080FB00000C7800060037003B
:104A0000380090000068A300EDFF3A00080078002D
:104A10002703070080007800380090000078A3008A
:104A20000C003A00FA8F500008003A00280090006D
:104A30000000E000E2FF3200180090000000E800F3
:104A400010049800180CE900DDFF3700ED8F5000CE
:104A5000E2FF3200010078004F04780000000600F9
:104A600080017800E10F4000170032003100900013
:104A70000008A300140032000098A30012003A00BE
:104A8000210290000400E0000F00320011019000AC
:104A900051009000800F51000B003200110078008F
:104AA000840F500002003A008008E800020037003E
:104AB0000200E800900098001100E90080087800EA
:104AC00003487800010037008081EB000300780084
:104AD000000006000001780000C2B30001003700AA
:104AE0000201E8009240780080CF5000FCFF3200C5
:104AF000E9CF5000FAFF3200D0C2B30080CF50009F
:104B000003003A000201E80014C0B30005003700BA
:104B10000042EB00B0C2B30080CF500001003A0069
:104B20000201E8008000EB0005FD2F0004003700C3
:104B30006A08B90000804100850040000201E800D9
:104B40009201FB0005804100E90F5000F8FF36009C
:104B50000404E000010032008100EA000100780056
:104B600000000600E6874700889FBE008A9FBE00BF
:104B70008C9FBE008E1F78000004780081067800AC
:104B80000100E00003003200800E780001003700D1
:104B90000804E800984478000900FB00D5EE0700FF
:104BA000800078000000E000F9FF3A00D0C2B300B6
:104BB00080CF540003003A000804E8001BC0B30093
:104BC00005003700B0C2B30080CF540001003A00A6
:104BD0000804E800814578000005EB000A0778002A
:104BE0006000B800F0B79F0081BF9F000B48A30092
:104BF00005003A00E0C2B300984F100002003A00EE
:104C00000B44A0001E003700984478000900FB0008
:104C10000CFD2F000C004000E90F50001A003E0070
:104C20000B14A0000B00FB00E90F5500110032002F
:104C30000048A300010032000E07E9000A05E80061
:104C4000A2002000030020007FB097008FB89700DB
:104C50005FEF07000CC144000281FB00030020004D
:104C60000000410081804900F0B79F0081BF9F0094
:104C7000030037000048A30001003A000E07E800D7
:104C80000804E800D9FF370050C6B30080CF5400B5
:104C9000040032000002EB0050C4B30080CF540087
:104CA00032003A008801E80093407800D0C2B30097
:104CB00080CF500002003A000B34A0000300370000
:104CC000B0C2B30080CF500003003A008881E800F2
:104CD000010037008301E8009340780006C3B30069
:104CE00086CF5000FBFF32000100FB0005FD2F00C6
:104CF00005004000E90F500003003600030478006F
:104D00000002EB001600370006C050000082FB00D6
:104D10000304E800184178000200FB000500400091
:104D2000E90F50000E003E006A20B9000641510014
:104D30000281FB00000241000384E80098407800F3
:104D40000100FB0005004000E90F500004003E0098
:104D50006A21B90006C050000080FB00020240003A
:104D60000B38A300010032000402EA0004054700EA
:104D70000D00E000030032000B18A3000100320018
:104D8000880E78007FB097008FB897003AF0070040
:104D90000004BE000006BE006011B80061F007000C
:104DA0006011B8000000E0005900320030F82F0018
:104DB000800F550003003D002002200050AB88000A
:104DC0005300370000082000800F55000A0034000F
:104DD0002002200050AB88000B08A3000300320023
:104DE0000200200003F82F004900370002002000D5
:104DF00003F82700460037000A00E0001C003D00D1
:104E00000A05EA0006003700922F20005301250012
:104E10000800BE00D6EF07000004BE006A0555007A
:104E2000E90F5500F8FF3C000006EB0006003700D4
:104E300002002000031224000800BE00CCEF07008F
:104E40000004BE000C06E8008A0F5600F8FF3A0086
:104E50000806BE0002002000030820000800BE0073
:104E600030F007000000E00025003D001C00370086
:104E70000A00E00007003C0021003700922F2000CC
:104E8000530125000800BE0085EF07000004BE00A6
:104E90006A055500E94F5500F8FF3E000006EB009B
:104EA0000600370002002000031224000800BE00A4
:104EB0007BEF07000004BE000C06E8008A0F5600D6
:104EC000F8FF3A000806BE00F2FF2F00F3F72700B4
:104ED0000800BE00C4EE07000000E0000800340037
:104EE0000B08A30003003200020020000308280082
:104EF00007003700020020000308200004003700EC
:104F00000B08A300010032000DF0A2000C01BE004E
:104F10000200BE004F0778004F06BE004F05BE00DE
:104F20004F04BE006F00B100000006008000EB00DF
:104F30000CFF3700F0874700889FBE008A9FBE00A5
:104F40008C9FBE008E1F78000006780081BF9F00F6
:104F50000100E00003003200800878000100370003
:104F60000C06E8001C4478000800FB00E1ED070097
:104F7000800078000000E000F9FF3A00D0C2B300E2
:104F8000804F540003003A000C06E8001EC0B30036
:104F900005003700B0C2B300804F540001003A0052
:104FA0000C06E800014778000000EB00A0B79F0066
:104FB000B0B79F006000B8006011B800C0B79F0094
:104FC000D1B79F00E2B79F00F3B79F000E48A30040
:104FD00005003A00E0C2B3009C4F100002003A0006
:104FE0000E44A000300037009C4678000D00FB0006
:104FF0000003B100E90F50002D003E000E14A00088
:105000000E00FB002FB19700F20F5100210032007B
:105010000048A30003003200BFB197008301E900FC
:10502000B3B79F002FB097000000E800A0B79F0023
:105030006022B80006002000470224004FB097000D
:10504000DFB097006FB19700FFB1970083F10700C1
:105050000004BE000205BE0001CDB30001C0460041
:105060000080FB00CF80DE008EF307000002BE0050
:105070000203BE000800BE000A01BE0048F207009D
:10508000C0B79F00D1B79F00E2B79F00F3B79F0062
:10509000050037000048A30003003A003FB1970025
:1050A0000201E800B2B79F000C06E800C7FF370016
:1050B00050C6B30080CF5600040032000002EB005F
:1050C00050C4B30080CF560032003A008C01E80093
:1050D00093407800D0C2B30080CF500002003A0065
:1050E0000E34A00003003700B0C2B30080CF5000E0
:1050F00003003A008C81E800010037008301E800DA
:105100009340780006C3B30086CF5000FBFF320007
:105110000100FB0005FD2F0005004000E90F5000D5
:1051200003003600030678000002EB00160037008B
:1051300006C050000082FB000306E8001C41780016
:105140000200FB0005004000E90F50000E003E0089
:105150006A20B900064151000281FB0000024100B3
:105160000386E8009C4078000100FB000500400039
:10517000E90F500004003E006A21B90006C050004B
:105180000080FB00020240000E38A3000100320044
:105190000402EA00BFB19700848641000FB897006F
:1051A0000000E000030032000E18A30001003200EE
:1051B0000C0878004FB09700DFB097006FB19700F0
:1051C000FFB197000004BE000205BE006022B800D7
:1051D0006033B800B5F107006022B8006033B80052
:1051E0000000E000AD00320030C02F00808F56007C
:1051F00003003D002002200050AB8800A7003700CC
:1052000000402000808F56000E0034002002200055
:1052100050AB88000E08A30005003200F4FF2F00F9
:10522000F5FF2F00F6FF2F00F7FE2F009B00370041
:10523000F4FF2F00F5FF2F00F6FF2F00F7FE2700E9
:10524000960037000D00E00042003D000D04EA002A
:105250000E003700D4372C0045592200D69A24007E
:10526000274B25004FB09700DFB097006FB1970034
:10527000FFB1970078F20700C0B79F00D1B79F0039
:10528000E2B79F00F3B79F004806B1003006200048
:10529000800F5400EFFF3C000E0037000400200098
:1052A00005002200F6052A00272024004FB09700B1
:1052B000DFB097006FB19700FFB1970066F207006B
:1052C000C0B79F00D1B79F00E2B79F00F3B79F0020
:1052D0006A045400E90F5400F0FF3C008004EB0026
:1052E0000D0037006022B8000600200047022400AD
:1052F0004FB09700DFB097006FB19700FFB19700F4
:1053000055F20700C0B79F00D1B79F00E2B79F00DA
:10531000F3B79F008904E800888F5400F1FF3A003A
:105320004FB09700DFB097006FB19700FFB19700C3
:105330000004BE000205BE006022B8000600200086
:105340000701200059F107000000E0004E003D0079
:10535000430037000D00E0000F003C004A0037001A
:10536000D4372C0045592200D69A2400274B25001B
:105370004FB09700DFB097006FB19700FFB1970073
:10538000B6F00700C0B79F00D1B79F00E2B79F00FB
:10539000F3B79F004D06B10030062000808F560005
:1053A000EFFF3C000E003700040020000500220043
:1053B000F6052A00272024004FB09700DFB09700A1
:1053C0006FB19700FFB19700A4F00700C0B79F002E
:1053D000D1B79F00E2B79F00F3B79F00EA8656005F
:1053E000E9CF5600F0FF3E000004EB000D0037004F
:1053F0006022B80006002000470224004FB097004A
:10540000DFB097006FB19700FFB1970093F00700EE
:10541000C0B79F00D1B79F00E2B79F00F3B79F00CE
:105420000804E8008D0F5400F1FF3A004FB09700D8
:10543000DFB097006FB19700FFB197000004BE0086
:105440000205BE00F4FF2F00F5FF2F00F6FF2F002E
:10545000F7FE27004DF107000000E0000A003400CD
:105460000E08A300040032006022B80006002000ED
:1054700007012800090037006022B800060020005C
:1054800007012000050037000E08A30001003200CC
:105490000BF0A2000802BE000A03BE000400BE001A
:1054A0000601BE004F0778004F06BE004F05BE0044
:1054B0004F04BE000F01B100000006008000EB00A9
:1054C0009CFE37000200FA00889FBE00A0FF9F00EC
:1054D00001047800B1009000810478000904B20052
:1054E000020032000000FB00360037000118A30064
:1054F00005003A000103B300310498001904980034
:105500000080EB002F003700580090000000E00002
:1055100006003A004800900012002000E680570084
:1055200084EC07001904980024003700280090003C
:105530000000E00008003A00E05521002004980037
:10554000000C7800200020005004980010049800FF
:105550000130A0003104980018019000A8009000CC
:105560004800900073EC070028009000000C7800C1
:105570000080EB001004980018007800AFF8970046
:1055800001587800000C78002FF89700EA4F50007F
:105590000A003A00380090000088A300070032009B
:1055A00018019000A80090004800900061EC0700EE
:1055B00019049800A8009000010C7800AFF897003B
:1055C0000100FB004F04BE000080FA00000006004E
:1055D000889FBE008A1F7800000478003000900089
:1055E0006300600024003200080078007E0007009D
:1055F0003805900080EF2F0000006500300498000F
:10560000280090000000E00004003200E80465007B
:1056100002003A00AD0007002904980048009000FD
:105620007BEC0700E10F400013003200B80090004F
:105630000102B20010003A000AC8A30018003200AC
:1056400070AB80000000E00015003200000178001F
:1056500081047800012A200012289000880F500051
:10566000070032004205B0004905B000818F5400A8
:105670000B003200F8FF37000080EB000900370014
:10568000020078006BEC070070AB8000090040005E
:105690008000EB001128980001007800010037001D
:1056A0000000EB004F0578004F04BE00000006002C
:1056B0000200FA00889FBE008A1F7800000478006C
:1056C0000000EB0010049800380090008080EB0090
:1056D0000008A3003F003200205621001004E00023
:1056E00010003200E95221004A5321001A007800CC
:1056F0006C0545002010B20021102000810F5000E1
:1057000002003A000900780037000700EC844400EA
:1057100020552100808F5400F4FF3A0020562100CC
:105720000048EB0048009000580190000200E000A3
:105730000D003A001204980012002000E880570083
:1057400045EC0700E10F500003003A000FF8970006
:105750008080FB001F003700380090000040A00050
:105760003004980012003700A80090003AEC0700BF
:10577000100498000000E00003003200E10F400038
:105780000D003A0003003700380090000040A000F0
:1057900002003700380090000003B3003004980086
:1057A000A8009000010C78000000EB0010049800A5
:1057B0008080EB0007003700A8009000010C780003
:1057C0000000E9001004980001007800B080FB00A0
:1057D000000C7800010078004F0578004F04BE00EF
:1057E0000080FA0000000600881F7800000478009E
:1057F000300090000008A30007003200800078000D
:105800000120B20004003A0011049800A8009000A2
:10581000010C7800170037000018A30019003200AF
:105820000098A30017003200A80090000100E000DB
:1058300014003200180190000200E0001100320054
:1058400048009000BBEB070098009000810F5000CB
:1058500003003200380090000003B30030049800C9
:105860000000EB001004980028009000000C780065
:10587000380090000058A300020032000080EB00C6
:10588000010037000000EB004F0478000000060024
:1058900061AB80000100E0000300320011007800DD
:1058A00060AB8800030037002000200023EC0700D5
:1058B00080007800E18F400002003A00906E2600E0
:1058C00050AB8800010078000000060061AB80004A
:0C58D0000108780060AB880000000600B2
:020000040000FA
:0200000401F009
:04000C00FBFF0000F6
:020000040000FA
:0200000401F009
:04001000FDFF0000F0
:020000040000FA
:0200000401F009
:040014007FFF00006A
:020000040000FA
:10000800480300007ABE00004ABE000062BE00003D
:1000180092BE0000AABE000048030000480300008A
:100028004803000022D00000480300006AE10000F5
:10003800480300004803000048030000480300008C
:10004800DABE0000480300004803000012DF000089
:10005800480300004803000048030000480300006C
:10006800480300004803000048030000480300005C
:10007800480300004803000048030000480300004C
:1000880048030000480300004803000066C200005F
:10009800FCC200004803000056C8000048030000E6
:1000A800480300004803000048030000480300001C
:1000B800480300004803000048030000480300000C
:1000C80048030000480300004803000048030000FC
:1000D8004803000048030000C2BE000048030000B7
:1000E80048030000480300004803000048030000DC
:1000F80048030000480300004803000048030000CC
:1001080048030000480300004803000048030000BB
:1001180048030000480300004803000048030000AB
:10012800480300004803000048030000480300009B
:10013800480300004803000048030000480300008B
:10014800480300004803000048030000480300007B
:10015800480300004803000048030000480300006B
:10016800480300004803000048030000480300005B
:10017800480300004803000048030000480300004B
:10018800480300004803000048030000480300003B
:10019800480300004803000048030000480300002B
:1001A800480300004803000048030000480300001B
:1001B800480300004803000048030000480300000B
:1001C80048030000480300004803000048030000FB
:1001D80048030000480300004803000048030000EB
:1001E80048030000480300004803000048030000DB
:0801F800480300004803000069
:020000040000FA
:10020800480300007ABE00004ABE000062BE00003B
:1002180092BE0000AABE0000480300004803000088
:100228004803000022D00000480300006AE10000F3
:10023800480300004803000048030000480300008A
:10024800DABE0000480300004803000012DF000087
:10025800480300004803000048030000480300006A
:10026800480300004803000048030000480300005A
:10027800480300004803000048030000480300004A
:1002880048030000480300004803000066C200005D
:10029800FCC200004803000056C8000048030000E4
:1002A800480300004803000048030000480300001A
:1002B800480300004803000048030000480300000A
:1002C80048030000480300004803000048030000FA
:1002D8004803000048030000C2BE000048030000B5
:1002E80048030000480300004803000048030000DA
:1002F80048030000480300004803000048030000CA
:1003080048030000480300004803000048030000B9
:1003180048030000480300004803000048030000A9
:100328004803000048030000480300004803000099
:100338004803000048030000480300004803000089
:100348004803000048030000480300004803000079
:100358004803000048030000480300004803000069
:100368004803000048030000480300004803000059
:100378004803000048030000480300004803000049
:100388004803000048030000480300004803000039
:100398004803000048030000480300004803000029
:1003A8004803000048030000480300004803000019
:1003B8004803000048030000480300004803000009
:1003C80048030000480300004803000048030000F9
:1003D80048030000480300004803000048030000E9
:1003E80048030000480300004803000048030000D9
:0803F800480300004803000067
:020000040000FA
:1058DC006865000061640000657200002E690000BC
:1058EC006E630000006600006F6F000074650000BE
:1058FC00722E0000696E000063000000214400005D
:10590C0045460000000D00000A00000074780000FD
:10591C0074000000687400006D00000068740000E2
:10592C006D6C0000006300006769000000780000E7
:10593C006D6C0000006300007373000000670000D2
:10594C0069660000007000006E670000006A0000CD
:10595C0070670000006300006C61000000770000BD
:10596C006176000000000000000000000000000054
:10597C008CAC000090AC000094AC000099AC000022
:10598C009DAC0000A1AC0000A5AC0000A9AC0000CF
:10599C00ADAC0000B1AC0000B5AC0000B9AC00007F
:1059AC0074650000787400002F7000006C610000BA
:1059BC00696E00000074000065780000742F000010
:1059CC00687400006D6C00000074000065780000C5
:1059DC00742F0000786D00006C00000074650000EE
:1059EC00787400002F6300007373000000690000DE
:1059FC006D610000676500002F670000696600009C
:105A0C00006900006D610000676500002F700000E8
:105A1C006E670000006900006D61000067650000A2
:105A2C002F6A0000706500006700000061700000C4
:105A3C00706C00006963000061740000696F000005
:105A4C006E2F00006A610000766100002D76000068
:105A5C006D00000061750000646900006F2F00008C
:105A6C00782D0000776100007665000000000000D2
:105A7C00D6AC0000E1AC0000E1AC0000E1AC0000F1
:105A8C00EBAC0000F4AC0000FDAC000007AD000076
:105A9C0011AD00001CAD000030AD00003DAD0000AC
:105AAC0048540000545000002F3100002E310000EB
:105ABC002032000030300000204F00004B0D000061
:105ACC000A4300006F6E00006E65000063740000F6
:105ADC00696F00006E3A0000206300006C6F0000DC
:105AEC00736500000D0A00000048000054540000CB
:105AFC00502F0000312E0000312000003430000007
:105B0C00302000004261000064200000526500005B
:105B1C007175000065730000740D00000A430000ED
:105B2C006F6E00006E65000063740000696F00000A
:105B3C006E3A0000206300006C6F0000736500007B
:105B4C000D0A00000D0A0000343000003020000067
:105B5C004261000064200000526500007175000075
:105B6C0065730000743A000020630000616E000051
:105B7C002774000020680000616E0000646C000057
:105B8C0065200000436F00006E740000656E00001D
:105B9C00742D00004C6500006E67000074680000F6
:105BAC000D0A00000048000054540000502F000063
:105BBC00312E000031200000343000003120000074
:105BCC00556E000061750000746800006F72000073
:105BDC00697A0000656400000D0A00005757000048
:105BEC00572D00004175000074680000656E0000C0
:105BFC007469000063610000746500003A200000C5
:105C0C0042610000736900006320000072650000AF
:105C1C00616C00006D3D000022500000726F0000AE
:105C2C00746500006374000065640000220D0000C0
:105C3C000A4300006F6E00006E6500006374000084
:105C4C00696F00006E3A0000206300006C6F00006A
:105C5C00736500000D0A00000D0A000034300000CE
:105C6C0031200000556E0000617500007468000062
:105C7C006F720000697A0000656400003A20000031
:105C8C005061000073730000776F000072640000B5
:105C9C0020720000657100007569000072650000DB
:105CAC00640D00000A00000048540000545000002D
:105CBC002F3100002E310000203400003034000061
:105CCC00204E00006F740000206600006F7500000D
:105CDC006E6400000D0A0000436F00006E6E000041
:105CEC0065630000746900006F6E00003A200000CC
:105CFC00636C00006F730000650D00000A43000028
:105D0C006F6E0000746500006E7400002D5400006E
:105D1C0079700000653A000020740000657800007E
:105D2C00742F0000687400006D6C00000D0A0000F8
:105D3C000D0A000034300000343A00002046000008
:105D4C00696C0000652000006E6F0000742000007C
:105D5C00666F0000756E0000643C0000627200000B
:105D6C003E55000073650000203C000061200000DF
:105D7C0068720000656600003D2200002F7500006F
:105D8C00706C00006F610000642200003E4D00004A
:105D9C005046000053200000557000006C6F00004E
:105DAC00616400003C2F0000613E00002074000084
:105DBC006F200000707200006F67000072610000BD
:105DCC006D2000007765000062200000706100000B
:105DDC0067650000730D00000A00000048540000C5
:105DEC00545000002F3100002E31000020340000F0
:105DFC003134000020520000657100007565000010
:105E0C00737400002D55000052490000205400000E
:105E1C006F6F0000204C00006F6E0000670D0000DB
:105E2C000A4300006F6E00006E6500006374000092
:105E3C00696F00006E3A0000206300006C6F000078
:105E4C00736500000D0A00000D0A000034310000DB
:105E5C00342000005265000071750000657300006D
:105E6C00742D00005552000049200000546F0000B2
:105E7C006F2000004C6F00006E6700003A2000009D
:105E8C00427500006666000065720000206F00001D
:105E9C0076650000726600006C6F000077200000D1
:105EAC0064650000746500006374000065640000A4
:105EBC000D0A00000048000054540000502F000050
:105ECC00312E000031200000353000003020000061
:105EDC00496E000074650000726E0000616C000079
:105EEC0020530000657200007665000072200000EF
:105EFC0045720000726F0000720D00000A43000032
:105F0C006F6E00006E65000063740000696F000026
:105F1C006E3A0000206300006C6F00007365000097
:105F2C000D0A00000D0A0000353000003020000082
:105F3C00496E000074650000726E0000616C000018
:105F4C00205300006572000076650000722000008E
:105F5C0045720000726F0000723A0000204500008C
:105F6C007870000065630000746500006420000018
:105F7C006461000074610000206E00006F7400000A
:105F8C002070000072650000736500006E740000E4
:105F9C000D0A00000048000054540000502F00006F
:105FAC00312E00003120000035300000312000007F
:105FBC004E6F000074200000496D0000706C0000F2
:105FCC00656D0000656E000074650000640D0000D6
:105FDC000A4300006F6E00006E65000063740000E1
:105FEC00696F00006E3A0000206300006C6F0000C7
:105FFC00736500000D0A00000D0A0000353000002A
:10600C00312000004E6F000074200000496D00002C
:10601C00706C0000656D0000656E0000746500001A
:10602C00643A0000204F00006E6C000079200000E4
:10603C004745000054200000616E00006420000001
:10604C00504F000053540000207300007570000086
:10605C00706F000072740000656400000D0A00008F
:10606C000048000054540000502F0000312E000056
:10607C003120000032300000302000004F4B000077
:10608C000D0A0000436F00006E6E00006563000097
:10609C00746900006F6E00003A200000636C000011
:1060AC006F730000650D00000A4300006F6E000066
:1060BC00746500006E7400002D54000079700000AF
:1060CC00653A00002074000065780000742F000011
:1060DC00687400006D6C00000D0A00000D0A0000D1
:1060EC003C680000746D00006C3E00003C620000D7
:1060FC006F6400007920000073740000796C00005C
:10610C00653D0000226D00006172000067690000AF
:10611C006E3A000031300000307000007822000030
:10612C003E3C0000666F0000726D0000206D0000A8
:10613C0065740000686F0000643D0000706F000023
:10614C00737400002061000063740000696F00002C
:10615C006E3D0000222F0000757000006C6F000077
:10616C006164000022200000656E00006374000072
:10617C0079700000653D0000226D0000756C000018
:10618C007469000070610000727400002F660000DA
:10619C006F7200006D2D00006461000074610000DE
:1061AC00223E00003C6200003E4D000050460000C4
:1061BC0053200000496D000061670000652000005D
:1061CC00557000006C6F0000616400003C2F0000F3
:1061DC00623E00003C7000003E3C0000696E000016
:1061EC007075000074200000747900007065000068
:1061FC003D660000696C0000652000006E610000C7
:10620C006D6500003D69000020730000697A000094
:10621C00653D0000343000003E200000266E00007A
:10622C0062730000703B0000203C0000696E0000AF
:10623C007075000074200000747900007065000017
:10624C003D730000756200006D6900007420000051
:10625C00766100006C750000653D00002255000061
:10626C00706C00006F610000642200003E3C000076
:10627C002F6600006F7200006D3E00003C2F000086
:10628C00626F0000647900003E3C00002F68000043
:10629C00746D00006C3E0000004800005454000077
:1062AC00502F0000312E0000312000003230000051
:1062BC00302000004F4B00000D0A0000436F00001F
:1062CC006E6E000065630000746900006F6E000064
:1062DC003A200000636C00006F730000650D000035
:1062EC000A4300006F6E0000746500006E740000BD
:1062FC002D54000079700000653A000020740000F5
:10630C0065780000742F0000687400006D6C00004C
:10631C000D0A00000D0A00003C680000746D0000BE
:10632C006C3E00003C6200006F64000079200000AD
:10633C0073740000796C0000653D0000226D000054
:10634C0061720000676900006E3A00003130000095
:10635C0030700000782200003E3C0000623E0000DD
:10636C004D500000465300002055000070640000A2
:10637C006174000065200000537500006363000029
:10638C006573000073660000756C00003C2F000004
:10639C00623E00003C7000003E3C000061200000AA
:1063AC0068720000656600003D2200002F2200008C
:1063BC003E53000069740000652000006D61000010
:1063CC00696E00002070000061670000653C0000F1
:1063DC002F6100003E3C00002F6200006F64000043
:1063EC00793E00003C2F0000687400006D6C0000CA
:1063FC003E00000048540000545000002F310000B3
:10640C002E31000020350000303000002049000003
:10641C006E740000657200006E6100006C2000005C
:10642C005365000072760000657200002045000084
:10643C00727200006F7200000D0A0000436F0000C2
:10644C006E6E000065630000746900006F6E0000E2
:10645C003A200000636C00006F730000650D0000B3
:10646C000A4300006F6E0000746500006E7400003B
:10647C002D54000079700000653A00002074000073
:10648C0065780000742F0000687400006D6C0000CB
:10649C000D0A00000D0A00003C680000746D00003D
:1064AC006C3E00003C6200006F640000792000002C
:1064BC0073740000796C0000653D0000226D0000D3
:1064CC0061720000676900006E3A00003130000014
:1064DC0030700000782200003E3C0000623E00005C
:1064EC004D50000046530000204900006D61000033
:1064FC0067650000204300006F7200007275000099
:10650C0070740000206F00007220000057720000B1
:10651C006F6E00006720000056650000727300006B
:10652C00696F00006E3C00002F6200003E3C0000D2
:10653C00703E00003C6100002068000072650000A5
:10654C00663D0000222F0000757000006C6F00008B
:10655C0061640000223E00005472000079200000AB
:10656C0061670000616900006E3F00003C2F000075
:10657C00613E00003C2F0000626F00006479000057
:10658C003E3C00002F680000746D00006C3E000063
:10659C000048000054540000502F0000312E000021
:1065AC00312000003330000032200000466F000024
:1065BC00756E0000640D00000A4300006F6E000051
:1065CC006E65000063740000696F00006E3A000095
:1065DC00206300006C6F0000736500000D0A000062
:1065EC004C6F000063610000746900006F6E000066
:1065FC003A2000000048000054540000502F0000C6
:10660C00312E000031200000343000003320000017
:10661C00466F00007262000069640000646500004F
:10662C006E0D00000A4300006F6E00006E650000E6
:10663C0063740000696F00006E3A00002063000074
:10664C006C6F0000736500000D0A00000D0A00005D
:10665C003430000033200000466F000072620000EE
:10666C0069640000646500006E3A0000205300006D
:10667C00534C000020520000657100007569000049
:10668C0072650000642000002D200000757300006E
:10669C00652000004854000054500000530D0000C9
:1066AC000A00000056AD000056AD00007BAD0000A6
:1066BC00D9AD00005AAE0000F4AE000061AF00008E
:1066CC00D1AF000037B000003DAD000053B1000069
:1066DC0000B20000CFB2000001B30000436F000015
:1066EC006F6B0000696500003A0000004175000006
:1066FC00746800006F720000697A00006174000019
:10670C00696F00006E3A0000004300006F6E0000DD
:10671C00746500006E7400002D4C0000656E000066
:10672C0067740000683A00000000000074B30000B9
:10673C007CB300008BB30000474500005400000000
:10674C00504F00005354000000750000706C0000A6
:10675C006F61000064000000696E00006465000059
:10676C00782E0000687400006D0000000D0A000017
:10677C000D0A000033300000342000005265000088
:10678C006469000072650000637400003A20000028
:10679C00004300006F6E0000746500006E74000012
:1067AC002D54000079700000653A000020000000B4
:1067BC00436F00006E740000656E0000742D0000C5
:1067CC00456E0000636F0000646900006E67000096
:1067DC003A200000677A0000697000000D0A000082
:1067EC000043000061630000686500002D43000059
:1067FC006F6E0000747200006F6C00003A20000095
:10680C00006E00006F2D00006361000063680000E3
:10681C00650000006D610000782D000061670000CC
:10682C00653D0000003600003030000000530000D1
:10683C00657400002D4300006F6F00006B69000051
:10684C00653A0000200000000D0A00000D0A00004F
:10685C00000D00000A0D00000A4D0000504600001B
:10686C005302000001000000705F00006170000026
:10687C00705F0000636F00006E66000069670000C7
:10688C0000730000726300002F4800007562000066
:10689C002F480000756200002E63000000250000E8
:1068AC00733A0000256900002025000073200000C9
:1068BC002D2D000020610000737300006572000034
:1068CC00746900006F6E00002066000061690000B2
:1068DC006C650000640A000000000000000000006D
:1068EC00000000000000000000000000000000009C
:1068FC00000000000000000000000000000000008C
:10690C00000000000000000000000000000000007B
:10691C00000000000000000000000000000000006B
:10692C00000000000000000000000000000000005B
:10693C00000000000000000000000000000000004B
:10694C00000000000000000000000000000000003B
:10695C00000000000000000000000000000000002B
:10696C00000000000000000000000000000000001B
:10697C00000000000000000000000000000000000B
:10698C0000000000000000000000000000000000FB
:10699C0000000000000000000000000000000000EB
:1069AC0000000000000000000000000000000000DB
:1069BC0000000000000000000000000000000000CB
:1069CC0000000000000000000000000000000000BB
:1069DC0000000000000000000000000000000000AB
:1069EC00000000000000000000000000000000009B
:1069FC00000000000000000000000000000000008B
:106A0C00000000000000000000000000000000007A
:106A1C00000000000000000000000000000000006A
:106A2C00000000000000000000000000000000005A
:106A3C00000000000000000000000000000000004A
:106A4C00000000000000000000000000000000003A
:106A5C00000000000000000000000000000000002A
:106A6C0000000000000000000046000069720000F9
:106A7C006D77000061720000652000003D20000071
:106A8C00257500002E250000752E000025750000D0
:106A9C00004C000045440000427200006967000091
:106AAC00687400006E65000073730000203D0000E8
:106ABC002025000075000000486100006E64000095
:106ACC0043740000726C0000203D00002025000083
:106ADC006400000057690000726500006449000002
:106AEC00502000003D200000256400002E250000F1
:106AFC00642E0000256400002E25000064000000B8
:106B0C000000000000000000000000000000000079
:106B1C000000000000000000000000000000000069
:106B2C000000000000000000000000000000000059
:106B3C000000000000000000000000000000000049
:106B4C000000000000000000000000000000000039
:106B5C000000000000000000000000000000000029
:106B6C000000000000000000000000000000000019
:106B7C000000000000000000000000000000000009
:106B8C0000000000000000000000000000000000F9
:106B9C0000000000000000000000000000000000E9
:106BAC0000000000000000000000000000000000D9
:106BBC0000000000000000000000000000000000C9
:106BCC0000000000000000000000000000000000B9
:106BDC0000000000000000000000000000000000A9
:106BEC000000000000000000000000000000000099
:106BFC000000000000000000000000000000000089
:106C0C000000000000000000000000000000000078
:106C1C000000000000000000000000000000000068
:106C2C000000000000000000000000000000000058
:106C3C000000000000000000000000000000000048
:106C4C000000000000000000000000000000000038
:106C5C000000000000000000000000000000000028
:106C6C000000000000000000000000000000000018
:106C7C000000000000000000000000000000000008
:106C8C0000000000000000000000000000000000F8
:106C9C00585F000052610000772000003D2000008A
:106CAC0025750000005900005F520000617700005C
:106CBC00203D00002025000075000000545F0000FE
:106CCC0052610000772000003D2000002575000077
:106CDC00004900006E6300005F4100007474000006
:106CEC006163000068650000642000003D20000026
:106CFC0025640000000000000000000000000000FF
:106D0C000000000000000000000000000000000077
:106D1C000000000000000000000000000000000067
:106D2C000000000000000000000000000000000057
:106D3C000000000000000000000000000000000047
:106D4C000000000000000000000000000000000037
:106D5C000000000000000000000000000000000027
:106D6C000000000000000000000000000000000017
:106D7C000000000000000000000000000000000007
:106D8C0000000000000000000000000000000000F7
:106D9C0000000000000000000000000000000000E7
:106DAC0000000000000000000000000000000000D7
:106DBC0000000000000000000000000000000000C7
:106DCC0000000000000000000000000000000000B7
:106DDC0000000000000000000000000000000000A7
:106DEC000000000000000000000000000000000097
:106DFC000000000000000000000000000000000087
:106E0C000000000000000000000000000000000076
:106E1C000000000000000000000000000000000066
:106E2C000000000000000000000000000000000056
:106E3C000000000000000000000000000000000046
:106E4C000000000000000000000000000000000036
:106E5C000000000000000000000000000000000026
:106E6C000000000000000000000000000000000016
:106E7C000000000000000000000000000000000006
:106E8C0000000000000000000000000000000000F6
:106E9C0000000000000000000000000000000000E6
:106EAC00000000000000000000000000004900008D
:106EBC00502000003D200000256400002E2500001D
:106ECC00642E0000256400002E25000064000000E4
:106EDC004D610000736B0000203D00002025000078
:106EEC00642E0000256400002E250000642E000096
:106EFC002564000000470000617400006577000005
:106F0C0061790000203D000020250000642E000067
:106F1C00256400002E250000642E0000256400006E
:106F2C0000500000726900006D6100007279000071
:106F3C00444E0000532000003D200000256400005A
:106F4C002E250000642E0000256400002E25000074
:106F5C006400000053650000636F00006E64000065
:106F6C0061720000794400004E530000203D000087
:106F7C0020250000642E0000256400002E25000052
:106F8C00642E0000256400000044000065660000CB
:106F9C00617500006C74000049500000203D000039
:106FAC0020250000642E0000256400002E25000022
:106FBC00642E00002564000000440000656600009B
:106FCC00617500006C7400004D610000736B000073
:106FDC00203D000020250000642E000025640000E8
:106FEC002E250000642E00002564000000440000E3
:106FFC0048430000502000003D20000025640000A4
:10700C00004E000065740000424900004F53000020
:10701C00203D000020250000730000004D410000C1
:10702C00432000003D2000002573000000000000FC
:10703C000000000000000000000000000000000044
:10704C000000000000000000000000000000000034
:10705C000000000000000000000000000000000024
:10706C000000000000000000000000000000000014
:10707C000000000000000000000000000000000004
:10708C0000000000000000000000000000000000F4
:10709C0000000000000000000000000000000000E4
:1070AC0000000000000000000000000000000000D4
:1070BC0000000000000000000000000000000000C4
:1070CC0000000000000000000000000000000000B4
:1070DC0000000000000000000000000000000000A4
:1070EC000000000000000000000000000000000094
:1070FC000000000000000000000000000000000084
:10710C000000000000000000000000000000000073
:10711C000000000000000000000000000000000063
:10712C000000000000000000000000000000000053
:10713C000000000000000000000000000000000043
:10714C000000000000000000000000000000000033
:10715C000000000000000000000000000000000023
:10716C000000000000000000000000000000000013
:10717C000000000000000000000000000000000003
:10718C0000000000000000000000000000000000F3
:10719C0000000000000000000000000000000000E3
:1071AC0000000000000000000000000000000000D3
:1071BC00000000000000000000000000004E000075
:1071CC00657700002048000075620000204900002F
:1071DC00502000003D200000256400002E250000FA
:1071EC00642E0000256400002E25000064000000C1
:1071FC004E650000772000004875000062200000FA
:10720C004D610000736B0000203D00002025000044
:10721C00642E0000256400002E250000642E000062
:10722C0025640000004E0000657700002048000037
:10723C007562000020470000572000003D20000030
:10724C00256400002E250000642E0000256400003B
:10725C002E250000640000004E6500007720000021
:10726C0048750000622000004448000043500000B4
:10727C00203D000020250000640000005345000064
:10728C00540000000000000000000000000000009E
:10729C0000000000000000000000000000000000E2
:1072AC0000000000000000000000000000000000D2
:1072BC0000000000000000000000000000000000C2
:1072CC0000000000000000000000000000000000B2
:1072DC0000000000000000000000000000000000A2
:1072EC000000000000000000000000000000000092
:1072FC000000000000000000000000000000000082
:10730C000000000000000000000000000000000071
:10731C000000000000000000000000000000000061
:10732C000000000000000000000000000000000051
:10733C000000000000000000000000000000000041
:10734C000000000000000000000000000000000031
:10735C000000000000000000000000000000000021
:10736C000000000000000000000000000000000011
:10737C000000000000000000000000000000000001
:10738C0000000000000000000000000000000000F1
:10739C0000000000000000000000000000000000E1
:1073AC0000000000000000000000000000000000D1
:1073BC0000000000000000000000000000000000C1
:1073CC0000000000000000000000000000000000B1
:1073DC0000000000000000000000000000000000A1
:1073EC000000000000000000000000000000000091
:1073FC000000000000000000000000000000000081
:10740C000000000000000000000000000000000070
:10741C00000000005365000072690000616C000000
:10742C00204E0000756D00006265000072200000A7
:10743C003D200000256C0000750000005468000021
:10744C00652000007265000063650000697600002D
:10745C0065640000206300006F6D00006D6100002A
:10746C006E6400002069000073200000666F00004D
:10747C00726D0000617400007465000064200000EF
:10748C00696E0000636F000072720000656300009B
:10749C00746C000079000000546800006520000046
:1074AC007265000063650000697600006564000089
:1074BC00206300006F6D00006D6100006E640000C1
:1074CC002077000061730000207400006F6F0000D3
:1074DC00206C00006F6E0000670000005468000014
:1074EC00652000007265000063650000697600008D
:1074FC0065640000206300006F6D00006D6100008A
:10750C006E640000206300006F6E00007461000068
:10751C00696E000065640000206900006E76000052
:10752C00616C000069640000207000006172000052
:10753C00616D00006574000065720000730000004E
:10754C00546800006520000072650000636500004F
:10755C006976000065640000206900006465000025
:10756C006E740000696600006965000072200000FE
:10757C0077610000732000006E6F00007420000023
:10758C0072650000636F0000676E0000697A00008E
:10759C006564000000540000686500002063000072
:1075AC006F6D00006D6100006E64000020720000C1
:1075BC0065630000656900007665000064200000CA
:1075CC007761000073200000666F000072200000DD
:1075DC00616E0000206900006E760000616C000096
:1075EC00696400002074000061720000676500008F
:1075FC00742000006465000076690000636500007B
:10760C000054000068650000206300006F6D0000EE
:10761C006D6100006E6400002069000073200000A2
:10762C00696E0000766100006C6900006420000047
:10763C006265000063610000757300006520000046
:10764C007468000065200000646500007669000025
:10765C00636500002069000073200000686F000063
:10766C006D6900006E670000005400006865000042
:10767C00206300006F6D00006D6100006E640000FF
:10768C002069000073200000696E00007661000024
:10769C006C6900006420000077680000696C0000D1
:1076AC00652000006E6F000020740000656D000006
:1076BC007065000072610000747500007265000056
:1076CC0020700000726F00006265000020690000ED
:1076DC007320000061740000746100006368000096
:1076EC00656400002E000000546800006174000006
:1076FC0020640000657600006963000065200000CE
:10770C007479000070650000206400006F65000053
:10771C00732000006E6F000074200000657800007C
:10772C0069730000742E00000045000072720000A6
:10773C006F72000020740000657800007420000057
:10774C006E6F000074200000646500006669000024
:10775C006E65000064000000556E00006162000060
:10776C006C650000207400006F200000636F000047
:10777C006E6E00006563000074200000746F0000E2
:10778C00205700006946000069200000426F00008D
:10779C0061720000640000004E650000772000005C
:1077AC0057690000466900002073000065740000F2
:1077BC00746900006E6700007320000061720000A5
:1077CC0065200000696E0000636F0000727200009B
:1077DC006563000074000000546800006520000020
:1077EC00636F00006D6D0000616E0000642000008E
:1077FC0066610000696C0000656400002062000096
:10780C006563000061750000736500002074000062
:10781C00686500002061000078690000732000009A
:10782C00697300002064000069730000636F00003E
:10783C006E6E00006563000074650000640000005B
:10784C005468000065200000636F00006D6D00003F
:10785C00616E00006420000066610000696C00002D
:10786C006564000020620000656300006175000023
:10787C007365000020740000686500002072000031
:10788C006F740000617400006F72000020690000CA
:10789C007320000064690000736300006F6E0000C9
:1078AC006E65000063740000656400000054000005
:1078BC0068650000206300006F6D00006D610000C2
:1078CC006E64000020660000616900006C650000B9
:1078DC0064200000626500006361000075730000A5
:1078EC0065200000746800006520000061780000CD
:1078FC006973000020690000732000006E6F0000A7
:10790C0074200000686F00006D65000064000000CA
:10791C005468000065200000636F00006D6D00006E
:10792C00616E00006420000066610000696C00005C
:10793C006564000020620000656300006175000052
:10794C007365000020740000686500002072000060
:10795C006F740000617400006F72000020690000F9
:10796C00732000006E6F000074200000686F000030
:10797C006D650000640000000000000000000000C5
:10798C0000000000000000000000000000000000EB
:10799C0000000000000000000000000000000000DB
:1079AC0000000000000000000000000000000000CB
:1079BC0000000000000000000000000000000000BB
:1079CC0000000000000000000000000000000000AB
:1079DC00000000000000000000000000000000009B
:1079EC00000000000000000000000000000000008B
:1079FC00000000000000000000000000000000007B
:107A0C00000000000000000000000000000000006A
:107A1C00000000000000000000000000000000005A
:107A2C00000000000000000000000000000000004A
:107A3C00000000000000000000000000000000003A
:107A4C00000000000000000000000000000000002A
:107A5C00000000000000000000000000000000001A
:107A6C00000000000000000000000000000000000A
:107A7C0000000000000000000000000000000000FA
:107A8C0000000000000000000000000000000000EA
:107A9C0000000000000000000000000000000000DA
:107AAC0000000000000000000000000000000000CA
:107ABC0000000000000000000000000000000000BA
:107ACC0000000000000000000000000000000000AA
:107ADC00000000000000000000000000000000009A
:107AEC00000000000000000000000000000000008A
:107AFC00000000000000000000000000000000007A
:107B0C000000000000000000000000000000000069
:107B1C0000000000000000004375000072720000BD
:107B2C00656E000074540000656D0000702000004C
:107B3C003D20000025730000004E00006F20000067
:107B4C00507200006F620000650000004375000079
:107B5C0072720000656E00007453000074650000C2
:107B6C00702000003D200000256C00007500000016
:107B7C0054610000726700006574000053740000CB
:107B8C0065700000203D0000202500006C75000091
:107B9C0000490000734D00006F760000696E000014
:107BAC00672000003D200000257500000049000002
:107BBC00734800006F6D0000696E000067200000C4
:107BCC003D200000257500000049000073480000AE
:107BDC006F6D000065640000203D00002025000052
:107BEC0075000000546500006D70000050720000BC
:107BFC006F620000652000003D200000257500002C
:107C0C0000520000656D00006F74000065490000B3
:107C1C004F2000003D2000002575000000480000AA
:107C2C004353000074610000747500007320000061
:107C3C003D20000025750000004800006F6D00001D
:107C4C006553000077690000746300006820000031
:107C5C003D20000025750000000000000000000021
:107C6C000000000000000000000000000000000008
:107C7C0000000000000000000000000000000000F8
:107C8C0000000000000000000000000000000000E8
:107C9C0000000000000000000000000000000000D8
:107CAC0000000000000000000000000000000000C8
:107CBC0000000000000000000000000000000000B8
:107CCC0000000000000000000000000000000000A8
:107CDC000000000000000000000000000000000098
:107CEC000000000000000000000000000000000088
:107CFC000000000000000000000000000000000078
:107D0C000000000000000000000000000000000067
:107D1C000000000000000000000000000000000057
:107D2C000000000000000000000000000000000047
:107D3C000000000000000000000000000000000037
:107D4C000000000000000000000000000000000027
:107D5C000000000000000000000000000000000017
:107D6C000000000000000000000000000000000007
:107D7C0000000000000000000000000000000000F7
:107D8C0000000000000000000000000000000000E7
:107D9C0000000000000000000000000000000000D7
:107DAC0000000000000000000000000000000000C7
:107DBC0000000000000000000000000000000000B7
:107DCC0000000000000000000000000000000000A7
:107DDC000000000000000000000000000000000097
:107DEC000000000000000000004E0000696300006D
:107DFC006B6E0000616D0000652000003D200000EE
:107E0C0025730000004D00006178000053740000E1
:107E1C0065700000732000003D200000256C000000
:107E2C007500000044650000766900006365000081
:107E3C005479000070650000203D000020250000F2
:107E4C0063000000424C0000436F00006D700000A6
:107E5C004F6E0000203D0000202500007500000042
:107E6C00424C0000436F00006D7000005374000022
:107E7C0065700000732000003D2000002575000097
:107E8C00004800006F6D0000654F00006E5300004D
:107E9C007461000072740000203D00002025000079
:107EAC0075000000736500006E640000436D0000F7
:107EBC00640000006178000069730000312E00003E
:107ECC00687400006D0000006E650000747700009F
:107EDC006F7200006B2F0000636F00006E66000075
:107EEC00696700002E680000746D000000690000D6
:107EFC0070000000677700000073000075620000DE
:107F0C00006400006E73000031000000646E00001D
:107F1C007332000000640000686300007000000011
:107F2C002F6E000065740000776F0000726B00000C
:107F3C002F720000656200006F6F0000742E00004D
:107F4C00687400006D3F0000002F00006E6500009B
:107F5C00747700006F7200006B2F0000636F0000DD
:107F6C006E660000696700002E680000746D0000EA
:107F7C000063000068650000636B0000656400002E
:107F8C00006200006C6F0000636B0000006E00006C
:107F9C006F6E000065000000000000000000000093
:107FAC0000000000002500006C75000000000000BF
:107FBC0000000000000000000000000000000000B5
:107FCC0000000000000000000000000000000000A5
:107FDC00000000000000000000000000256600000A
:107FEC000000000000000000000000000000000085
:107FFC000000000000000000000000000000000075
:10800C000000000000000000000000000000000064
:10801C000000000000000000000000000000000054
:10802C00000000000000000000000000747200005E
:10803C007565000000660000616C0000736500004F
:10804C000000000000000000000000000000000024
:10805C000000000000000000000000000000000014
:10806C000000000000000000000000000000000004
:10807C0000000000000000000000000000000000F4
:10808C0000000000000000000000000000000000E4
:10809C0000000000000000000000000000000000D4
:1080AC0000000000000000000000000000000000C4
:1080BC00000000000000000025750000000000001A
:1080CC0000000000000000000000000000000000A4
:1080DC000000000000000000000000000000000094
:1080EC000000000000000000000000000000000084
:1080FC000000000000000000000000000000000074
:10810C000000000000000000000000000000000063
:10811C00000000000000000000250000752E00008B
:10812C00257500002E2500007500000000000000E1
:10813C000000000000000000000000000000000033
:10814C000000000000000000000000000000000023
:10815C000000000000000000000000000000000013
:10816C000000000000000000000000000000000003
:10817C0000000000000000000000000000000000F3
:10818C0000000000000000000000000000000000E3
:10819C0000000000000000000000000000000000D3
:1081AC0000000000000000000000000000000000C3
:1081BC0000000000000000000000000000000000B3
:1081CC0000000000000000000000000000000000A3
:1081DC000000000000000000000000000000000093
:1081EC000000000000000000000000000000000083
:1081FC000000000000000000000000000000000073
:10820C000000000000000000000000000000000062
:10821C000000000000000000000000000000000052
:10822C000000000000000000000000000000000042
:10823C00000000004574000068200000536F00002F
:10824C00636B00006574000020440000697300003B
:10825C00636F00006E6E0000656300007420000008
:10826C00436F0000756E0000743A0000203D000062
:10827C0020250000750000004574000068200000F7
:10828C00536F0000636B0000657400002043000016
:10829C006F6E00006E6500006374000020430000E8
:1082AC006F7500006E7400003A2000003D20000045
:1082BC002575000000450000746800002042000095
:1082CC00797400006573000020520000783A0000B9
:1082DC00203D0000202500006C750000000000000F
:1082EC0047450000544400004E4E0000004700007B
:1082FC004554000053540000410000004745000065
:10830C005443000046470000004400004F48000062
:10831C00414C000054000000534500005444000040
:10832C004E4E0000004D00004F5600004142000030
:10833C00530000004D4F0000564100004E47000016
:10834C00004400004F4800004F4D00004500000065
:10835C00434500004E5400004552000000530000FD
:10836C004554000042430000450000005345000006
:10837C0054420000435300000053000045540000D9
:10838C00484F0000530000005245000053450000C8
:10839C0054460000005300004554000044450000C2
:1083AC00560000004D4F0000564500005746000097
:1083BC00004600004F5200004345000048000000FA
:1083CC00464F00005243000045500000004400009E
:1083DC004F4D00004F560000450000004E69000054
:1083EC00636B00006E6100006D650000203D0000B5
:1083FC0020000000256C00007500000025660000C0
:10840C0000250000750000004745000054430000A3
:10841C004647000000530000455400004C45000046
:10842C00440000004745000054440000424700004F
:10843C0000520000454200004F4F00005400000065
:10844C00524500005345000054480000004700000E
:10845C0045540000484900005000000053450000FE
:10846C0054530000495000000053000045540000D4
:10847C00485300004D0000005345000054480000D4
:10848C0053470000005300004554000048530000BF
:10849C0044000000534100005645000049500000C4
:1084AC0000530000495000005253000054000000DB
:1084BC005345000054440000445600000053000093
:1084CC004554000053450000520000004745000091
:1084DC005453000045520000004700004554000072
:1084EC00494E000043000000534500005449000071
:1084FC004E430000002500007500000053450000AD
:10850C0054000000256C000075000000454E000072
:10851C00440000003000000073720000632F000064
:10852C00436C0000696500006E740000436F00002E
:10853C006E6E000065630000746900006F6E0000D1
:10854C00732F0000436C0000696500006E7400001E
:10855C002E63000000250000733A0000256900001E
:10856C0020250000732000002D2D0000206100004C
:10857C007373000065720000746900006F6E000078
:10858C0020660000616900006C650000640A000050
:10859C000021000000000000004500004E440000D7
:1085AC00007000005F6300006C690000656E0000E5
:1085BC00742D00003E7700007269000074650000A5
:1085CC0000450000525200004F52000020490000AC
:1085DC00442000003D200000256400000045000000
:1085EC00525200004F520000205400004558000029
:1085FC00542000003D2000002573000000210000E5
:10860C000000000008000000C80000002C01000061
:10861C0008000000C80000002C0100000800000049
:10862C00C80000002C0100000A00000080010000BE
:10863C00800000000A0000008001000080000000A3
:10864C000A00000080010000800000000D0A0000FC
:10865C0044480000435000002F5000006F7700008A
:10866C006572000020650000766500006E740000E5
:10867C00206F0000636300007572000072650000DB
:10868C006400000000040000A300000000000000D3
:10869C00414C0000544100005A0000004D500000B5
:1086AC004653000002010000000000002575000088
:0486BC0000000000BA
:020000040000FA
:1086C00080407800FAD2BF00814F50000F00320086
:1086D000E24F400004003200100B07000E000900BA
:1086E00030197800E201B10001007800FAF2B70019
:1086F000E2CF40000500320001407800070B070080
:108700000E00090032187800E201B10000000600F6
:10871000FBD2BF00A12F2100914078000104E100AD
:1087200017003200E24F40000C003200E2C1B300FB
:108730000440BC007C0341006599200062807A00FF
:1087400081FD2F00010040008402200013C0B3000F
:10875000A2A42000E6C07A006C0A0700FAD2BF008B
:10876000FBF2B70082FD2F0071558000010141002E
:1087700084022000160B0700A0A42000630A070053
:1087800000000600889FBE008A9FBE008C1F7800F4
:10879000FC12E20007003A00EAB602000000000006
:1087A000F27F200002006000024020000200400032
:1087B000E0978800C20320008000EB0020A7200083
:1087C000301102000000000048F920000005EB0015
:1087D00099302C000A407800B9FF07000900E80032
:1087E0009000780063804400100178001904E000D4
:1087F00008003A000280400008004000AB02200060
:108800008085450000ED2100808F55000200360074
:10881000FFFF3700FFFF3700CA6AEF008002200029
:108820000800400070558800008040000000E8000B
:10883000805588000000410090558800D00020003D
:1088400020568800C66AA900B1FF070079F8970092
:1088500071EAB700FC0607000A05E800E684440058
:10886000E60F5500020032000B047800D9FF3700F4
:108870004F0678004F05BE004F04BE000000060002
:108880000400FA00889FBE008A9FBE008C1F7800FB
:1088900090BF9F00A1BF9F0082457800030678002B
:1088A000844478000004EB00084578000840780014
:1088B00083FF070020568000ED0F50005B003A0058
:1088C00093FF070009407800714AE30057003A001F
:1088D00080212000705388000B04E00006003A005D
:1088E000DC528800C66AA80040002000205688009C
:1088F0004C5688004B00370000C02F00FC12B4001B
:1089000081F82000810F5000020036000040200056
:10891000E0978800E0978000D05288000000E800CF
:10892000E0978800CC5288000CE1020000000000B3
:10893000E0558800F1558800C68AA800E3CF5500AD
:108940001400320003003E00E1CF5500350039002D
:1089500003003700E4CF550032003A001900370019
:10896000740A07000B4078000014A2000080FB008E
:108970000000E9004F00DE004200DD00615380008E
:108980000120A1008080700061538800C42AEF009C
:10899000240037002FB897009FB8970001004000CF
:1089A00000004600D1528000010068004056880057
:1089B000600A0700640A0700200020002056880093
:1089C000180037001FB99700224090000080FB007C
:1089D000B2409000C808DD00808070009281FB00EA
:1089E000124090004800DD000300700080804000CD
:1089F00081004600D0528000808068004156880087
:108A000000A620000900090032587800A200B10039
:108A1000500020002056880011C0B30020C0B300D1
:108A2000820407000A80FB00040037000804E80005
:108A3000E60F54009CFF3A00E00F20004F0678003C
:108A40004F05BE004F04BE000080FA000000060083
:108A500011002000E54F500009003E0018FF0700FC
:108A600031568000000021000080600002003A00C2
:108A70008000780002003700C78AA900110020009A
:108A800001007800000006008000EB00E54F500078
:108A900005003E000AFF07008000EB002F0A0700D8
:108AA00001003A0011002000F5FF3700E54F5000AB
:108AB00035003E0002FF0700C0558000D0558800F9
:108AC00020568000E50F50002E00320006003E00C8
:108AD000E10F50000D0032002A003900E30F500072
:108AE00025003E0027003700EB0F50001500320034
:108AF00003003E00E70F50001F003E000700370054
:108B0000EE0F50001C003A0018003700969F02003C
:108B1000000000004C0607001B00370011C0B30026
:108B200010C1B300410407005C0AE20002003200F9
:108B30000D0A0700F9FF3A00800020002056880047
:108B40001100370011C0B30010C1B3003704070093
:108B50005C0AE20002003200030A0700F9FF3A0053
:108B6000C00020002056880007003700D0002000F9
:108B700020568800040037008040EB0040C1B3005D
:108B80002A0407003006070000000600881F78004E
:108B900000447800E54F500004003E00C8FE070086
:108BA000C66AA90008407800C0FF07004F0478009B
:108BB000000006008000EB00E54F500009003E0079
:108BC000BFFE0700D2FE0700A098200001A62000EB
:108BD0000900090031587800C0528000A04C88007C
:108BE000A1982000A6FF3700E54F500006003E0088
:108BF000B3FE0700C6FE0700DB09070002003200D3
:108C0000DD0907000904070000000600E54F5000D9
:108C100012003E00AAFE0700C4CABF00E74F500082
:108C200002003200EB4F50000C003A00A2558000C9
:108C3000B1558000810F510005003900D1090700AE
:108C400082805000010040000000E900040037006D
:108C5000028050000000E900010037000000EB0036
:108C6000000006000200FA00889FBE000044780061
:108C7000A1FF9F00E54F500031003E0090FE07002D
:108C800008407800E1FF0700800478000000E00061
:108C90002B003200E10F500002003A00084078003B
:108CA000D1FF0700C70AAB0007003A00B50907006B
:108CB0000000D100808F540003003E00084078007F
:108CC000C9FF0700C70AA800BB090700A05580001C
:108CD0001400200084417800668157000B090700CA
:108CE000A15580008100E800A155880080558000D2
:108CF000808F50000200390070558000A055880018
:108D0000E18F540004003A0008407800B6FF0700E5
:108D1000090078000B00370010002000C6AAAB0045
:108D200008003A00C6AAA80024E1020000000000E2
:108D30007800400000568800100020000100370035
:108D40000000EB004F04BE000080FA0000000600A7
:108D5000889FBE008A9FBE008C9FBE0000447800A2
:108D600001067800820578000000EB00E54F540012
:108D70003F003E000840780051FE070008407800A0
:108D8000A2FF0700000578000000E00004003A00A0
:108D90000840780094FF07000A007800340037008C
:108DA0008B0F5000020036008B0478000100370062
:108DB00080047800C70AAB0007003A007109070079
:108DC0000000D100800F550003003E0008407800ED
:108DD00085FF0700C70AA800A555800081558000BF
:108DE000058044008006EB00810F50000B00390025
:108DF00085865000700907000D02780013C0B3008B
:108E00000C01780005007800C00807000D06460038
:108E10008D84540070558000A055880066090700B5
:108E2000A05580000902780013C0B3000C0178003F
:108E3000B608070009007800B42AB4008B0F55006B
:108E400003003E000840780067FF07000700370076
:108E5000C6AAAB0005003A00C6AAA80024E1020099
:108E6000000000007800400000568800098046009D
:108E70004F06BE004F05BE004F04BE0000000600B6
:108E8000889FBE00804478000104780001007800CB
:108E9000F411020000000000000178008800780052
:108EA00009407800AAFF0700000044004F04BE00FC
:108EB00000000600889FBE00804478000000EB00A0
:108EC000E5CF540009003E0009407800FCFD070092
:108ED0007855800080558000080450000804E9009F
:108EE0000940780049FF0700000054004F04BE000D
:108EF00000000600881F7800004478000A00070080
:108F00000000E0000600320008407800ECFD070099
:108F1000C0558000D055880017090700430307009B
:108F20004F047800000006008000EB00E54F500081
:108F30000B003E00E2FD07001509070002003900A2
:108F400081005100060037009055800081005000DC
:108F50008055800000005100808040008100E800C2
:108F6000C7FE3700889FBE008A1F78000044780043
:108F700001057800ECFF0700800478000000E000A5
:108F80001500320008407800CDFD07000A00E0001F
:108F900006003200D25580001400200009090700A5
:108FA000844078000A00780058080700D1558000F6
:108FB0008100E800D155880090558000808F5000D6
:108FC0000200360080558000D0558800E18F5400A3
:108FD00003003A00C74AA8000900780009003700DA
:108FE00010002000C6AAAB0006003A00C6AAA800DE
:108FF00024E1020000000000A007B0000056880035
:10900000100020004F0578004F04BE00000006004D
:10901000889FBE008A9FBE0080447800810578004A
:1090200002047800C0FF0700000578000000E0009F
:109030002C00320009407800A1FD0700880F550080
:10904000010031000A047800D2558000915580005B
:10905000020044008004EB00810F50000B0036003A
:10906000028050008004E8000B00E00004003200A1
:10907000090278006A08070024080700898545006E
:109080000904540080558000D05588000B00E00092
:1090900003003200D2558000530807001B08070068
:1090A00008007800BA2AB40008844400080055007B
:1090B000800F540003003900C74AA8000800780058
:1090C00008003700C6AAAB0005003A00C6AAA800EF
:1090D00024E1020000000000A007B0000056880054
:1090E000080078004F05BE004F04BE0000000600D7
:1090F000889FBE00804478000000EB00E5CF54005C
:1091000008003E00094078006DFD0700885580008A
:1091100090558000080450000940780082FF070045
:10912000000054004F04BE0000000600889FBE00EF
:109130008A9FBE000044780081057800020578000F
:1091400083047800E54F500022003E000200E0005A
:10915000200032005AFD07000840780072FF070027
:109160008000780009004500808F50000100310028
:1091700009855000D0558000008144009155800041
:10918000810F5100010036002808070002805000BE
:109190000004E800880F550005003E000A02780030
:1091A0001F080700D90707000A0078000A003700E7
:1091B0000D080700D5070700825580000B0044000A
:1091C0000802550082080700D00707000A0078004F
:1091D000010037000000EB004F05BE004F04BE0049
:1091E000000006000200FA00810178001200200051
:1091F0008F80E900CDFF0700EFF897000180FB00AA
:109200000080FA00000006000F03B000889FBE0037
:109210008A9FBE008C9FBE008E1F7800004478009D
:10922000E1B79F00F2B79F008305780084047800BF
:1092300085BF9F00E54F5000A1003E000200E00006
:109240009F0032001EFD07000840780036FF07002F
:109250000B0750007FB097008E0F50009A003E0021
:109260000900E00003003200890F570001003600BA
:1092700009077800D0558000008145009155800095
:10928000810F510001003600E807070002805000FE
:109290000000E800C0B79F00EFB09700A1B79F00A3
:1092A000B1447800A1B79F000FBA97000400E00016
:1092B00006003200F0C9B30000C04400F94F50006E
:1092C00002003E0000CEB30080C444007FB597008A
:1092D000BBB79F00D2B79F002FB697008006EB0068
:1092E0000BC2B3004FB09700FF0F500001003E00CB
:1092F0008FED97000B80FB00800F570001003100BD
:109300008E4578000B84FB00080278002D080700CA
:109310005FB1970011C0B30040FC2F000F00400068
:109320007A07070088027800DFB097008880400045
:10933000D1B79F004FB2970008025200C4B79F00F8
:1093400004003A0080558000D0B79F008080EB0079
:10935000C1B79F000FBA97000400E0005F003A0019
:109360005B0037000042EB0043FC2F008F8141007F
:10937000F6C9B30007CEB3003FB09700FFB0970027
:1093800001045000030178009340780006C04000BB
:10939000F94F500001003E0087C9400092CF5400B1
:1093A0000E003A000A05E90004003A000480FB00C0
:1093B000000044000000E8004B003700BC44780087
:1093C00006C044001D002000F94F500010003E0070
:1093D00087C444001D0020000D0037000D00E00090
:1093E00002003A007FB59700090037006FB0970080
:1093F0009044780006C04400F94F500001003E0040
:1094000087C444007FB597002FB697008006EB0015
:109410000442E8008301E80084CF550021003200B7
:10942000D8FF37000041EB008000EB003FB297000F
:109430007FB097008001520044FC2F000F024200D1
:1094400064C0780080CF540009003A000A05E900A2
:1094500004003A000280FB00008041000000E800A8
:1094600021003700BC4478001D00200009003700AF
:109470000D00E00002003A007FB5970005003700BC
:109480006FB09700904478007FB597002FB6970093
:109490008006EB000241E8008100E80082CF550021
:1094A000E5FF3A00050757008E0F550006003E0005
:1094B000BFB0970085804000B1B79F0088FF37009C
:1094C0000000EB00080037000080EB0006003700CA
:1094D0000B04E000D3FF3A00F2FF37000B04E0007A
:1094E000A0FF3A00EFFF37004F0778004F06BE009D
:1094F0004F05BE004F04BE000F03B1000000060080
:109500000200FA00E1FF9F00840278000302780065
:1095100082017800120020008F80E9003AFF0700E6
:109520000080FA0000000600E6874700889FBE0022
:109530008A9FBE008C9FBE008E1F78000005EB0046
:109540002E0020000DA720000A4678000A4078006F
:109550005BFC0700305680000160200001006000C5
:1095600031003200526A0200000000000000E000FA
:109570002D003200305680004A00DE00E105600018
:1095800009C1B3002A00370061FC07007440B9002C
:109590008001780022A720000200400001A62000E0
:1095A00009000900B0587800A000B100EA8041002D
:1095B000E1007900C1528800EC80410082804000C7
:1095C000160020000700200031024300A1824B005A
:1095D00094528800A55288000153800017538000E0
:1095E00087804000C252800082804000D2528000BA
:1095F0008280680041568800610020002156880062
:10960000620214007422B90061A8200001814100A7
:1096100013C0B30083407800BC060700AA2AEF00FD
:1096200029C1B300310037008044EB008005EB0016
:10963000C6AAAB00070032000856800024E10200F1
:1096400000000000000454004240A90001003C005A
:1096500009C1B300C6CAAB0007003200185680002B
:1096600024E1020000000000000454004240A90070
:1096700001003C0009C1B30020568000EB0F5000F0
:1096800009003A001856800024E1020000000000A2
:10969000000454004240A90003003C00C000200028
:1096A0002056880019C1B30020568000E40F5000F6
:1096B0000C003A00425680000004EB0021A8200074
:1096C000110078000000E00006003200820F500018
:1096D000ADFF32000804E800F4804000E30F5400BE
:1096E000F7FF3A000904E0000400320011C0B300A3
:1096F0008BC05000094078004C010700C68AAB00BF
:109700001D003A0015070700CF003A000CE10200E7
:1097100000000000CA060700CB003300315680006D
:1097200067806000E60F50000B003A00430CDE003B
:10973000614464000C407800DCFC07000C407800B9
:10974000DAFC07000804E000BF003A00E000200057
:1097500020568800BC003700EDFB070021C0B30095
:1097600000C1B300310107000CE10200000000005D
:109770000B070700B40037000CE1020000000000F6
:10978000AF060700B0003300E1FB07002056800061
:1097900001002000EC0F5000E08F580087003E00D1
:1097A000006001000C0037001C0037003700370054
:1097B0003F00370081003700570037006200370054
:1097C0006A003700710037008000370073003700EF
:1097D00066003700750037008A9F02000000000015
:1097E0000000E000750032001100200021568800C2
:1097F0006C4AAB000400320000538000B09F0200AE
:10980000000000006D0037000053800011C0B3005D
:10981000B09F02000000000068003700728057000F
:10982000DA9F0200000000000000E0006300320048
:10983000969F0200000000000000E0000E003200D1
:109840007FB097008FB897000053880011538800AD
:109850002E56880000538000620AB400C152800076
:1098600001004000D152800001006800405688008D
:10987000B5060700510037000CE1020000000000AF
:10988000C7060700C42AEF004C00370024E102009D
:10989000000000000056880000A62000DECE020076
:1098A00000000000300020002056880043003700F0
:1098B00041A6200000A620000ACF02000000000000
:1098C0000000E0000F003A0024E102000000000068
:1098D000025680000200500052528000820F500059
:1098E0003600360070CABF00E54F500003003E004E
:1098F0000040E80070EAB700560607002E568800C0
:109900002E00370050002000205688000004EB0095
:1099100029C0B3004600370029C0B30012C0B3000D
:109920009D4F11006E0036000E00780070EAB700FF
:10993000444B2C005452880044002000645288009C
:109940008E4478006600370015C0B3009DCF12002A
:109950005E00360030568000680060001B003A0050
:1099600029C0B300000478001A00370026C0B300F5
:109970009D4F1300570036008000200020568800BD
:1099800019C1B3000004EB001200370027C0B30078
:109990009DCF1300510036000C00370020C0B300EB
:1099A0009D4F10004B0036000800370021C0B30067
:1099B0009DCF100049003600040037000004EB0082
:1099C0000904E00003003A001F00370049C1B3005A
:1099D000180020000B00E00015003200706AEC0057
:1099E0001C060700B0528000B355800003015000F0
:1099F000830F5000020031006206070000014100A1
:109A0000705280008152800002005000E0805800B7
:109A100066060700020078005C2AB400B352880092
:109A20008040EB0009407800800007000300370009
:109A300011C0B300094078007C0007000800E00076
:109A400001003200800207000A05E800E60F550019
:109A5000BDFE3A008004EB002AA720007448B9003C
:109A6000000478007000400060007D000000E0000D
:109A70001D00320024E102000000000072014400D9
:109A800062017D000200500072722000820F5000BF
:109A90000A003600628214007422B90062A8200015
:109AA000020144000A00440013C0B3008340780060
:109AB00096050700AA2AEF008904E9008904E80056
:109AC000E28F540008003E00E4FF370029C1B300D4
:109AD0000300370009C1B3000100370019C1B3000A
:109AE0000004EB00BDFF37004F0778004F06BE00B3
:109AF0004F05BE004F04BE006F00B100000006001D
:109B00002000FA00889FBE008A1F78008004780039
:109B1000020578001082FB00104090004800DD0034
:109B200004017000294290000482FB00394090003B
:109B30004800DD008401700072845700028CBE0072
:109B40001101BE0092BF9F00A3BF9F000040EB0029
:109B5000E0F79F0060C0B300F0F79F00CABF9F000E
:109B60000A00780044B9020000000000C0BF9F0056
:109B7000C10020000800780084B902000000000045
:109B8000000478000A007800CA6D0200000000009E
:109B90008880EA00808F50001D003A000000EB0032
:109BA00000DC02000000000041012000A0FD2F00A9
:109BB0000F004000FE6F020000000000A0FD2F001B
:109BC0000F004000FC0107003FB097004400DE009A
:109BD0006F4060004200DD00744050000080FB00D8
:109BE000000055007404500089007800A0FD2F008B
:109BF0000F0040005B0107000000E000040032009D
:109C000088007800A0FD2F000F0040007A020700B6
:109C1000686A020000000000100020004F05780074
:109C20004F04BE000080FA00000006002600FA0083
:109C3000889FBE008A9FBE000044780001457800DE
:109C4000B3FA07000808A30002003200C76AA800A0
:109C50000804A100C6AAA900C6CAA900C6EAA900AC
:109C6000C72AA900C74AA900C70AA900526A020068
:109C7000000000000000E000FCFF3200660064000D
:109C80008004EB004E003A00A0558000B2528000E4
:109C90008004EB00820F50003E00320011003600BD
:109CA00002005000E1528000810F50000100360098
:109CB0000100780079538000890F500002003E00B7
:109CC0008004780001003700C74AA8000902780024
:109CD000670507000D05070009007800562AB40043
:109CE0002C0037008155800082815000B3BF9F0057
:109CF000830040007055800000805000E1528000D9
:109D0000810F500001003600010078007953800077
:109D1000890F500002003E008004780001003700E7
:109D2000C74AA800838F540001003100B9BF9F00CB
:109D30003FBA97004E050700F40407003FB89700AC
:109D400000825400B4BF9F000800320072558000AA
:109D5000B0528000B00AB500919D20000100400083
:109D6000980507008040EB00E8040700B05280002F
:109D700080804400B152880082558000828F50005C
:109D80000400390070558000000051000080500030
:109D9000B0528800C76AAB0007003200E052800072
:109DA000808F54000400320070538000808F540074
:109DB000010032000804A0000900E00002003A009F
:109DC0006300640011003200090078005C2AB500CD
:109DD0000900E000010032000834A0000A08A300D6
:109DE00005003200706AEF00D11223005152880042
:109DF00011002000615288000CE102000000000008
:109E0000FB040700C68AA800250037000A18A30033
:109E10000E003200305680008040E800E78060008D
:109E200082FF2F00020060000100700030568800A1
:109E3000705280008152800061005000E080580024
:109E40005A05070019002000150037003056800021
:109E50007000600002003A008004780010003700B3
:109E60000A08A3000A003A0070CABF0008003200C6
:109E70000040E90070EAB700505280006152800053
:109E80008100D1000080D3005052880061528800C8
:109E90000CE1020000000000D50407008004EB0084
:109EA00041FD2F0001804700D25280000208780057
:109EB000C1528000110098007252800083528000CD
:109EC000C2AF9F00D3AF9F00ED040700E0AF9F003B
:109ED000F1AF9F000FB09700F1FF23000100600079
:109EE00001FF2F000100600080B79F0098E79F00EE
:109EF0000000EB00B0B79F0009014100E08149007C
:109F000072528800835288008880FB000100D100D3
:109F100061006000804578000004E000130032001A
:109F20000148A30003003A006000B800E0AF9F00C2
:109F3000F1AF9F006C2AAB00070032004FA89700DA
:109F4000DFA8970061005000E0805800C0AF9F007C
:109F5000D1AF9F000500370061014100E081490059
:109F600072528800835288006C2AA8000808A30057
:109F7000010032006C0AA800050507000600390040
:109F800080558000B20AB5008100510001005000E8
:109F900090B79F0003003700028050000000E900E6
:109FA00090B79F00926A02000000000080007800D5
:109FB00090AF9F00F0032000808F500003003E0010
:109FC0008000EB0091AF9F000300370000FC2F00E2
:109FD0000080400090AF9F009FA897001FB097009F
:109FE000810F50000100360091B79F0042FD2F0005
:109FF00002804700F000070074854400F2F02F0053
:10A000000FB09700820060000105B30081B79F0088
:10A010000B04E0000A0032007885440020C0B30041
:10A0200080EF9F0040C0B30090EF9F002080210090
:10A03000D0B79F00028060000006B30080B79F0089
:10A0400021802000914078008180FB0003C8BF0080
:10A050004800DD000101700041802000914078003F
:10A060008180FB0005C8BF004800DD008101700051
:10A0700074845700028CBE0000538000115380008E
:10A0800080BF9F0091BF9F000040EB00C0F79F0082
:10A0900069C0B300D9F79F00BABF9F000A007800DB
:10A0A00044B9020000000000B0BF9F00C1002000C2
:10A0B0000800780084B90200000000000080EA0077
:10A0C000A0B79F00109B2000226D0200000000003E
:10A0D0000A0178008940780000A6200078DB0200A1
:10A0E000000000004101200042FD2F0002804700D7
:10A0F0009E700200000000000B04E000040032002B
:10A1000041002000788057009E700200000000008F
:10A11000509C20004C6D0200000000000A007800F6
:10A12000CA6D02000000000090AF9F00509D20000B
:10A13000226D0200000000002100200020FD2F0001
:10A140000F0040009E70020000000000FE6B020045
:10A15000000000004F05BE004F04BE000080FA0062
:10A1600000000600889FBE008A9FBE008C1F7800FA
:10A170008005780001067800900190000300E0005F
:10A1800088003200214090000080FB00B140900028
:10A19000C808DD00808070001C81FB001C4090001E
:10A1A0004800DD0002007000808040009B8040007D
:10A1B00001856900E9CFB3000004EB000840780096
:10A1C0003FF9070020568000ED0F500018003200C4
:10A1D000E40F500006003A009B00900040568000BB
:10A1E000810F500012003A008844780010003700B8
:10A1F00040568000800F55000D003A0044F90700DA
:10A200009B009000D0528000808F500008003A00E0
:10A21000C05280009B0F100005003A001B0407008D
:10A220000053800011538000220407001500320003
:10A230000804E800E60F5400E0FF3A00E2CF4400D3
:10A2400031003200094078001DF9070030F907009D
:10A250004A56880000A62000090009003C587800F2
:10A26000AC00B1001B017800C25288009B05900031
:10A27000DB52880073558000B35288001000200024
:10A2800049003700100020004700370024E1020099
:10A29000000000007449B9007201410024A72000A9
:10A2A00000317A000000EB003F003700744CB90029
:10A2B0002AA720000A004400090009003C58780041
:10A2C000A000B100AC00B1006A0044001B307D006A
:10A2D0000A0044002B019000BB019000620098002E
:10A2E00073009800700044009B0590000B307D00C7
:10A2F00024E10200000000007204440000347D00EC
:10A300000000EB00280037006B0090000098A300CD
:10A3100024003200AA0AE20022003A008004EB0086
:10A3200024A82000940078000100E0001000320012
:10A330001B009000808F500009003A0054B897002D
:10A340009B0F500006003A00D003070004B89700A6
:10A3500094B89700820F5000838F5800CBFF3200D3
:10A360008904E80074024200E38F5400EDFF3A00D4
:10A370000004EB0008407800D1F80700C66AAB0083
:10A3800005003200E2F807009B009000D0528000E8
:10A39000810F5000C5FF32000804E800E60F5400AA
:10A3A000F4FF3A000000EB004F0678004F05BE00B6
:10A3B0004F04BE0000000600881F780000047800EB
:10A3C0001000780044B9020000000000000C780082
:10A3D0001800900044B9020000000000100498002A
:10A3E00028009000B800900056B90200000000005C
:10A3F000200498003104980048009000D800900094
:10A4000056B9020000000000400498005104980072
:10A410007800900044B90200000000007004980029
:10A420000808900044B9020000000000000C9800E9
:10A430001808900044B9020000000000100C9800B9
:10A440004F04780000000600B1F80700D0528000E9
:10A450004056880070558000A0558800B05588008F
:10A4600080558000C0558800D055880040002000ED
:10A47000C66AAB0001003A00D000200020568800D8
:10A48000C60AA900C62AA900C64AA900C68AA90008
:10A49000C6AAA900C6CAA900C6EAA900C70AA90097
:10A4A000C72AA900C74AA900C76AA900C78AA80085
:10A4B0006C0AA9006C2AA9006C6AA9006C8AA90020
:10A4C00070558000B0528800B0B602000000000055
:10A4D00070528800B0B60200000000008052880070
:10A4E0006AAAEF0010002000E05288000000060079
:10A4F0000200FA00889FBE00C000200000DC0200BD
:10A5000000000000E86F020000000000000FB20031
:10A510004280DE00F444500033003200710020001D
:10A520000000EB00FE6F0200000000002B0037006F
:10A53000E86F0200000000000004E0002A00320082
:10A54000E14F500025003200E24F500017003A0062
:10A55000E2CF5400240036000000EB00D0BF9F0083
:10A56000E86F020000000000E44F500006003A00CF
:10A57000E86F020000000000B0FF9F00E86F0200DB
:10A5800000000000A0FF9F00DFB8970070212000AE
:10A59000808F500014003600D039B000808F5000FA
:10A5A00012003E000100780010003700E1CF540097
:10A5B0000D003600E86F0200000000000044780043
:10A5C000894F500008003E008080FB000000EB0037
:10A5D000FE6F02000000000088C454008944E900B6
:10A5E000E1CF4400D2FF3A00802120004F04BE009A
:10A5F0000080FA0000000600F0874700889FBE0038
:10A600008A9FBE008C9FBE008E1F780000057800D8
:10A6100001077800504C900040069000D006900052
:10A62000B000900020009000D0B79F00E1B79F00DD
:10A63000C60AA900C62AA900C64AA900C68AAB0054
:10A6400003003A000CE10200000000005403070080
:10A6500024568000E40F520003003200E50F520040
:10A6600045003A00160037000880FB000028A300D0
:10A6700038023A000048A300060032007C528800ED
:10A680008D5288008040EB0040C0B30067FD07009A
:10A69000300237000018A3002E0232005FB197008D
:10A6A000EFB1970061014100E081490092528800BA
:10A6B000A35288008EFF07007053880028003700DF
:10A6C0008880FB000128A30026023A004408DE002F
:10A6D00061006000804578000004E0000A0032005C
:10A6E0007852800089528000880F5600898F5E0062
:10A6F00005003200F20207004CFD07007852880086
:10A7000089528800170237000118A3001502320091
:10A710005FB29700EFB2970061024200E0824A0008
:10A7200094528800A55288007A059000EA52880069
:10A730006FFF0700705388000B04E0000800320030
:10A740000D03070039FD0700700020002056880027
:10A750000CE1020000000000DE02070001023700E9
:10A7600011C0B30020C1B30030FD0700600020001D
:10A7700020568800FB0137008882FB00E1856200DB
:10A780008BF79F000B04E00002003A00CEB79F0059
:10A79000020037008E00E800C1B79F000884FB006C
:10A7A0000818A300030032004FB197000201E8002F
:10A7B000C2B79F00F60207000500390080558000EF
:10A7C000B20AB50081005100810450000200370038
:10A7D000028050008004E900A90207005FB19700E1
:10A7E000EFB1970000005100818059000001BE00C8
:10A7F000F0B79F004FB397000600E0001E00320044
:10A800000900E00027003200E00F5000E08F580000
:10A81000040035006148B800820F5000838F580053
:10A8200009003E004FB3970006004100E080490058
:10A830004240A9000600340006805400CF80DE00AC
:10A840009C02070002003C001600200001003700B7
:10A850000003EB006148B800960207000F003D00BE
:10A86000FFB097004FB19700028040004240A9001E
:10A870000F003C0009003700E00F5000E08F580047
:10A880000B003200070035006148B800820F50000D
:10A89000838F580006003E00020037000600E000EB
:10A8A00003003A000828A300AE013A00AB013700CC
:10A8B00066806200A7013A000848A300A90132009F
:10A8C000EB0F520005003E00E70F5200150031006B
:10A8D000E60F5200BB003A0003003700EC0F5200B5
:10A8E000B8003A00AF0037007452800085528000F3
:10A8F000A4B79F00B5B79F00840F5600858F5E00F8
:10A90000060032006E020700C8FC07002FB0970057
:10A91000BFB09700A5020700920137007000200029
:10A9200020568800B4528000A25580008400510057
:10A9300002003B00930207008080400072528000BA
:10A940008352800001004100E08049000000560071
:10A9500081805E004240A9000B0034006C0AAB000D
:10A9600003003200E10F5000E08F58000400320075
:10A970008040EB0000C1B300ACFC07007901370058
:10A9800061065600E0865E00B55580000500520065
:10A99000CF80DE000003510081835900850F5200F3
:10A9A000020039000600BE000300370075020700F0
:10A9B00000005300E0805B000001560081815E00D2
:10A9C0004240A900280034006E0207000100200068
:10A9D0003802070024003E006C6AA9006C8AA900B6
:10A9E000C70AA900B055800002024000B455880093
:10A9F000B1528000810F500005003E00810F5200CF
:10AA00000900360001005200350207000600370039
:10AA10005C02070000804000800F520002003600F8
:10AA2000000052002E02070081558000810F520065
:10AA30000400390070558000008050000000520072
:10AA4000B0558800B252800081558000810F5100BE
:10AA50001A0039007055800000805000000051003D
:10AA6000B052880015003700850F520013003200E5
:10AA7000605380000038A3000F0032000048A3009C
:10AA80000C0032007652880087528800B052800055
:10AA9000808F5200050036003A020700CF80DE00AA
:10AAA0000000530081805B0040020700B55288001F
:10AAB000C74AA8006C8AA8006C6AA800B15580003B
:10AAC000A0558000808F50000C003A00C76AAB0090
:10AAD00004003A000CE1020000000000FD01070044
:10AAE000060037000502070004003A006C0AAB00BC
:10AAF00002003200C68AA900C76AA900735280000A
:10AB00008C8051007A009000010050005C0AE20045
:10AB100003003A000000E00001003200C72AA8004C
:10AB2000E052880020568000E80F50000D003A00E7
:10AB3000F201070023003A006C0AAB00210032004A
:10AB40000CE102000000000022BC2E00B300200037
:10AB5000A9010700C68AA80090002000205688009E
:10AB600018003700E90F500009003A000B00E00020
:10AB700014003A007C5288008D5288008B40780087
:10AB800040C1B30029FC07002FFE0700F500370085
:10AB9000EA0F50000B003A00D8010700F1003A001C
:10ABA000EC00370074528000855280006100420042
:10ABB000E0804A00800F5600818F5E00E9003A0075
:10ABC000E40037000858A300E6003A002056800051
:10ABD000EB0F5000E3003200EA0F5000E1003200BA
:10ABE000EC0F5000DF0032000E00E0009400320055
:10ABF000FFB597000B00E00044003C006A009000A5
:10AC00004200DE00C003B2000B00500000DC020076
:10AC1000000000007FB39700060547008A8F5400AC
:10AC20000100310009057800950107000A00400085
:10AC3000E080480090528800A1528800C5558000ED
:10AC40009155800005004500810F50000E00360030
:10AC5000058450000804E8006C0107002B01070080
:10AC600008045500D40107008055800008027800D0
:10AC7000A70107002501070080558000000444005B
:10AC8000C855880006003700CB0107000A0278008B
:10AC9000600107001D0107000A007800B82AB4000F
:10ACA00050538000E10F4000650032008A005000E0
:10ACB00051538800F05280000081400011003300A1
:10ACC0000100E0005E003C006D0107000200400052
:10ACD000E080480090528800A1528800C055800052
:10ACE00080004100C155880090558000808F500041
:10ACF00004003600B00AB500008040000000E90002
:10AD0000C05588006AAAEF004D003700FFB09700D9
:10AD100001004700808F540001003100018754007A
:10AD20006A0090004200DE00C003B20000DC0200B6
:10AD300000000000C15580007FB1970081024100F2
:10AD40009255800005004700820F50001600360023
:10AD500001005100FFB19700030050000004E8001B
:10AD60000800330029010700E800070092010700EE
:10AD7000805580000802570065010700E3000700C6
:10AD80000D0037008C01070002007800B00AB50002
:10AD9000008042000000E9000E0278005C0107001C
:10ADA000DA00070004003700830107000E02780074
:10ADB00018010700D500070050538000E10F400044
:10ADC00003003A005B538800FE5288001C003700E5
:10ADD000800078007FB29700800F52000E00310093
:10ADE00004014700F052800000804000800F5100B5
:10ADF00002003E00828F500002003600FE528800A2
:10AE000003003700FFB2970005005000F0528800A1
:10AE10005B5388000A0037007FB3970006014700A4
:10AE2000F052800000804000800F51000400360086
:10AE3000800F530002003E0001005100F0528800D4
:10AE40004FB097000000E0001200320043010700FD
:10AE500002003200C1558000D1558800C6EAAB001F
:10AE6000040032004401070070FB070028F60700C9
:10AE700008003700C6EAA800C6CAAB0005003A00C1
:10AE8000C6CAA80024E1020000000000D003B00000
:10AE9000105688000FF197000204E00031003200E4
:10AEA00094528000A552800061014200E0814A0076
:10AEB0004FB397005FB29700EFB2970006004200D1
:10AEC000E0804A00FB00070026003A00925288000A
:10AED000A3528800210107000F00320003003E004A
:10AEE000E60F50001D003A0005003700E80F500043
:10AEF00010003200E90F500018003A00120037002D
:10AF0000C00020002056880011C0B30010C1B3005B
:10AF100046FB070013003700B000200020568800D1
:10AF200024E1020000000000A007B00010568800D5
:10AF30000A003700F100070003003200A0002000E3
:10AF400020568800050037008040EB0000C1B300A8
:10AF500036FB07003CFD0700020037000601070032
:10AF600032FB07004F0778004F06BE004F05BE00BA
:10AF70004F04BE000F01B10000000600889FBE0014
:10AF80008A9FBE000104780082057800834478001F
:10AF9000E54F500058003E00C9F507000800E000EA
:10AFA00001003A001800200070558000B20AB50078
:10AFB0000005E9000B044400880F55004E003900DD
:10AFC000D3F507006380640001003A003940B30004
:10AFD000080055008981FB000318A30002003A0015
:10AFE0008B007800060037000308A300030032003E
:10AFF0000000D100808045000100370080804500BE
:10B0000070558000008040000004E800C4558000B6
:10B0100051538000E18F400009003200F05280005F
:10B02000008040000002420090558000800F5200D6
:10B0300003003600B00AB500000042000002E9003B
:10B04000D0558000800F520003003600800F54005E
:10B050000A00360005003700800F5200050031005D
:10B0600080558000800F5400070036000328A3009D
:10B0700021003A00D8558800C8558800D055800076
:10B08000800F5200100031000328A3000E00320090
:10B0900082558000C80007000202520081417800FA
:10B0A0000800780019000700C1558000D0558000C5
:10B0B000808F50000400310008007800B00AB5000D
:10B0C00000805000C0558800885588007055800069
:10B0D000B0528800B0558800A055880011002000AB
:10B0E0009E00070005003A00A3000700CFFA070002
:10B0F00011002000010037008000EB000100780003
:10B100004F05BE004F04BE0000000600889FBE0031
:10B110008A1F780000057800820478000404780013
:10B120000304E00016003200E1CF51002B003A008A
:10B130000104E00008003200E1CF500027003A008F
:10B1400004017800890078000A00780010120200DB
:10B150000000000021003700E10F4500030032002D
:10B160000A007800226D02000000000088007800CC
:10B17000090078009E7002000000000017003700F0
:10B180000104E0000C003200E1CF500013003A004F
:10B19000E10F410003003200020078004C6D020014
:10B1A00000000000880078000A007800FE6F0200AE
:10B1B00000000000090037000401780089007800D1
:10B1C0000A0078005A6E020000000000D26F0200F0
:10B1D000000000000000E000FCFF32004F05780096
:10B1E0004F04BE0000000600080278000C00370083
:10B1F0005252800063528000000141008181490069
:10B20000E2558800F3558800000006006A00070038
:10B21000080278003E0007000500780000000600E4
:10B220006B0007000B0078000000060001007800AA
:10B23000B00AB500000041000001E900000006006E
:10B24000E2558000F35580000200500083805800D2
:10B250000000060050528000615280000000400053
:10B26000818048005052880061528800000006002A
:10B27000540007008040EB00909D20000000060075
:10B2800090528000A1528000000006009C80FB00CC
:10B290001C4090004800DD0001017000AC409000AF
:10B2A0008180FB003C4090004800DD00810170007F
:10B2B00000000600800F5100818F59000000060039
:10B2C0007C5288008D52880011C0B30040C0B3008A
:10B2D0000000060032000700C68AA9000000060030
:10B2E000725280008352800000004100E0804900DB
:10B2F0002E000700B4528800000006007052800043
:10B3000081528000800F5600818F5E000000060091
:10B310008041EB000081EB0000000600E2C1B300B9
:10B320000440BC006099200000014100E0AA200018
:10B33000000006007FB097008FB897000053880088
:10B340001153880000000600706AEF008109200098
:10B35000515288004C2AEF00000006002056800061
:10B36000E70F500000000600A1558000B052800099
:10B37000808F50000000060011C0B30000C1B30070
:10B380000000060070558000B00AB50000000600FD
:10B39000C2558000D1558000810F51000000060089
:10B3A00042782D007301200093FF3700705288000F
:10B3B0008152880000000600A1AC20009140780076
:10B3C00000000600A3AC20009341780000000600B6
:10B3D000FCFF070011C0B30000000600E2022000DD
:10B3E000820F5000E08F58008D003E000060010089
:10B3F0002E0037008A0037002F0037008800370002
:10B40000870037008600370085003700840037004A
:10B41000830037008200370081003700800037004A
:10B420007F0037007E0037007D0037007C0037004A
:10B430002400370026003700280037002A00370094
:10B440002C0037002E003700300037003200370064
:10B450003400370036003700380037003A00370034
:10B460003C0037006E0037003D0037003F003700DA
:10B4700041003700430037004500370047003700E0
:10B48000490037004B003700650037004C0037009B
:10B490004E0037005000370052003700540037008C
:10B4A00056003700580037005A003700E0C62A001F
:10B4B000550607006000370090C72A0052060700B3
:10B4C0005D00370018850200000000005A003700B8
:10B4D0003E8502000000000057003700C4850200CE
:10B4E0000000000054003700EC850200000000005E
:10B4F0005100370002850200000000004E003700B6
:10B500007E840200000000004B003700FE83020032
:10B5100000000000480037000A840200000000001C
:10B52000450037001A840200000000004200370086
:10B530002E840200000000003F0037004284020019
:10B54000000000003C0037005684020000000000AC
:10B55000390037006A84020000000000360037001E
:10B56000DC8402000000000033003700E0840200A9
:10B570000000000030003700648502000000000079
:10B580002D00370094850200000000002A003700DB
:10B590004487020000000000270037006A8702008D
:10B5A00000000000240037001486020000000000A4
:10B5B0002100370036860200000000001E00370020
:10B5C000B6870200000000001B003700E48702007D
:10B5D00000000000180037009C86020000000000F8
:10B5E00015003700C286020000000000120037007C
:10B5F000E8860200000000000F0037000E870200FE
:10B60000000000000C003700588602000000000017
:10B61000090037007A8602000000000006003700AB
:10B62000F90607004200200041C82A00BC060700B6
:10B63000A84602000000000000000600F206070015
:10B64000E1C7B30082D82000604079003246020092
:10B650000000000000000600889FBE008A9FBE0018
:10B660000040EB008EEDB7006BD820008004EB00AB
:10B670006A0920000084FB004244DD000B00440006
:10B680000908780084C0B300030520000941780050
:10B690006000B80040440200000000000884E80098
:10B6A00000F47D0000C0EB0004EDB70005EDB7002D
:10B6B000E2D82000124178000281FB000A91B90013
:10B6C00000ED210002004000226D02000000000099
:10B6D000000478008A00780000CF20009E700200ED
:10B6E0000000000008007800226D02000000000049
:10B6F0008E4DEC008EEDB700E14F5000DDFF3600BF
:10B70000090078008EEDB7004F05BE004F04BE0063
:10B7100000000600889FBE008A9FBE008C1F780034
:10B720008004EB0088D820006CD820008945780080
:10B730000805780018407800E24F400027003200EA
:10B7400028450200000000000000E0001800320060
:10B750000940780029000700AB0607000C004000F4
:10B760000008EB0004CDBF00E14F400003003200B1
:10B77000029602000000000004EDEF0005CDBF00BE
:10B78000E14F40000300320002960200000000007A
:10B7900005EDEF006506070043C0B3000001EB00B4
:10B7A0001100200060407E00BE5702000000000033
:10B7B00078B897000000E00005003A001A407800D1
:10B7C00094470200000000000000E0000300320087
:10B7D0000B40780009000700320007008904E800E8
:10B7E00064044400E28F5400D0FF3A004F06780012
:10B7F0004F05BE004F04BE0000000600889FBE003B
:10B800008A9FBE008C1F7800804578008ECDBF00D7
:10B810008B4F50001F0032000080FB0068092000A1
:10B820000880B9000CED210000004600226D0200E6
:10B8300000000000800478000ACF20008800780013
:10B840000A0078009E7002000000000009007800E5
:10B85000226D0200000000000B80FB000880B90090
:10B86000000046004C6D02000000000080047800DB
:10B87000880078000A007800FE6F020000000000D7
:10B88000090078004C6D0200000000000B007800F9
:10B890008EEDB7004F0678004F05BE004F04BE0086
:10B8A00000000600F6874700889FBE008A9FBE0002
:10B8B0008C9FBE008E1F78006ED820008ECDBF00FA
:10B8C0000081FB004210DD0060007F0001002000CD
:10B8D00018002000EB0F5000E08F580001033E00DD
:10B8E00000600100150037003600370013013700F3
:10B8F000750137008A01370090013700D201370007
:10B90000E601370052023700C2023700D202370088
:10B91000E102370005060700220020008000EB004E
:10B9200060407F0008480200000000003606070063
:10B930003100200001307F00E0FF370069D820008F
:10B940004210DD000080E80060C07C0094470200E7
:10B95000000000000000E000E4023200C0D020003F
:10B9600000688800280607001100200001B07C0054
:10B9700007EDEF000044EB000004FD0006EDB7000A
:10B980000004FD000CE1020000000000EA050700D1
:10B99000FCACEF00FEACEF00F02CEF00F22CEF005F
:10B9A0000800780084EDB700E005070053C0B3003D
:10B9B0000001EB001100200060C07C00BE570200B7
:10B9C0000000000068D82000E205070060407C000D
:10B9D000804A020000000000E10F400012003A001F
:10B9E00098050700784802000000000018002000B9
:10B9F0000000E00003003A00500020004B05070063
:10BA00000004EB000CE1020000000000D405070078
:10BA1000B4023400D80507005645020000000000BB
:10BA2000D8050700A5FF37000CE102000000000068
:10BA3000C1050700D6050700804A0200000000008B
:10BA4000E50F500001003600500020000001E80022
:10BA5000D205070008480200000000003200200064
:10BA6000213A2B00C0D02000DC10020000000000B2
:10BA70000000E00002003A00406888000D00370036
:10BA800042002000613A2B00C0D02000DC100200F0
:10BA9000000000000000E00003003A001400200055
:10BAA0004468880003003700700020004068880068
:10BAB0006B013700B6050700804A02000000000055
:10BAC00000047800E105070088017800040178008F
:10BAD000F1C3B30060407F00804A02000000000014
:10BAE00008017800800F5400010036000001780042
:10BAF000B0062000800F51000200360050002000E8
:10BB00004C013700A50507000848020000000000AE
:10BB1000C1D02000010040000048EB000100780087
:10BB20003E030700C0D02000F41102000000000016
:10BB30000004780072002000B13A2B00D0D0200021
:10BB4000DC100200000000000000E00009003A00E4
:10BB5000080DE20003003A008000200040688800E1
:10BB60000200370090002000406888008E05070022
:10BB700052FF37008804E900B0D0200000004400E4
:10BB8000F1C2B30090CF100004003200D0D02000EA
:10BB9000C89402000000000004EDB70040D020006F
:10BBA00000C2EB00904F120014003A007C80440069
:10BBB00002CF200002004000F1C2B30090CF10007D
:10BBC000030032007C004400017079000804E800A2
:10BBD000C0D0200000004400213B2B0009000900D8
:10BBE00031587800A000B10069044400D0D0200092
:10BBF000C89402000000000004EDB700B0D020009F
:10BC000080004400C0D02000808F50000700320028
:10BC1000E0C2B300914F1000040032008100E9003F
:10BC2000C0D02000808F5000F9FF3A000104E800E6
:10BC30000000EB0050688800E9CB2A0000004000BB
:10BC4000E0807C0008007800F4B8020000000000EA
:10BC50000004E000040032000A0DEC005068880087
:10BC6000EA0F5000F5FF360004CDBF00E14F400061
:10BC70000B003200FC980200000000000018A30036
:10BC80000700320004CDBF00C6990200000000008A
:10BC90000000E800AC9502000000000005EDB700D0
:10BCA00069D820005F05070060C07C00804A020060
:10BCB00000000000400507001600320010C0B3006D
:10BCC00006EDB70019050700E1FD2F008F80400049
:10BCD00060C07C00B2470200000000000801E900DB
:10BCE00050072000800F5100020036003505070084
:10BCF000F2FE3700086880002805070008480200A7
:10BD0000000000000004440060C2B300005C780042
:10BD1000086888000F05070060407F00804A020025
:10BD2000000000000001E8004105070060407F00BE
:10BD300008480200000000001B0507001800200052
:10BD40006DD82000F2FD2F000F01410082BF9F003F
:10BD50000005070060C07E00804A0200000000006D
:10BD600080047800E10F400014003A001905070034
:10BD70007848020000000000800078000000E00029
:10BD800004003A00B20407007400200004B07E00F2
:10BD9000010478000CE1020000000000F00407003C
:10BDA000D00134000B0507005645020000000000DA
:10BDB0000B05070001B07E00C0FE37000CE1020059
:10BDC00000000000DC040700E18F5400D1FE3200C7
:10BDD0006BD820001D050700890178000401780058
:10BDE000A1C3B30060C07D00804A020000000000D3
:10BDF000000578000084E800F00F540013003600BE
:10BE00000901E8009504070008480200000000004E
:10BE10000004EB00CEFF37000A4078001A0207004A
:10BE2000C204070008027800880178000801780041
:10BE3000A1C0B30060C07E00804A02000000000084
:10BE4000000678001800200019003700860407005B
:10BE50008FB8970060C07E00084802000000000014
:10BE60008A00E8000040EB000FB99700807079006D
:10BE7000088654000005EB00C9392B00FBFD2F009C
:10BE80008F854500990078000B00780010110200A2
:10BE900000000000C8040700DFFF32000A05E800C8
:10BEA0008984E800E30F5500F6FF3A000004EB0038
:10BEB0000C01E800DE04070060C07E0008480200B4
:10BEC00000000000A2FF3700006880000048EB007F
:10BED000C0D0200051020700006888004068800040
:10BEE000E80F500004003A00C70407007400200067
:10BEF00004307F0071FE3700C30407008E0040004D
:10BF00004000200080087800064DE20002003A0060
:10BF10005000200080087800066DEF0067FE3700B3
:10BF2000E281020000000000E20F50006F013200C9
:10BF3000B50407005100200001307F001204070003
:10BF400094470200000000006101B80049040700A6
:10BF50000A003A000CE10200000000008004070023
:10BF600006003400370407005645020000000000B8
:10BF70009B04070001307C0050FE370040688000C1
:10BF8000E10F50000400320069005000E20F500041
:10BF9000050036002900370026820200000000005C
:10BFA000E0DF9F000400370004030700E0DF9F008C
:10BFB0000004E0002A0032006FD89700E24F5000E2
:10BFC00008003A006C0407009447020000000000DB
:10BFD0000000E90001002000E0678800F1678800A8
:10BFE00042013700E14F500014003A00E603070019
:10BFF000944702000000000001002000E067880074
:10C00000F16788000CE10200000000004A0407000C
:10C01000750407001704070005003600090407002F
:10C0200078480200000000000000E0002F013A0004
:10C0300060002000BD03070020FE370072040700E7
:10C040006100200001307F0040D0200000C2EB00E2
:10C05000904F120005003A00400020004068880020
:10C060000904070001307F0014FE3700F02CEF00B8
:10C07000F22CEF0005CDBF00E14F400003003A0075
:10C08000F4ACEF00F6ACEF000300370041CF200026
:10C090000E97020000000000A503070068D82000EA
:10C0A0002204070023C0B3000001EB0011002000B0
:10C0B00060407C00BE570200000000004068800025
:10C0C0000000400081352B00E0807800DD03070090
:10C0D000404702000000000040688000EC0F500064
:10C0E0000E003A00EA03070040470200000000008B
:10C0F0000E040700C13B2B0060407C00404702005B
:10C1000000000000E20307004047020000000000BA
:10C11000E203070040470200000000004068800082
:10C12000E10F50000200360016040700EF00370050
:10C1300050688000EB0F50000F003200FB03070037
:10C14000F13C2B0060407F004047020000000000EF
:10C150005068800000004000E1D32A00E0807800B1
:10C16000050407004047020000000000CE0307005E
:10C17000404702000000000004CDBF00FC98020010
:10C18000000000000008A30005003200E7030700DC
:10C19000E13D2B0060407F004047020000000000AE
:10C1A000E2030700713F2B0060407F004047020020
:10C1B0000000000040688000E10F500005003200E0
:10C1C000A0678000B1678000E10F4000E08F480069
:10C1D00006003200D503070071402B0060407F004D
:10C1E00040470200000000000A003700CF030700AC
:10C1F00001412B0060407F0040470200000000002A
:10C20000CA03070091412B0060407F0040470200B5
:10C210000000000068D82000A0030700404702008B
:10C2200000000000064DE20004003200F6030700A3
:10C230008100200001307C00A0FD37009A03070038
:10C2400040470200000000009A0307009BFD3700F2
:10C25000C0D0200010688800064DE200690032005E
:10C2600069D82000B1030700D1412B0060C07C00D9
:10C2700040470200000000002800370000C2B30061
:10C2800080CF500005003A008D03070060C07C009D
:10C29000324602000000000020003700F0C2B30068
:10C2A00080CF50000B00360060CCB30000C04000CF
:10C2B000E64F50000700360050CAB30000C04000EF
:10C2C000E54F500003003600A0C7B30080CF5000F8
:10C2D0000F0036007D03070060C07C00324602007C
:10C2E000000000006FD89700CEB8020000000000E8
:10C2F000804078007803070032460200000000000A
:10C300006FD89700E2B8020000000000804078007B
:10C3100071030700324602000000000071030700AD
:10C32000D6FF3A0081030700D1C3B30060C07C0090
:10C33000324602000000000068D8200028003700C4
:10C3400000C2B30080CF500005003A005C03070034
:10C3500060407C00324602000000000020003700F0
:10C36000F0C2B30080CF50000B00360060CCB300A9
:10C3700000C04000E64F50000700360050CAB3002E
:10C3800000C04000E54F500003003600A0C7B300D6
:10C3900080CF50000F0036004C03070060407C0047
:10C3A00032460200000000006FD89700CEB80200AD
:10C3B000000000008040780022030700324602009F
:10C3C000000000006FD89700E2B8020000000000F3
:10C3D000804078001B030700324602000000000086
:10C3E00040030700D6FF3A008203070060C07C00CC
:10C3F0004047020000000000064DED0006EDB700CA
:10C4000098FF3A00280307004047020000000000A0
:10C41000280307003B0007000000E00002003A008C
:10C42000000478000600370004CDBF000296020029
:10C430000000000004EDEF00520307001800200088
:10C440004D03070006460200000000000000E00067
:10C4500024003A002500370068D820004210DD0093
:10C460000080E80060407C000646020000000000FA
:10C47000EF0F50001D003600C0678000D1678000BC
:10C48000D6FB07001D03070018003A005C030700F5
:10C4900001307C0009FD370004CDBF00E14F4000B2
:10C4A00003003200029602000000000004EDEF00DD
:10C4B00005CDBF00E14F40000300320002960200AC
:10C4C0000000000005EDEF002B03070056450200B9
:10C4D000000000004C0307000E0040000008EB00C5
:10C4E000020037000800E000F4FC32004F0778003B
:10C4F0004F06BE004F05BE004F04BE006F01B100E5
:10C50000000006004200FA00889FBE008A9FBE001D
:10C51000FF0207000646020000000000846780005A
:10C5200095678000A2678000B36780000401510016
:10C530008581590001002000800F5100818F590032
:10C54000010036000001BE008204780002004200B3
:10C55000E0804A008E0207000200E0001500320071
:10C560000A0420006BD82000090178008A8F54004B
:10C57000010036000A01780004CDBF0073FB2F00D4
:10C580008380470098960200000000000A0307001D
:10C5900036003200B402070073FB2F00838047008F
:10C5A00060C07D00A846020000000000888454009E
:10C5B000EDFF3A000C030700A0678000B167800020
:10C5C000800F5100818F59002A003A007302070042
:10C5D000A100200001307900FC2CEF00FE2CEF00C0
:10C5E00004CDBF008000EB001496020000000000A4
:10C5F000E8C7B30004CDBF0061FB2F008F8040006F
:10C6000014960200000000000000E0000400320068
:10C610004B020700EF70970088CF5000F5FF3A00FB
:10C620004702070005CDBF0081CF20000E97020012
:10C630000000000005CDBF0041CF20000E97020092
:10C6400000000000DC0207000A003A00F4ACEF0032
:10C65000F6ACEF0005CDBF0002960200000000001E
:10C6600005EDEF00080078000300370010002000FF
:10C67000010037000000EB004F05BE004F04BE0074
:10C680000080FA00000006000004E00002003A000A
:10C690000500070003003700E24F500001003A0098
:10C6A0004300070000000600889FBE008A9FBE006E
:10C6B00069D820003C0207002200200091C82A000F
:10C6C00060C07C0004490200000000000004780003
:10C6D00020D820000168800001005000800F540025
:10C6E0002E003900B70207002E0037003302070082
:10C6F000B1C3B30080D8200065407800804A0200B2
:10C7000000000000800478000A68800008017800BA
:10C71000800F540001003600000178006BD8200023
:10C72000820207008A00780060C07D00084802008D
:10C73000000000000000450061C2B300015878000D
:10C7400000688800890F54000E003600430207007D
:10C75000B2470200000000000B047800030037001D
:10C760001E020700B247020000000000AD020700F1
:10C7700060407C00804A0200000000000000E000F1
:10C78000F7FF320018020700044902000000000011
:10C790008902070003003200D4FF37000800E000E0
:10C7A000D2FF3A004F05BE004F04BE000000060055
:10C7B0000A00FA000C020700044902000000000011
:10C7C00080007800E90F50000500360020002000AE
:10C7D00040688800F02CEF00F22CEF000D003700CD
:10C7E0008902070001017800EA8057004C02070027
:10C7F00008480200000000008040EB006A00500082
:10C8000001F07F006A8057001E1202000000000045
:10C81000DF0107000080FA00000006000200FA00B5
:10C82000889FBE008A1F780000047800F41102007F
:10C8300000000000800178000000E00028003200C5
:10C84000080578000801780002047800B8407800F4
:10C850008304E900D0C3B30080CF5000030032004E
:10C860007740500080CF500002003A00005DEB009E
:10C8700017003700B0C2B30080CF500003003A0069
:10C880006B405000005D78001100370050C2B300CB
:10C8900080CF50000D003A00E18F540011003600A7
:10C8A0001844780098FF9F002240900080FF9F006E
:10C8B00063044100E38451004FB8970086B802003A
:10C8C00000000000005D780001003700015D780085
:10C8D0000900E000030032000801BE00DAFF370063
:10C8E000080578008040EB00015D78000A007800C0
:10C8F000014D78004F0578004F04BE000080FA001B
:10C9000000000600889FBE008A1F7800000478009F
:10C91000010578001004E00018003200880078005B
:10C920000A00780010110200000000000000E00082
:10C9300006003A000A007800F4110200000000002E
:10C94000000044000000E8000D00370008007800F7
:10C95000F411020000000000000044000004E800A0
:10C9600008007800F41102000000000000004400FC
:10C970000004E8001804E000E8FF3A000000EB00C3
:10C980004F0578004F04BE0000000600889FBE00DF
:10C99000000478000101780080007800D0C3B30063
:10C9A0002F000700800478000800E0000400320037
:10C9B0001804E000020032000800780097FF07002A
:10C9C000090078004F04BE0000000600889FBE00EA
:10C9D0008A9FBE008C1F7800000578000106780051
:10C9E000010178008000780060C2B3001C000700DD
:10C9F00080057800E20F50000E003A008867800042
:10CA000099678000C20107009447020000000000FF
:10CA100001002000800F5400818F5C0005003A0067
:10CA20000C0178008A0078000040EB000C00070041
:10CA3000800578000A00E000040032001A04E000DB
:10CA4000020032000A00780074FF07000B00780033
:10CA50004F0678004F05BE004F04BE0000000600E0
:10CA6000889FBE008A9FBE008C9FBE008E1F7800EC
:10CA70000047780081067800020678000004E00094
:10CA8000080032004D0107008040780080D8200067
:10CA900065407800804A02000000000080057800B0
:10CAA000040037009A0107009447020000000000CC
:10CAB000800578002A002000E18F4500390032000F
:10CAC000E10F560008003E000D00E00008003200B3
:10CAD0002001070008480200000000004E01070086
:10CAE0001A002000260037000D00E00006003A0082
:10CAF0001801070008480200000000004601070076
:10CB00000005EB001E0037000C81E900828F550004
:10CB100012003600120107008D00780060407D0091
:10CB200008480200000000003B0107000C8155008E
:10CB30000281E800BE01070060407D000848020055
:10CB400000000000340107008C8046000040EB002C
:10CB5000E0F89F001A0020000900370033010700A9
:10CB60008D0078006E0107000848020000000000F8
:10CB7000290107000040EB0080F57E000005EB0076
:10CB80000E04E000070032002B0107008000EB00DC
:10CB900082D8200060407900B24702000000000007
:10CBA0001D0107000A0078004F0778004F06BE00FD
:10CBB0004F05BE004F04BE00000006001000FA0042
:10CBC000889FBE008A1F780040688000EA0F5000EE
:10CBD00058003200EB0F50003F003200E90F5000C8
:10CBE00084003A0068D82000EF00070042002000CF
:10CBF000A1422B0060407C000449020000000000BC
:10CC000080007800E10F4000290032004701070052
:10CC1000010178008000EB0060407C0008480200C1
:10CC200000000000D2000700060107009447020040
:10CC300000000000E90F50006E0036003B010700C5
:10CC4000A2002000F680570060407C0008480200E7
:10CC500000000000C6000700A2002000F1422B00E7
:10CC600076805700DC100200000000000000E000A9
:10CC70000B003A00A000200040688800DE97020008
:10CC80000000000004EDB70062002000F2805700B1
:10CC90001E9802000000000020002000560037000F
:10CCA000B0002000406888002000200052003700BB
:10CCB000B500070094470200000000006401500026
:10CCC000C60007000848020000000000A800070096
:10CCD0001000200048003700A100070060407D00E0
:10CCE0009447020000000000CB0007000F0107007E
:10CCF00060407D007A47020000000000C0F92F006C
:10CD0000F1FF2F0038010700020040008380480037
:10CD1000C2F92F00F3FF2700820F5000838F5800C5
:10CD200034003600D800070001307D000000EB0021
:10CD300031003700F60007009447020000000000B1
:10CD4000000478002801070001002000820F500035
:10CD5000838F580001003600020478000800E000CC
:10CD6000170032006AD8200008017800F00F540044
:10CD70000100360002012000EC000700F680570099
:10CD800060407D00084802000000000000017800BB
:10CD9000806780009167800002005000E0805800AA
:10CDA0007B0007000204540004CDBF00F68057004A
:10CDB0001E980200000000000800E000EAFF3A00B0
:10CDC0008067800091678000E00F5000E08F58007E
:10CDD00008003A00100020008298020000000000C5
:10CDE0006E00070071002000013079000000EB00A8
:10CDF00001003700100020004F0578004F04BE00EE
:10CE00000080FA00000006004000FA00889FBE0083
:10CE10008A9FBE008C1F780000017800B7000700D1
:10CE200010003A0002007800C894020000000000E0
:10CE300000457800E14F400037003200C6990200FB
:10CE400000000000E0678800110037000A40780009
:10CE50000296020000000000FC2CEF00FE2CEF0008
:10CE60002D003700E0678000AC9502000000000054
:10CE700000457800E14F400027003200F267800053
:10CE80000300200021002000209702000000000085
:10CE90009F000700064602000000000080047800A2
:10CEA0000000E000150032000B0420006CD82000C8
:10CEB000090178008B8F5400010036000B017800C7
:10CEC00061FB2F008F8040000A4078009896020096
:10CED00000000000B8000700DCFF3200620007001D
:10CEE00061FB2F008F80400060407E00A84602005A
:10CEF0000000000088845400EDFF3A000A407800EA
:10CF0000B099020000000000F06788000A40780035
:10CF100002960200000000004F0678004F05BE0098
:10CF20004F04BE000080FA00000006004068880040
:10CF3000B50007007200200002307F0000000600EC
:10CF4000806780009167800061004000E0804800B9
:10CF50000F003700350007008000EB00700037003D
:10CF600088678000996780006AD820006F003700CA
:10CF70009D00070000015100E08159008267880090
:10CF8000936788000000060068D820002D00370055
:10CF90008067880091678800000006009A000700FB
:10CFA00062D8200000000600600007008002EB004D
:10CFB000050278008501780000000600E5D8200011
:10CFC000954278008582FB00C22ADD000002EB005A
:10CFD0008401780004017800000006009400070036
:10CFE00060407C0000000600E6D820001643780070
:10CFF0000683FB004233DD008002EB00050278006F
:10D00000850178002200200091C82A0080D82000E5
:10D01000664078000000060000045400E0845C00D4
:10D0200088678800996788000000060002000700F2
:10D030000B01780000000600886780009967800077
:10D04000710037003900070060407C0000000600D6
:10D0500050002000406888006B0037007400070013
:10D0600060C07D0000000600300007000801780065
:10D0700000000600E0678000F1678000800F51002B
:10D08000818F5900000006005F0007007100050055
:10D090006100070060407C000000060055000700AA
:10D0A00060407C00000006005200070060407F00E6
:10D0B000000006005200070001307F00000006005B
:10D0C0001A000700B1C2B3000000060017000700F5
:10D0D00051C2B300000006001400070060C07C00CD
:10D0E0000000060010688000B0407800A1DF9F00BB
:10D0F000106888000104E00000000600E06780007E
:10D10000F1678000E00F5000E08F5800000006003B
:10D110003D00070081D8200060C0780000000600B4
:10D1200083D8200060C079000000060036000700A8
:10D130000080E80000000600229D2400B3062000C5
:10D140000001410081814900C2678800D3678800DF
:10D150000000060039000700A1C0B300000006006F
:10D16000C2678000D36780000200500083805800AF
:10D170004240A90000000600ECFF070060407F006D
:10D18000000006001600070001307F0000000600C6
:10D190002400070060407F00000006001E0007001A
:10D1A00060407F00000006001700070021002000FB
:10D1B00001307F0000000600000478000000E0005D
:10D1C00000000600A2FF07007100200001B07C00F3
:10D1D00000000600D5FF070060C07E0000000600CA
:10D1E00009000700B1000500826780009367800096
:10D1F00000000600CDFF070091C82A0000000600CD
:10D2000001000700910005008ECDBF000080FB00EB
:10D210004200DD0000000600C4FF0700C1D020006E
:10D22000000006000500070001C2B3000000060070
:10D23000BEFF07008000EB000000060003000700AF
:10D24000840178000401780000000600B7FF0700A1
:10D250000002EB00000006000200FA00889FBE00FA
:10D26000CD22A800C922A9008000EB00011288008D
:10D27000F000200010128800211288004302A8004C
:10D2800042A2A80041E2A800F1030700D1C1B30007
:10D290006680570002040700AFF897000180FB008A
:10D2A0000038A300F8FF3A000080EA00E1046000C3
:10D2B000F5FF3A0018002000F8958800D9958800FD
:10D2C0008940780080C0B30043040700894078009B
:10D2D00090C0B3004004070011CAB300C0C0B3003F
:10D2E0003D04070091C0B300D0C0B3003A0407006A
:10D2F00011CAB300A0C0B3003704070091C0B30047
:10D30000B0C0B3003404070021CAB30040C0B3006A
:10D310003104070091C0B30050C0B3002E040700D1
:10D3200021CAB30020C0B3002B04070091C0B30092
:10D3300030C0B300280407000940780070030700DC
:10D340000020200076040700D1C0B3000940780017
:10D350002104070021C3B30020C0B3001E0407004E
:10D3600021C1B30040C0B3001B04070001C4B300D7
:10D3700030C0B30018040700F1C3B30090C0B3007D
:10D380001504070021C1B30060C0B30012040700F8
:10D39000C1C0B30070C0B3000F040700E1CEB300FA
:10D3A000A0C0B3000C04070051C0B300B0C0B3006C
:10D3B000090407004030200059040700F1822000D2
:10D3C0009140780040C0B3000304070001832000AF
:10D3D0009140780050C0B300FF0307001183200084
:10D3E0009140780020C0B300FB0307002183200098
:10D3F0009140780030C0B300F7030700318320006C
:10D400009140780009407800F30307004183200031
:10D410009140780008407800EF03070089407800C9
:10D4200050C1B300EC03070021C1B3006580570071
:10D430009B0307003FF89700C0F2B70001102000DF
:10D4400000C1B3001A0407002147230040C1B30004
:10D4500017040700890078000940780014040700C9
:10D46000090078002E04070041C0B300F0C1B300EA
:10D47000FE0307004F04BE000080FA000000060013
:10D480000200FA0011C0B3000F80E900A6030700F4
:10D490007FB897004200DE00610060000080FA0063
:10D4A000000006000200FA00F1C1B3000F80E9009D
:10D4B0007B030700EFF897000180FB004300DE00CC
:10D4C0000000A200610060000080FA000000060079
:10D4D000881F7800BE12E20010003A001000200001
:10D4E000F0958800D89580000804E90061040700E1
:10D4F000010036000004780001C4B300E0C1B300AD
:10D50000DA03070088407800C0C0B300B203070008
:10D51000C840DE00D0C0B300AF0307004F0478005E
:10D52000000006000600FA00889FBE008A9FBE0029
:10D5300090112000FA0307000AF02F00FB0F2000D3
:10D5400091C1B3006E805700550307002FF4970078
:10D55000E0002000F2030700E1C0B3006D80570037
:10D560004F0307003FF097000080FB008A846400AF
:10D5700080847400F1C0B3006C805700480307003A
:10D580004FF097004800DD008B84640080847400B5
:10D5900090112000E203070091C1B3006B80570097
:10D5A0003F0307005FF09700804F5400E4FF3A000C
:10D5B000C0002000DA030700C1C0B3006A80570032
:10D5C000370307006FF097000080FB000A04640037
:10D5D00000047400D1C0B300698057003003070015
:10D5E0007FF097004800DD000B0464000000740029
:10D5F000808F54000400360080805400109A200070
:10D600000101500005003700129A2000808F54005D
:10D6100002003200090050000001E9000200780019
:10D620004F05BE004F04BE000080FA000000060057
:10D630001600FA00889FBE008A1F780080047800D8
:10D640000105780090112000B503070091C1B300D7
:10D6500068805700120307000FFC97000000EB00E2
:10D66000AF0307000000EB000804E0003A003200BE
:10D67000BE12E20003003A0095FF07000000EB0035
:10D6800035003700D0958000E0958800C12B21003F
:10D69000914078000040EB004F030700D12B2100A0
:10D6A0009140780010C0B3004B03070041012000F7
:10D6B0007C805700510207003FB8970044B9020030
:10D6C00000000000B0BF9F002FB19700109A20000B
:10D6D000800F51000D003E00CFE0970061C0600058
:10D6E0000A003A00CFB197000001280000806100D5
:10D6F00006003A00BFB09700E05E2000808F500027
:10D7000002003E000378A30001003A000000FE0082
:10D71000D29588007080570005000900B05C780041
:10D720006900B1006000B10000CDEB007FF0970010
:10D73000E84F500006003A006FF097000004E00048
:10D7400002003200E64F500001003A00004D780020
:10D75000BE32EF00100020004F0578004F04BE00DD
:10D760000080FA00000006000200FA00889FBE0058
:10D770000004780081447800D2BF9F0031CAB30012
:10D7800020C0B3001403070091C0B30030C0B30041
:10D7900011030700009B2000DFB897008080400045
:10D7A000D1BF9F00AFF8970060C0B3000A03070025
:10D7B000BFF8970070C0B3000703070061002000A6
:10D7C000080078005D02070061002000F082200060
:10D7D0005A02070080C0B3004902070060C0B300CE
:10D7E0000904E00001003A00094078004402070003
:10D7F0004F04BE000080FA00000006001000FA008E
:10D80000889FBE008A9FBE008C9FBE00AA030700AF
:10D8100016030700A803070003030700A1C0B30015
:10D82000C0C1B30000030700A60307000F030700F1
:10D83000C0D2BF0065405000E14F50006F003E0075
:10D840000004EB00893E2000C1C1B3007480570082
:10D85000930207004FE897006A00600003003A0057
:10D860000804E800890F5400F7FF3A00C1C1B30073
:10D87000738057008A0207005FE897000018A30032
:10D8800003003A00703E2000800F54005B00360019
:10D890008C030700E40207008040EB007280570011
:10D8A0007F0207006FE897000080FB0009F02F005F
:10D8B000090565000005750011C0B30071805700AF
:10D8C00077020700FFEE97004868DD00F80F2000A0
:10D8D000080565000005750061C0B3007080570041
:10D8E0006F0207000FF097000080FB00898464003E
:10D8F0008084740071C0B3006F8057006802070015
:10D900001FF097004800DD00888464008084740064
:10D910000904E80088457800884078000040EB0062
:10D92000AD0207004844DE00884478008840780053
:10D9300010C0B300A80207007C86570081002000B9
:10D940000C007800AD0107000044EB00C1C1B3003A
:10D950006E805700520207002FF097000018A300B6
:10D96000200032003FB0970000D8A3001D00320015
:10D9700051030700BD0207004F030700AA0207007A
:10D98000A1C0B300C0C1B300A70207004D03070048
:10D99000B6020700C1C1B3006D8057004002070006
:10D9A0003FF097006A006000FAFF3200450307006D
:10D9B0009D0207008B4078000040EB0086020700C4
:10D9C0008940780010C0B300830207008100200066
:10D9D0000C007800890107000844E800F04F54006B
:10D9E000DAFF3A008A4078000040EB007A02070034
:10D9F0008D40780010C0B300770207004F06BE00CC
:10DA00004F05BE004F04BE000080FA000000060073
:10DA1000881F7800090307000200360020672F00E6
:10DA200000844000884078000040EB006A02070054
:10DA3000C840DE0010C0B300670207004F04780042
:10DA4000000006000400FA00881F78006681570075
:10DA50000019780021C0B30002007800100207000E
:10DA6000FA02070031C0B300638057000C020700C0
:10DA70001703070020C0B30057020700BFF8970044
:10DA800030C0B30054020700080078004F0478004B
:10DA90000080FA00000006000400FA00881F7800E9
:10DAA00066815700001978008040EB000200780082
:10DAB000FB010700E502070011C0B30063805700B7
:10DAC000F7010700020307000040EB0042020700D5
:10DAD000BFF8970010C0B3003F02070008007800AD
:10DAE0004F0478000080FA00000006000200FA00EF
:10DAF000889FBE008A9FBE0081057800CF02070084
:10DB00000200360020672F00008440008040EB00B8
:10DB10006A805700E20107006A8057003081FB00ED
:10DB200001F02F00010565000205750011C0B3006A
:10DB3000DB010700FFF497004848DD000A85FB0081
:10DB400000057500884078000040EB0022020700C5
:10DB5000C840DE0010C0B3001F0207000B007800B1
:10DB60000C000700000478008A4078000040EB00B9
:10DB7000190207008940780010C0B30016020700A0
:10DB8000080078004F05BE004F04BE000080FA0078
:10DB900000000600FA874700889FBE008A9FBE00EB
:10DBA0008C9FBE008E1F7800800578006044B8000E
:10DBB0008040EB0070805700B90107000FF097001C
:10DBC000D9020700010666000006760011C0B30006
:10DBD0006F805700B20107001FF797004870DD0003
:10DBE0000C86FB00000676000B00E00020003200EF
:10DBF000C0FD2F00808647008B007800F48F550011
:10DC00000100360041012000D1AF9F000D007800D7
:10DC1000FA000700DFA89700818555006180600049
:10DC2000050032000040EB0080F07E005FA9970005
:10DC30000201E800D2AF9F00DFA897000100E000DA
:10DC400009003200C0FD2F0000814700320078003B
:10DC500000044400E0844C000180E900800078006A
:10DC6000FAFF3A00D0AF9F000B00E000E2FF3A005D
:10DC70008C4078000040EB00D70107008E40780010
:10DC800010C0B300D40107006148B8000804400088
:10DC9000E0844800090044000080EA004F07780053
:10DCA0004F06BE004F05BE004F04BE00AF01B100DD
:10DCB000000006001000FA00889FBE008A9FBE0088
:10DCC0008C9FBE00A0B79F00B1B79F00C2B79F0056
:10DCD0008005EB000B057800E10F400002003200E8
:10DCE0000B0678000C00370021C0B3007680570087
:10DCF0006B0107002FE897000080FB00A0B79F0092
:10DD000031C0B30075805700650107003FE89700F8
:10DD1000D0E79F001C0020008006EB003FB097007A
:10DD2000E10F40000C003A008040EB007480570087
:10DD30005B0107004FE897000080FB00B0B79F0031
:10DD400011C0B30073805700550107005FE89700CA
:10DD5000F0E79F001D002000CFB49700E18F540032
:10DD600045003E000D00E0000E003A008D407800B6
:10DD7000728057004A0107006FE897006A020700A7
:10DD8000818565008085750011C0B30071805700E2
:10DD9000430107007FE897004800DD008B85FB000A
:10DDA000808575000C00E0000E003A0021C0B30031
:10DDB000708057003A0107000FF097005A020700E1
:10DDC000010565000005750031C0B3006F80570084
:10DDD000330107001FF097004800DD000A85FB00B3
:10DDE00000057500EFE097000040EB007A010700A6
:10DDF000FFE0970010C0B30077010700CFE0970065
:10DE000020C0B30074010700DFE0970030C0B3000A
:10DE1000710107000900E000060032000004EB0079
:10DE20006B000700B60007000804E800888F540064
:10DE3000FBFF3A000D00E00006003A008B4078003E
:10DE40000D40780064010700C858DE0010C0B30020
:10DE5000610107000C00E0004D003A008A407800A4
:10DE600020C0B3005C010700C850DE0030C0B30022
:10DE700059010700460037000C00E000080032009E
:10DE80002FB09700008544008A40780020C0B3007E
:10DE900051010700C850DE0030C0B3004E0107003A
:10DEA0003FB49700088544008A04E900C9B79F0081
:10DEB000F1C1B3006E805700F90007002FF0970002
:10DEC0000058A300FAFF3A00EFE0970000C1B3004A
:10DED00041010700FFE0970010C1B3003E010700B9
:10DEE000CFE0970040C1B3003B010700DFE097009F
:10DEF00050C1B30038010700DE01070005003E00F5
:10DF0000808F540003003600D0652F0000004500CC
:10DF1000C0B79F00788557009A40780020C1B300B1
:10DF20002D010700F78457009940780030C1B300F5
:10DF30002901070001C1B300F0C1B3003A01070095
:10DF400001C2B300F0C1B300480107000D00E000BA
:10DF50000F0032004FB197008200E800C1B79F0068
:10DF6000C401070004003E00808F5000020036000C
:10DF700000005100C0B79F009A4078000040EB00BD
:10DF8000150107009940780010C0B3001201070086
:10DF90004F06BE004F05BE004F04BE000080FA00D1
:10DFA000000006000200FA00F1C1B3000F80E90092
:10DFB000BB000700EFF897000180FB004500DE0082
:10DFC0000000A200610060000080FA00000006006E
:10DFD000AB01070000A0230040128800C201070027
:10DFE000FEFF3A00C3010700FCFF3200C401070036
:10DFF000CD22A8000080FB00000006000200FA000D
:10E0000080017800CD22A900A003200040128800E2
:10E010000300E000010032008301E900B2010700C3
:10E02000FEFF3A00B3010700FCFF3200B701070012
:10E030000002EB00E18F5000130036009101070051
:10E040006022B800451288000482E800A60107009B
:10E05000FEFF3A00A7010700FCFF320042128000D9
:10E060000300E000040032004810DE0090419800F8
:10E070008381E8008249780004805000E10F50005D
:10E08000F0FF3E00A4010700848F50001800360006
:10E090000001EB008002EB008480500045128800F4
:10E0A0000300E000080032008301E8008E01070051
:10E0B000FEFF3A008F010700FCFF32004012800093
:10E0C000804978000600370087010700FEFF3A000C
:10E0D00088010700FCFF32008C0107008001EB0083
:10E0E0000201E800828F5000ECFF3A000202420079
:10E0F000CD22A800040078000080FA00000006008D
:10E100000200FA005E0107000080FB0001A027006A
:10E11000010070004012880073010700FEFF3A0002
:10E1200074010700FCFF320075010700E0FF9F004B
:10E13000CD22A8000080FA00000006000200FA00CC
:10E140008001780001027800CD22A900A0072000FC
:10E150004012880064010700FEFF3A0065010700D5
:10E16000FCFF320069010700E10F52002800360071
:10E170001380FB004800DD000281FB0000017100FC
:10E180001340900068010700010161000001710067
:10E190008381E8003B010700421288000482E90005
:10E1A000E10F520014003600F10F200005F02F009F
:10E1B0001380FB004800DD000101610000017100D7
:10E1C000134090000080FB00050161000001710018
:10E1D0008381E80044010700FEFF3A004501070083
:10E1E000FCFF320049010700421288000482E90066
:10E1F000E10F5200EEFF3E003B010700FEFF3A0038
:10E200003C010700FCFF320040010700420107000B
:10E210000400E0000B00320003017800848041001C
:10E220003280FB00401288002F010700FEFF3A00F9
:10E2300030010700FCFF320034010700810F51005C
:10E24000F7FF3A00CD22A8000080FA000000060087
:10E250000200FA0001C2B300E0C1B300720007007F
:10E2600010002000DCE2020000000000CD22A90026
:10E27000F00F2000401288001B010700FEFF3A004B
:10E280001C010700FCFF3200020107001000200003
:10E29000DCE20200000000000080FA00000006003E
:10E2A0000001070010010700FEFF3A0011010700FE
:10E2B000FCFF3200401280004822EF000A010700F4
:10E2C000FEFF3A000B010700FCFF32004012800005
:10E2D000CD22A80000497800020078000000060066
:10E2E000F000070000010700FEFF3A0001010700EF
:10E2F000FCFF3200401280004822EF00FA000700C5
:10E30000FEFF3A00FB000700FCFF320040128000D5
:10E310004822EF00F4000700FEFF3A00F500070076
:10E32000FCFF3200E9FF37000400FA00889FBE00BE
:10E330008004780001447800402120007800070024
:10E340008840780040C1B3002300070011C0B3002B
:10E3500020C1B30020000700A0302000700007009B
:10E36000A1C0B30068805700DDFF07000FF89700D9
:10E3700061446000FAFF3A00402120006800070075
:10E380008840780020C1B3001300070081C1B300AA
:10E3900067805700D2FF07001FF89700AC00070006
:10E3A00091C1B30066805700CDFF07002FF897009A
:10E3B0004800DD000884FB00000474000000EB004E
:10E3C00057000700880C7800090078004F04BE0051
:10E3D0000080FA00000006000200FA00CD22A90029
:10E3E0000064A0000080FB0040128800BE0007000F
:10E3F000FEFF3A00BF000700FCFF32009800070054
:10E40000B9000700FEFF3A00BA000700FCFF320027
:10E41000BE0007000000000000000000CD22A800A0
:10E420000080FA00000006000200FA00CD22A900D8
:10E430000080FB00000AB30040128800AA00070019
:10E44000FEFF3A00AB000700FCFF3200840007002B
:10E45000A5000700FEFF3A00A6000700FCFF3200FF
:10E460008C0007000080FA00000006000200FA009D
:10E47000CD22A9000074A0000080FB00401288009B
:10E4800099000700FEFF3A009A000700FCFF3200E7
:10E490007300070094000700FEFF3A009500070094
:10E4A000FCFF32007B0007000080FA00000006003D
:10E4B0000400FA00881F780000447800D1BF9F0054
:10E4C00040212000160007008840780040C1B300BA
:10E4D000C1FF0700AFF8970060C1B300BEFF07009F
:10E4E000BFF8970070C1B300BBFF0700A030200049
:10E4F0000B000700A1C0B3006480570078FF07003D
:10E500004FF897000008A300FAFF3A000000EB0064
:10E51000030007004F0478000080FA0000000600A6
:10E520000200FA00F0BF9F0031C0B300F0C1B30099
:10E53000BDFF0700FFF89700F0C1B300CBFF070055
:10E540000080FA00000006000200FA0041C0B3009B
:10E55000F0C1B300B4FF0700D1C1B3000F80E900E0
:10E560004FFF0700EFF8970064C06000FAFF3A0021
:10E57000F1C1B3000F00E90049FF07007FF89700E1
:10E580000038A300FAFF3A0001C2B300E0C1B300B3
:10E59000B6FF07000080FA00000006000200FA0043
:10E5A00001C2B300E0C1B3009FFF0700D1C1B300B7
:10E5B0000F80E9003AFF0700EFF8970061C06000A4
:10E5C000FAFF320041C0B300F0C1B300A7FF07005B
:10E5D0000080FA0000000600881F780000447800E0
:10E5E00050312000CEFF07008840780050C1B300B2
:10E5F00079FF07000000EB00C9FF07004F04780017
:10E60000000006000200FA00881F78005031200048
:10E61000C3FF070051C1B3006480570020FF07000B
:10E620004FFC97000000EB00BDFF07000880FB00D7
:10E630004F0478000080FA0000000600E195800099
:10E6400081004000748440000A0037000FF89700F2
:10E650003500070001046400000474000000060097
:10E6600040128000A0FF9F000180FB004012880044
:10E6700000000600109A2000800F540000000600E1
:10E68000CD22A90041E2A9004342A80041E2A8002E
:10E690000000060040128000A0FF9F00CD22A800CD
:10E6A0000000060000017800CD22A9008180FB0057
:10E6B000411288000000060001C8B300F0C1B30099
:10E6C0000000060081C0B300F0C1B30000000600E6
:10E6D0001FF897004800DD000884FB000004740068
:10E6E000EFF097000000060040C2BF000018A30032
:10E6F0000000060040C2BF000008A30000000600A2
:10E700000500070040128000000006004012800053
:10E71000A0FF9F000000060041E2A9004342A900BB
:10E7200041E2A800000006000080FB0001F02F007D
:10E73000000006000041EB0022D898000001EB0029
:10E74000422898006011B800120098002300980039
:10E750003200980043009800704990000204A10024
:10E7600072489800704990000214A1007248980005
:10E77000704990000224A1007248980070499000EE
:10E780000254A10072489800601190000220A1007C
:10E790006210980041609900C005B000F4CF0200FB
:10E7A000000000000000060000017800C061910038
:10E7B0000304E00016003A0010C4B30010519800A2
:10E7C000C0C6B3002051980041C7B3003151980032
:10E7D0006340500040519800515198006C404000F7
:10E7E0006051980071405000705198000040E8005E
:10E7F00000599800135998002359980033599800EC
:10E8000043599800535998006359980016003700EF
:10E8100010C4B30010519800A0C7B3002051980055
:10E8200071405000305198006440400040519800C1
:10E8300068404000505198000040E9006051980045
:10E840006C405000705198000040EB000059980057
:10E850001059980020599800305998004059980054
:10E8600050599800605998008002200010119800BB
:10E8700062109000C1FF2F0001006000601198003D
:10E88000000006000400FA00889FBE008A1F78007E
:10E890008C9FBE0000057800C005B00074D0020057
:10E8A00000000000919780000100E8009097880028
:10E8B0000100E00003003200E18F5000040032004C
:10E8C000F232EF000A0078003C0007000200370037
:10E8D0000A007800920007006A1090000028A30048
:10E8E0002E0032004A6091000004E00005003A006A
:10E8F000D0CC2C00C1E4230090BF9F00A1BF9F009B
:10E9000004003700606626006100240090BF9F006D
:10E91000A1BF9F000CE10200000000002A16900039
:10E92000BA1690000C0150008D815800040033008D
:10E930000200BE00000307000004BE000300370011
:10E9400061006100C90207000004BE0002682900DE
:10E9500083812400EC0207000001BE000800BE0015
:10E96000F4040200000000000000E00005003C008C
:10E970000CE1020000000000800F5600818F5E0055
:10E98000060036006A1090000020A1006015980073
:10E990000A007800349E0200000000000A0078009F
:10E9A000A09A0200000000004F06BE004F0578004C
:10E9B0004F04BE000080FA0000000600889FBE00E1
:10E9C0008A9FBE008C9FBE00800478006028900063
:10E9D000E20F500006003200794890000054A10078
:10E9E000D70207000000EB00E084980048003700E1
:10E9F00079289000E10F500042003A0069869000AB
:10EA0000EE0F560017003C00798D9000899590001C
:10EA100059899000E98990000A00BE00F8040200BC
:10EA2000000000000000E00039003200DA8C98009D
:10EA3000EB8C98000C044600E806B00002002400AD
:10EA4000C36124000A00BE00B1020700FC040200FA
:10EA50000000000000B47C000C00E800E084980096
:10EA60002B003700EA062000090545006066B80063
:10EA70008005EB001A0478006140B900AE0207007F
:10EA80000800E00003003D0002002000037824009D
:10EA9000950207000001BE000C00BE0092020700B4
:10EAA0000006BE008B05E8000A85E800EF8F5500E0
:10EAB000F0FF3A000000EB00E08498000200200024
:10EAC000031724000C00BE00930207003205020069
:10EAD000000000004200DD00A2002000110009003B
:10EAE0000280D800E292200000015100828C980040
:10EAF000820C7800794890000054A0009002070032
:10EB000003003700794890000054A100F04C9800B1
:10EB10004F06BE004F05BE004F04BE0000000600B9
:10EB2000881F78000004780070289000E20F5000E1
:10EB300006003200784890000034A100704C980024
:10EB40000000EB00108C98003500370078489000EA
:10EB50000034A000704C9800784890000018A30082
:10EB60002F003A0018889000E10F50001E0032007C
:10EB7000E20F50002100320098909000E023200026
:10EB8000808F50000A003E00784890000018A300D3
:10EB900023003A0010002000108C98006011B8008B
:10EBA00008007800089E0200000000001C003700EA
:10EBB000502D2000808F50001900360078489000BA
:10EBC0000018A30016003A0020002000108C9800C6
:10EBD00018219000A821900008007800089E0200EB
:10EBE000000000000E00370098909000E023200005
:10EBF000808F50000A003600040037009890900083
:10EC0000502D2000808F500005003E000800780045
:10EC1000FE9D0200000000000000EB00108C980038
:10EC20004F047800000006000002BE000000E00073
:10EC300004003D00D0C2B300804878000402EA001E
:10EC400002003700B0C2B3008048780042062000BE
:10EC5000110009000202D80001C3B3008141400045
:10EC6000934298000280B90000005200A2002000E8
:10EC7000801F7800110009000200D8000001780010
:10EC80004F00780001C3B30001424100A442980044
:10EC9000E4C2B300B44298006A11B9000200500007
:10ECA00001404000C04298000040EB00D042980074
:10ECB00000000600D000FA00889FBE008A1F78007E
:10ECC0008004780001057800A0F22F000F004000BA
:10ECD000A1CC2B00C700090031587800800CB1008E
:10ECE000794890000058A300110032006E8457004C
:10ECF00020CC2B0007000900305C78008800B100B0
:10ED00001900780088007800C7FF0700881F780086
:10ED100021D92B00811F780060F22F000F004000E6
:10ED2000B012020000000000E4875700090037001D
:10ED300032DA2B00821F780020D92B00801F780048
:10ED400060F22F000F004000B0120200000000002F
:10ED5000E4875700F20107000F00400002000100A5
:10ED6000794890000018A300020032006000B8004B
:10ED70000200370019009000A9009000809FBE009B
:10ED8000C1DA2B00811F780040F22F000F004000F5
:10ED9000B012020000000000E6875700E001070003
:10EDA0000F0040000200010039009000C9009000EF
:10EDB000809FBE00E1DB2B00811F780040F22F0016
:10EDC0000F004000B012020000000000E101070047
:10EDD00040F22F000F00400002000100794890002F
:10EDE000E11F6000F2DC2B00821F780000F22F0090
:10EDF0000F004000B012020000000000D501070023
:10EE000000F22F000F00400002000100794890003E
:10EE10000000D100E11F6000D0DD2B00801F7800D2
:10EE2000C0F12F000F004000B012020000000000EF
:10EE3000C8010700C0F12F000F00400002000100D0
:10EE4000794890004200DE00E11F6000B1DE2B0037
:10EE5000811F780080F12F000F004000B0120200E7
:10EE600000000000BB01070080F12F000F004000F0
:10EE700002000100794890004500DE00E11F6000BB
:10EE800082DF2B00821F780040F12F000F0040002E
:10EE9000B012020000000000AE01070040F12F0098
:10EEA0000F00400002000100794890004300DE009E
:10EEB000E11F600070E02B00801F780000F12F0040
:10EEC0000F004000B012020000000000A101070086
:10EED00000F12F000F00400002000100794890006F
:10EEE0004400DE00E11F600051E12B00811F78002B
:10EEF000C0F02F000F004000B01202000000000020
:10EF000094010700C0F02F000F0040000200010034
:10EF1000FE875700496091000004E0000D003A00B0
:10EF2000C2C2BF000000FB000080EA004F00DE000C
:10EF3000801F780032E22B00821F780060F22F00E1
:10EF40000F004000B012020000000000E4875700EC
:10EF50000C003700CBC2BF000080FB004300DE0086
:10EF60000000A200E11F600030E22B00801F78004B
:10EF700060F22F000F004000B012020000000000FD
:10EF8000E4875700660107000F00400002000100FF
:10EF90004F0578004F04BE000080FA000000060014
:10EFA000C800FA00889FBE000004BE0040F32F0096
:10EFB0000F00400031E32B00C700090031587800F2
:10EFC000800CB100F11F4400B0EF2B00801F7800CF
:10EFD00000F32F000F004000B012020000000000FC
:10EFE0005201070000F32F000F0040000200010053
:10EFF00018209000A8209000809FBE0091F02B0068
:10F00000811F7800A0F22F000F004000B012020014
:10F010000000000045010700A0F22F000F00400093
:10F0200002000100085090000000FB00801F7800E3
:10F0300082F12B00821F780060F22F000F00400049
:10F04000B0120200000000003801070060F22F003B
:10F050000F0040000200010068109000E11F6000F6
:10F0600080F22B00801F780020F22F000F0040005C
:10F07000B0120200000000002C01070020F22F0057
:10F080000F0040000200010098109000811F7800DE
:10F0900062F32B00821F7800E0F12F000F00400088
:10F0A000B01202000000000020010700E0F12F0074
:10F0B0000F00400002000100681090000000D10025
:10F0C000E11F600070F42B00801F7800A0F12F007A
:10F0D0000F004000B0120200000000001301070002
:10F0E000A0F12F000F00400002000100FA87570036
:10F0F0004F04BE000080FA0000000600889FBE009A
:10F100008A1F7800000578008104780002047800E6
:10F1100001012000020078007AE3020000000000F4
:10F120000004E00005003A002100200009007800FA
:10F130005AD70200000000000700370071004500A8
:10F140008800780020110200000000000A0078000A
:10F150003CAF0200000000004F0578004F04BE00E5
:10F1600000000600000278008101780010C4B3009E
:10F17000924F1000050032001100200003007800BB
:10F180005AD70200000000000500370010C4B30089
:10F1900000529800040078003CAF0200000000001C
:10F1A0000000060001017800704890001100200066
:10F1B0000018A30005003200510020000200780072
:10F1C0005AD70200000000008000EB000100780028
:10F1D000000006000001BE00704890000018A30067
:10F1E0000600320051002000030078005AD70200C8
:10F1F000000000008000EB0009003700724890001A
:10F20000110020000028A30005003A00C1002000E2
:10F21000030078005AD70200000000008000EB00D5
:10F22000EAFF37008180FB008100EA00CF08DE00A2
:10F23000601190000200A1000101710062109800AD
:10F240003CAF020000000000000006001210980011
:10F250003CAF020000000000000006008180FB00BF
:10F260008100EA00CF08DE0081804000601190003C
:10F270000210A10001017100621098003CAF020071
:10F280000000000000000600889FBE008A9FBE00AC
:10F290008C9FBE000004BE000205BE000406BE0036
:10F2A000930007000801BE00990007000A01BE0094
:10F2B000970007000004BE00E00F5600E08F5E00DC
:10F2C000030035000C00BE009B000700050037005E
:10F2D00061006600010020008D01D1000C81D30087
:10F2E000650007000200200003F0230082000700F1
:10F2F0000200200003F023007B000700FC04020052
:10F30000000000004F06BE004F05BE004F04BE00C7
:10F31000000006000400FA00889FBE008A9FBE001D
:10F320008C9FBE000004BE0082BF9F0093BF9F0061
:10F330000405BE006E0007000006BE00E00F54008A
:10F34000E08F5C000200350050000700010037002C
:10F3500052000700E00F5500E08F5D00020035000D
:10F36000550007000100370055000700590007004D
:10F370000C00BE00660007000FB997009FB9970008
:10F38000650007004F06BE004F05BE004F04BE00DB
:10F390000080FA00000006000400FA00889FBE000A
:10F3A0008A9FBE008C1F7800000678000204BE0011
:10F3B000406091008080EB00E14F5000010032007E
:10F3C000110020001C259000AC2590006108B900B8
:10F3D0005900070090BF9F00A1BF9F00E00F54009D
:10F3E000E08F5C00020035002800070001003700B4
:10F3F0002A000700E00F5500E08F5D000200350095
:10F400002D000700010037002D0007003100070024
:10F410003D0007000004BE000C29900003002000FE
:10F420000A00BE0074050200000000000001BE00DA
:10F43000E00F5000E08F5800020035003E0007004A
:10F440000200370061006000080007000001BE00F4
:10F450000800BE00300007004F0678004F05BE00D0
:10F460004F04BE000080FA000000060001002000EA
:10F470008301D1000281D3000200700083807000FC
:10F480002D0007000001BE00170037000800BE0075
:10F49000290007000004BE000000060061006400AF
:10F4A000010020008901D1000881D300F2FF07008C
:10F4B0000004BE00000006000A00BE001E00370067
:10F4C00061006500010020008B01D1000A81D3009A
:10F4D000E9FF37000200200003F02B0006000700C0
:10F4E0000001BE00000006009605040000000000B8
:10F4F0006130B90010003700050007000001BE00B0
:10F500000800BE00F8FF37007FB097008FB8970063
:10F510005006040000000000B806040000000000CF
:10F520000C000700A0F22F00000006001901900057
:10F5300011C0B300000006003C07040000000000FA
:10F54000F04C9800794890000034A100F04C9800ED
:10F55000000006001A01900011C0B3000000060070
:10F56000F612E20003003A0010002000B097880075
:10F57000ECF1EF00ECD1BF00E14F4000030032009E
:10F5800030AB020000000000ECF1EF002F03070099
:10F59000F071EF00F091A800F031A8000000060023
:10F5A000ECD1BF00E14F40000300320030AB02005D
:10F5B00000000000ECF1EF00EE31EF00000006006B
:10F5C000EE11E20002003A0020030700F011A9004A
:10F5D00000000600708F80000000E0000100320093
:10F5E0001000200000000600808F80006100600095
:10F5F00000000600808F8000620060000200320080
:10F60000F031A9001000200000000600808F80006B
:10F610004300DE00F5FF370012030700000006007C
:10F62000889FBE008A9FBE008C9FBE00728F8000A4
:10F630000080EB008080EB0002004000E08048008A
:10F64000EB0F5000E08F58000E013E0000600100FB
:10F650000B00370012003700390037004400370034
:10F6600059003700AE003700D5003700E6003700FC
:10F67000D3003700E4003700D1003700E200370044
:10F680000303070096A9020000000000ECF1B70098
:10F69000E14F4000FB00320020002000708F880006
:10F6A000C0032000D08F8800FC31EF001672EF00FD
:10F6B000F011A900F051A900406A0200000000000A
:10F6C0000000E000EF003200ECD1BF006EAB0200A2
:10F6D00000000000B1122000810F5000E900360048
:10F6E000818F80004408DE000080EA006100600035
:10F6F0004400DD000140A10080807000818F8800FF
:10F70000E8020700F10F20003011020000000000A5
:10F710008000EB0010C0B300E20107000CE1020022
:10F7200000000000E5020700B0B602000000000083
:10F73000EE02070030002000708F8800D1003700F3
:10F74000ECD1BF0058AC020000000000910F200077
:10F75000810F500022003600F071A800CD00070094
:10F76000E24F5000C7003A0040002000708F880030
:10F77000ECD1BF006EAB02000000000011102000B1
:10F78000810F5000BF003600C60207008180E900EB
:10F7900030110200000000008000EB0030C0B30018
:10F7A000C00107000CE1020000000000C3020700D6
:10F7B000B0B6020000000000CC020700500020009C
:10F7C000708F8800AF003700ECD1BF0058AC02004A
:10F7D00000000000910F2000810F50000F003E003C
:10F7E0000CE1020000000000CF020700A500340079
:10F7F000B08F8000C18F8000F2032000820F500084
:10F80000E08F58009D003E000000400081804800CD
:10F81000B08F8800C18F8800980037009D000700D6
:10F82000E54F50008A003A00ECD1BF0030AB020037
:10F8300000000000ECF1EF000CE10200000000000D
:10F84000BF020700F011A800B39080000308A300D6
:10F8500001003200830207000328A3000A003200DF
:10F86000509080006190800006E8B7004801DE00FB
:10F870000200780007E8B7000100780008E8B70048
:10F880004808DE0009E8B7000318A3000A003200A8
:10F8900030908000419080000AE8B7004801DE0007
:10F8A000020078000BE8B700010078000CE8B70010
:10F8B0004808DE000DE8B7000338A3000800320056
:10F8C000709080000EE8B7004800DE000FE8B70037
:10F8D0008090800010E8B7004800DE0011E8B70013
:10F8E0000040EB0012E8B70013E8B70014E8B700D7
:10F8F00015E8B7000348A300620032009090800032
:10F9000012E8B7004800DE0013E8B700A0908000BE
:10F9100014E8B7004800DE0015E8B70059003700CA
:10F920000CE1020000000000948F8000A58F800091
:10F9300004005000858058009225260023002000F6
:10F94000820F5000838F58004E003600B08F800029
:10F950006300B800C28F80006311B90081004100CC
:10F96000D28F8000E38F8000800F5100818F59007B
:10F970000B003600A02526002100200004004000D6
:10F9800085804800908F8800A18F88006100510019
:10F99000E0805900D08F8800E18F8800390037005F
:10F9A0003B02070096A9020000000000ECF1B7003E
:10F9B000E14F40003300320070002000708F88005B
:10F9C000ECD1BF006EAB020000000000111020005F
:10F9D000810F50002B0036001100200030C0B30012
:10F9E00030010700F051A9000CE102000000000006
:10F9F00032020700B0B60200000000003B02070020
:10FA0000EE31EC001F003700ECD1BF0058AC020013
:10FA100000000000910F2000810F500009003E00FF
:10FA20000CE10200000000003F0207001500340056
:10FA3000EE11EC00708F8800EC0F500011003600C2
:10FA40000E00370013000700E54F5000030032009E
:10FA5000E64F50000B003A0008003700ECD1BF0021
:10FA600030AB020000000000ECF1EF000CE10200FE
:10FA700000000000320207000200370020002000D2
:10FA8000708F88004F06BE004F05BE004F04BE00B9
:10FA9000000006000800FA00889FBE000040EB004E
:10FAA000E0F79F006C80570076AC02000000000079
:10FAB0004FF09700E24F5000DD003A00C0012000F7
:10FAC0005EAB020000000000F88220005983200095
:10FAD0006C80570076AC020000000000CFF0970069
:10FAE00098CF1000E9003A000804E800888F54001D
:10FAF000F7FF3A00F051AB0008003A000001200087
:10FB00005EAB020000000000410020002020210028
:10FB10009AAC0200000000001612A800000F20009E
:10FB20005EAB0200000000006C80570076AC020063
:10FB3000000000000000E000BD003200CFF09700A0
:10FB400030C3B30080CF50008A00320007003E006F
:10FB5000E3CF500031003200E6CF50004F003200BA
:10FB6000E1CF5000AA003A001700370060C3B3008D
:10FB700080CF50006C003200E1CF4000AC0032007A
:10FB80000040E90080CF5000A1003A006C8057008F
:10FB900076AC0200000000004FF29700E14F5200E7
:10FBA000BA003A006A80570076AC020000000000FC
:10FBB000F051AB00DCFF32006FF09700E24F5000D5
:10FBC000D9FF3A00B10037006C80570076AC0200D4
:10FBD000000000004FF09700E44F5000AB003A00E7
:10FBE000F051AB000700320048C0B3006C805700F2
:10FBF00076AC0200000000000844E900CAFF3200B1
:10FC0000FAFF370041002000A02021009AAC02003A
:10FC1000000000001652A800C3FF37006B80570099
:10FC200076AC0200000000005FF09700E34F500048
:10FC300096003600F051AB00080032000044EB00A3
:10FC40006C80570076AC0200000000000844E80019
:10FC5000E44F540006003200F9FF37004100200055
:10FC6000602021009AAC0200000000001632A800BB
:10FC70005FF0970065405000D0F79F00E14F4000D3
:10FC8000A9FF32006C80570076AC02000000000033
:10FC9000B1010700A4FF3200FAFF37006B80570064
:10FCA00076AC0200000000005FF09700E34F5000C8
:10FCB00076003600F051AB0018003A0041002000F9
:10FCC000E02021009AAC0200000000001672A8009B
:10FCD0005FF0970064405000D0F79F00E34F500062
:10FCE0000E003600F051AB000C003A00410020003D
:10FCF000202121009AAC0200000000001692A8000A
:10FD00005FF0970064405000D0F79F000300370079
:10FD10006C80570076AC0200000000008E010700E6
:10FD200081FF3200FAFF37006C80570076AC02008A
:10FD300000000000CFF09700E4CF500053003A00DD
:10FD40006580570076AC0200000000006680570016
:10FD500076AC0200000000006780570076AC02001D
:10FD6000000000006880570076AC02000000000030
:10FD70006DFF37006C80570076AC02000000000079
:10FD80004FF29700E44F520040003A00F051AB00B0
:10FD9000080032000044EB006C80570076AC020093
:10FDA000000000000844E800E44F54005EFF320009
:10FDB000F9FF3700D01F210076AC020000000000E0
:10FDC000C01F210076AC020000000000B01F21001F
:10FDD00076AC020000000000A01F210076AC0200FB
:10FDE00000000000D08F8000E18F8000C509DE0098
:10FDF0004B0ADD004501DE000201720002005000E6
:10FE000083805800D08F8800E18F880046FF37003C
:10FE10006B805700010037006C80570076AC020001
:10FE2000000000004C0107003FFF3200FAFF3700DE
:10FE30006FF09700E24F500006003A004FB897006D
:10FE4000DFB89700F08F880001908800F051A8007B
:10FE500009003700F28F8000039080004FB89700B0
:10FE6000DFB89700800F5100818F590002003200E7
:10FE70000040EB00E0F79F00C0AC02000000000073
:10FE80006FF097000080FB0003003700C0AC020059
:10FE9000000000000000EB004F04BE000080FA00EC
:10FEA00000000600889FBE008A1F7800804478000A
:10FEB0000105780010C0B30098AB020000000000FC
:10FEC00010C0B30098AB02000000000060C0B30097
:10FED00098AB0200000000000040EB0098AB02006D
:10FEE0000000000020C1B30098AB02000000000039
:10FEF00030C2B30098AB02000000000040C3B30062
:10FF000098AB02000000000060C5B30098AB02008F
:10FF1000000000000040EB0098AB02000000000071
:10FF20000040EB0098AB0200000000000040EB0036
:10FF3000F091AB0001003A0000C8B30098AB02009A
:10FF4000000000000040EB0098AB02000000000041
:10FF5000E3CF540007003A000A00E0000500320039
:10FF60004100200020202100C0AB02000000000062
:10FF70000C0037000040EB0098AB020000000000CE
:10FF80000040EB0098AB0200000000000040EB00D6
:10FF900098AB0200000000000040EB0098AB0200AC
:10FFA000000000000044EB000040EB0098AB0200B2
:10FFB000000000000844E800EC4F5400FAFF3A004B
:10FFC00061002000F0822000C0AB020000000000B1
:10FFD000A8CCB3000040EB0098AB0200000000008A
:10FFE0000844E900FBFF3A0030C6B30098AB0200BA
:10FFF0000000000020C8B30098AB02000000000021
:020000040001F9
:1000000030C5B30098AB02000000000030C6B3005A
:1000100098AB02000000000050C3B30098AB020090
:100020000000000010C0B30098AB02000000000008
:100030000940780098AB020000000000E1CF5400B6
:1000400002003A00F051A90016003700E3CF540037
:1000500014003A000A00E00012003A0060C3B30046
:1000600098AB02000000000040C0B30098AB020053
:100070000000000001D2BF0098AB020000000000A9
:1000800000D2BF0098AB020000000000FFD1BF000B
:1000900098AB020000000000FED1BF0098AB020048
:1000A0000000000070C3B30098AB02000000000025
:1000B00040C0B30098AB02000000000010C0B300C5
:1000C00098AB02000000000030C0B30098AB020003
:1000D0000000000060C0B30098AB02000000000008
:1000E000C0C0B30098AB020000000000E3CF540092
:1000F00003003A000A00E000080032001100370057
:10010000E1CF54000F003A00109080002190800051
:10011000E00F5000E08F58000A00320020C3B30007
:1001200098AB02000000000040C0B30098AB020092
:10013000000000004100200020202100C0AB020090
:1001400000000000C0C0B30098AB02000000000037
:100150000004EB00E281200001C2B3006840790096
:10016000814F5000030032000804E800EF0F5400F4
:10017000FAFF3A000840780098AB02000000000047
:1001800088007800E0812000C0AB02000000000081
:1001900000C0EB0098AB020000000000018A800064
:1001A000B0122000808F500007003E00000478004D
:1001B0000040EB0098AB020000000000008A8000C5
:1001C000880F5000FAFF360021802000914078000F
:1001D0008180FB0003C8BF004800DD0001047000FF
:1001E00041802000914078008180FB0005C8BF005D
:1001F0004800DD00810470000A00E00006003A00BB
:100200000005FD0002E8B70003E8B70004E8B70006
:1002100005E8B7000005FD0002AC02000000000088
:100220000800780002E8B7004840DE0003E8B700A5
:100230000900780004E8B7004848DE0005E8B70088
:100240004F0578004F04BE0000000600200020008B
:10025000B08F8800F831EF0010002000708F880008
:1002600000000600109080002190800002E8B70096
:100270004801DE000200780003E8B70001007800C2
:1002800004E8B7004808DE0005E8B70000000600F3
:1002900034042000430420000041EB006000B8005B
:1002A00000000600ECD1BF0082C1B3000440BC00D6
:1002B000E00D210000004100A20005000006BE0084
:1002C000B08F8000C18F80006011B800A425260087
:1002D000250020006033B8009C07020000000000E9
:1002E0000205BE000004BE00000006000100200060
:1002F0000200200003002000A42526002500200085
:100300006033B800FA080200000000000804400052
:10031000898448000C0444008D844C00988F880028
:10032000A98F880000000600928F8000A38F8000B4
:1003300002005000838058004240A90000000600DF
:10034000908F8800A18F880060002000708F880047
:10035000F031A800000006001FF097000040E900FF
:1003600090F79F00E14F40000000060050678800B2
:10037000610A200080804000616788007067880003
:100380000000060082C5200001C5200040CE2000EC
:10039000BADF02000000000000C5200000000600D7
:1003A000000006000000EB00EE52E2000200320006
:1003B000EE72EF00100020000000060080C5200053
:1003C00000000600889FBE0081F52B00C0D02000F1
:1003D0008264020000000000800478000000E00059
:1003E00017003200C0C3B300994F100014003A0048
:1003F0000004EB00E8C07C0040CE2000C6DF020015
:10040000000000000000E00006003200E20F500093
:10041000060032000804E800FE0F54000800320015
:10042000F4FF3700EEF2B7000500370010C0B3004C
:10043000EEF2B70040CE2000C4DF02000000000052
:100440000000EB004F04BE00000006001400FA009C
:1004500004CDBF0042012000F48057007E990200C5
:10046000000000009200200001F62B00748057006D
:10047000DC100200000000000000E00003003A0071
:10048000400120000000E900FEFF3A0022012000A8
:10049000A1F62B0074805700DC1002000000000061
:1004A0008000EB000000E00002003A0004000700BA
:1004B00080007800010078000080FA00000006004B
:1004C0003400FA00889FBE008A9FBE0088678000C3
:1004D000996780006BD8200006030700944702004C
:1004E00000000000000578000203070078480200C1
:1004F000000000000000450001002000800F5400B3
:10050000818F5C0090003E00FA02070094470200D1
:10051000000000006101B800140020008067800026
:1005200091678000800F5100818F59008F00390042
:100530003303200042FC2F000F0141006000200027
:10054000010020009CD20200000000000FB89700BC
:100550000060A10080BF9F005B00370061002000A9
:10056000C0D02000C6640200000000000000E000CF
:1005700075003A000107200020D12000E664020047
:10058000000000000000E0006F003A00C8D020002A
:10059000D1F72B00080078001011020000000000C5
:1005A0000000E0000C003A0041FC2F008F8040006A
:1005B00020D1200096B70200000000000000E000FB
:1005C000610032002FA09700BFA09700C0AF9F002E
:1005D000D1AF9F003C00370001F82B0008007800E5
:1005E00010110200000000000000E00002003A00CC
:1005F000C0FC2F002100370031F82B0008007800E4
:1006000010110200000000000000E0000C003A00A1
:1006100080FC2F008080470020D1200096B7020088
:10062000000000000000E000470032004FA09700EB
:10063000DFA09700E0AF9F00F1AF9F0022003700DE
:1006400071F82B0008007800101102000000000073
:100650000000E00002003A0000FD2F000700370014
:10066000C1F82B0008007800101102000000000003
:100670000000E00008003A0040FD2F0080804700A5
:1006800020D1200096B70200000000000000E0002A
:100690000D003A002C00370011F92B0008007800FB
:1006A00010110200000000000000E00006003A0007
:1006B00010C3B300124DE30003003A000FB89700D7
:1006C0000060A00080BF9F0080678000916780006D
:1006D000E00F5000E08F5800A0FF3A0040FC2F00D0
:1006E0000F0040009AC1020000000000C1D02000AD
:1006F00060F92B0014000900B058780041FC2F006D
:100700008F8040007C80400001D220000F00090053
:10071000B05878000001B100306DEF0000D2200029
:1007200002C2B3008041EB0001D32000904F1100C2
:1007300001003A00034878000000E800808F500074
:10074000FAFF3A00060037001000200070628800AF
:10075000C0D02000B1FA2B001300090031587800F6
:10076000C0002000406888000002EB000400780010
:100770004F05BE004F04BE000080FA0000000600D6
:100780000800FA00889FBE006C84570000ACBE00D1
:1007900069D820000A0037006880570000405400E4
:1007A000E14F40000500320055020700E1C2B300EE
:1007B00060C07C0032460200000000000804E8002F
:1007C0001880FB00EC8057004AB8020000000000CF
:1007D0004B020700EC80570060C07C0040470200DD
:1007E0000000000065805700880F5000EAFF3A00C3
:1007F0004F04BE000080FA0000000600430207001C
:10080000E1812000200207004047020000000000B4
:10081000000006002EC8AB00050032003B020700B6
:10082000F1FB2B0018020700404702000000000007
:1008300000000600238020001602070032802000FE
:100840001702070043802000120207005280200098
:1008500017020700CAFF070000000600A38020005F
:100860000C020700B28020000D020700C3802000A8
:1008700008020700D28020000D020700C0FF070019
:100880000000060063802000020207007280200042
:100890000302070083802000FE01070092802000F1
:1008A00003020700B6FF070000000600E3802000F7
:1008B000F8010700F2802000F90107000381200001
:1008C000F401070012812000F9010700ACFF0700C6
:1008D0000000060023812000EE0107003281200085
:1008E000EF01070043812000EA0107005281200048
:1008F000EF010700A2FF070000000600889FBE006E
:100900008A1F78000102070081D8200060C07800AB
:100910000646020000000000F10F50000300360000
:100920008044EB00FA8220000C0037001000200009
:10093000E0678800FE2CEF001C0037000904E0008F
:1009400005003200F1010700A1C3B300CE0107008A
:1009500032460200000000000A05E8001A40780054
:10096000CEB80200000000008040780068D8200067
:10097000D301070032460200000000001A40780050
:10098000E2B802000000000080407800CC010700BF
:1009900032460200000000008944E800E6CF54001F
:1009A000E6FF3A00FC2CEF00FE2CEF004F0578002C
:1009B0004F04BE00000006000000FE00000006001C
:1009C000D2010700C1D02000AF010700404702005C
:1009D00000000000000006004C0CE20004003200A1
:1009E00090010700404702000000000003003700AC
:1009F0008F01070040470200000000004C2CEF0070
:100A0000000006004E0CE2000400320085010700E1
:100A10004047020000000000030037008401070087
:100A200040470200000000004E2CEF0000000600CE
:100A30000800FA006880570021FD2B00A301070081
:100A40007E010700829FBE0093FD2B00831F78006C
:100A50006E805700B012020000000000AB010700DA
:100A6000EE805700880107004047020000000000A8
:100A7000E68757000080FA00000006000800FA0030
:100A800068805700D1FD2B00930107006B01070020
:100A9000829FBE0093FD2B00831F78006E8057005D
:100AA000B01202000000000098010700EE8057001D
:100AB000750107004047020000000000E68757006C
:100AC0000080FA00000006001000FA007080570055
:100AD00041FE2B000F000900315878000001B100E1
:100AE0005067800055010700CC790200000000002B
:100AF000809FBE0040FF2B00801F7800768057004B
:100B0000B01202000000000080010700F6805700CC
:100B10005D0107004047020000000000E687570023
:100B20000080FA00000006001000FA0070805700F4
:100B300071FF2B000F000900315878000001B1004F
:100B4000606780003D010700CC79020000000000D2
:100B5000809FBE0040FF2B00801F780076805700EA
:100B6000B01202000000000068010700F680570084
:100B7000450107004047020000000000E6875700DB
:100B80000080FA00000006000800FA0068805700A4
:100B900071002C004D01070010219000A021900051
:100BA000829FBE0093FD2B00831F78006E8057004C
:100BB000B01202000000000054010700EE80570050
:100BC000310107004047020000000000E68757009F
:100BD0000080FA00000006000800FA006880570054
:100BE000E1002C003C01070010219000A0219000A2
:100BF000829FBE0093FD2B00831F78006E805700FC
:100C0000B01202000000000040010700EE80570013
:100C10001D0107004047020000000000E687570062
:100C20000080FA00000006000800FA006880570003
:100C300051012C00040107000028A30001003A0024
:100C400011022C00688057002011020000000000F3
:100C50002E010700E88057000B0107004047020003
:100C6000000000000080FA00000006000800FA0002
:100C70006880570071022C00F70007000028A300CD
:100C800001003A0011022C00688057002011020078
:100C9000000000001D010700E8805700FA0007006F
:100CA00040470200000000000080FA00000006003B
:100CB0000800FA0068805700E1022C00E2000700FB
:100CC0000018A30001003A0011022C0068805700B0
:100CD00020110200000000000C010700E88057000E
:100CE000E900070040470200000000000080FA0011
:100CF000000006000800FA006880570051032C002D
:100D0000D50007000018A30001003A0011022C00D2
:100D1000688057002011020000000000FB0007005F
:100D2000E8805700D800070040470200000000009C
:100D30000080FA00000006000800FA0068805700F2
:100D4000C1032C00E100070060109000C1012C00DD
:100D50000018A30001003A0011022C00688057001F
:100D60002011020000000000E8000700E8805700A2
:100D7000C500070040470200000000000080FA00A4
:100D8000000006000800FA006880570031042C00BB
:100D9000D100070060109000C1012C000018A300D2
:100DA00001003A0011022C00688057002011020057
:100DB00000000000D5000700E8805700B2000700DF
:100DC00040470200000000000080FA00000006001A
:100DD0000800FA0068805700A1042C00C100070039
:100DE0002ACEBF00C1012C00E14F500001003200AB
:100DF00011022C0068805700201102000000000042
:100E0000C2000700E88057009F000700404702002B
:100E1000000000000080FA00000006000A00FA004E
:100E2000706780009028910000289100E10F400039
:100E3000E08F5800010036006000B8006A8157005A
:100E400013052C000900090033597800A200B100F5
:100E5000809FBE0090FD2B00801F7800708057009F
:100E6000B012020000000000A8000700F080570048
:100E7000850007004047020000000000E687570099
:100E80000080FA00000006000800FA0068805700A1
:100E9000B1052C0093000700F0618000801F7800EE
:100EA00021062C00811F78006C805700B0120200D0
:100EB0000000000095000700EC805700720007005A
:100EC0004047020000000000E48757000080FA005D
:100ED000000006000800FA006880570051062C0048
:100EE0008000070000628000801F780021062C002F
:100EF000811F78006C805700B012020000000000D3
:100F000082000700EC8057005F00070040470200A6
:100F100000000000E48757000080FA00000006008F
:100F20000800FA0068805700C1062C006D00070019
:100F300010628000801F780021062C00811F78003D
:100F40006C805700B0120200000000006F00070024
:100F5000EC8057004C0007004047020000000000F2
:100F6000E48757000080FA00000006002000FA0025
:100F700000FE2F000F00400031072C003A00070050
:100F8000801F7800801F780020002000801F7800DC
:100F900031092C00811F780080FD2F000F004000D8
:100FA000B012020000000000340007008F804000F3
:100FB000350007004047020000000000E8875700A6
:100FC0000080FA00000006002000FA0000FE2F005A
:100FD0000F004000C1092C0023000700801F78008B
:100FE000801F780020002000801F780031092C002D
:100FF000811F780080FD2F000F004000B01202001A
:10100000000000001D0007008F8040001E00070048
:101010004047020000000000E88757000080FA0007
:10102000000006003900070071FC2B001600370095
:1010300036000700D1FC2B00130037001001900090
:10104000A0019000000006002000070070489000FA
:10105000C1012C00000006001F000700704890002E
:10106000C1012C00000006001F0009003158780063
:101070000002B1000000EB000000060023000700A2
:1010800081FD2F000000060082D82000604079001A
:1010900000000600934178008381FB0000000600F9
:1010A000124178004811DD000300710000000600C5
:1010B000124178004811DD00830071000000060035
:1010C0000F00070060407C000000060005000700DC
:1010D0005067800000000600020007006067800083
:1010E0000000060006000900315878007000B100C9
:1010F000000006000200070060C07D00000006003E
:10110000020007000080E800000006008ECDBF004E
:101110000080FB004200DD00000006008018210076
:101120008001EB0000C1EB00E11B21000308780007
:101130006248980072004000810F5000FBFF3A00A7
:1011400000000600E20F500023003A000200E00019
:1011500008003A00620020000A0307000500320080
:101160000001EB006A004000808F500001003A004F
:1011700012012000641821008001EB0016002000FD
:1011800083427800140090000000E0000E003A0056
:10119000010A7800E0062000808F500003003A002A
:1011A000F10F51000C003A0004003700F50207006F
:1011B00009003A00E60F510007003A0016029800B5
:1011C0000580FB0005003700720242008301E80041
:1011D000E38F5100EAFF3A00E00F20000000060014
:1011E000889FBE000102780082007800E24F500024
:1011F00021003E00E6020700E10F50001E003A0009
:10120000EF8F50001C003600E402070081047000DC
:1012100008003A00A99780008900E800A19788009B
:1012200080382100808F50000200360000402000EE
:10123000A0978800E0062000980F100009003A00EF
:101240000002EB0089017800044178006000B800DA
:1012500096A902000000000000549800E14F4000F1
:101260000500320029049800200020001004980096
:101270000000EB00010037000080EB004F04BE00CF
:1012800000000600889FBE008A9FBE008C9FBE00A3
:10129000E24F500036003E00CF020700C4020700B4
:1012A00033003A0018009000E30F500001003A00AC
:1012B000E80090000080E900E10F50002C003E00A3
:1012C0002F003700000578006C1821008086EB00A5
:1012D0008005EB00801821001000E00020003A009B
:1012E000A4C0B300A80190000041EB006000B8006A
:1012F000404402000000000080447800E24F4000BB
:101300001B003200284502000000000030002000D1
:10131000100498006A0498007258B90070014000E7
:1013200009717E008081E8004200200082317E0049
:10133000EE0140001200200082317E006401400076
:10134000A800900001317E004206200002307E009D
:101350000A05E9008D0F550007003200DCFF370059
:101360008B05E80072004000E38F5500DAFF3A0079
:101370000080EB00060037000000EB00040037009F
:101380000100E900E10F4000CEFF3A00FAFF37000C
:101390004F06BE004F05BE004F04BE000000060011
:1013A000E4874700889FBE008A9FBE008C9FBE00D6
:1013B0008E1F78008105780002067800E24F500009
:1013C00045003E0072020700E30F500042003A0061
:1013D0007702070040003A000005EB008918210061
:1013E000FD0F20006E18210040002000990F100012
:1013F00035003A00990090007002070032003A0070
:10140000E948900081F79F000140780028450200DC
:10141000000000000FF097004445020000000000AB
:101420000000E000280032000FF09700DA450200CB
:1014300000000000800178000B00E0001500320081
:101440000C00E00013003200F40020009C0F12009A
:101450002100360010806600C0459800934290003D
:10146000D5459800130090000D006000E0459800FD
:1014700033409000F0459800530090000D0060004C
:10148000A0459800B3489000B145980000012000A5
:10149000000E78007250B9006601400053029000BF
:1014A00004317F000E0140001302BE004401980089
:1014B000550198000080E8006200200002307F00A3
:1014C0000A80FB00050037000A05E800F2844400AA
:1014D000E30F5500C4FF3A00E00F20004F077800EB
:1014E0004F06BE004F05BE004F04BE004F00B100C6
:1014F00000000600889FBE008A9FBE0080427800E0
:101500000103780082007800E24F500062003E0044
:1015100031020700180190000200E0005E00320076
:10152000EF8F50005C003600A64090008180FB00E9
:10153000364090004800DD0081047000C6409000F5
:101540008180FB00564090004800DD0001057000DE
:10155000E64090008180FB00764090004800DD006E
:1015600081057000E00F5500E08F5D004A003200F9
:101570000900E000480032000D0207002A003A008E
:10158000E50F51000900320004003E000200E900AE
:10159000E10F500040003E00120037008000EB00D9
:1015A000E60F51003D0032003B0037000540780057
:1015B000CA0107000000E00037003A000850900020
:1015C0004445020000000000E1FF2F000000E000A1
:1015D0003200320060002000100498008000EB0010
:1015E0002E003700B4C0B3008901780032C0B300C8
:1015F0000A00BE00404402000000000000549800B1
:10160000E24F4000240032002845020000000000A4
:101610000000EB00700498005000200010049800B7
:10162000E1FF2F001D003700E10F510012003A00CA
:10163000A39780008300E800A197880080382100EC
:10164000808F50000200360000402000A0978800E4
:10165000090278000041EB006000B80096A9020082
:101660000000000000549800E14F40000A003200E2
:10167000200020001004980018009000E20F500095
:1016800005003A00390498004A0498005B04980069
:101690008000EB00010037008080EB000100780043
:1016A0004F05BE004F04BE00000006008002EB00A4
:1016B0000502780001000700000006001A00FA0089
:1016C000889FBE008A9FBE008C1F78000043780070
:1016D0008104780002047800E24F50008C003E0044
:1016E00022C1B3000440BC00601821000005410085
:1016F0009A0390000700E000850032009A0078000D
:10170000E0062000808F50006F003A004A009000F1
:10171000DA009000E0AF9F00F1AF9F003A06900022
:101720000400E00020003200F08F520078003A0000
:101730009A01070001067000C44090008180FB0000
:10174000544090004800DD0001017000E44090002A
:101750008180FB00744090004800DD008101700032
:10176000E2AF9F00F3AF9F00E18F53000E003A00FD
:10177000FA8057006011B8008288BE00768057005A
:101780000288BE00728057000288BE006E8057003B
:101790000288BE00050178000640780090FE070030
:1017A000E10F40005A0032006FA89700FFA8970091
:1017B000E00F5000E08F580004003A000080EB007A
:1017C0008080EB00E0AF9F00F1AF9F007E0107003B
:1017D000EB0D21000B0141006FA89700FFA89700B7
:1017E000B20F1000A28F18002600320000FE2F005A
:1017F00080804700640050000F0040000ACF0200C4
:10180000000000000000E000090032006E01070047
:101810000B014100C1FD2F008F804000090009002D
:1018200031597800A200B100A100B10015003700C5
:101830000CE1020000000000128C8000238C80006C
:101840000200500083805800A225260023002000BB
:10185000820F5000838F58002D003600C0FD2F00EE
:101860000F004000DECE0200000000000CE102008C
:1018700000000000108C8800218C88000084EB00A0
:10188000240037000A5090006EAB020000000000F8
:101890000000E0001E0032004B0107006A01410019
:1018A000E00D21000C3178008800780009007800F4
:1018B000C0AB0200000000000004780002AC02008F
:1018C00000000000130037002E01070010003A004E
:1018D000E68F53000E003A0006407800FF00070034
:1018E0000000E0000A003A000800E00009003200B1
:1018F0000A5090000801780089007800A84602008C
:1019000000000000000478000000E00001003A0040
:101910000084EB00080078004F0678004F05BE00F9
:101920004F04BE000080FA0000000600889FBE0041
:101930008A1F7800804178000105780082047800D1
:10194000E24F500021003E0023010700980078007C
:101950000C0107000D003A0018009000E60F50003F
:101960001A003A0003407800DC0007000000E000A5
:1019700016003A0008509000090178008A007800AB
:10198000084802000000000013003700E0062000B5
:10199000808F50000F003A0018009000E20F5000B6
:1019A0000A003A000850900058AC02000000000005
:1019B0000000E00007003200890078000A0078008B
:1019C0009AAC020000000000030037000080EB002A
:1019D000010037000000EB004F0578004F04BE0007
:1019E00000000600889FBE008A9FBE008C9FBE003C
:1019F00000457800810678000206780085057800A9
:101A0000F500070084047800E0062000980F10001D
:101A10002C003A0018009000E20F500047003A00F6
:101A20000850900058AC0200000000000000E000E8
:101A3000420032000900E0001D0032000B00E0000F
:101A40001B003200F00020009B0F10001800360031
:101A50000850900082C1B3000440BC00E10D210099
:101A60000101410012407800C044980012409000EB
:101A7000D044980022409000E04498003241900009
:101A8000F24498000850900082C1B3000440BC00AA
:101A90006A01410062C07800A04498000101410041
:101AA00012419000B244980000012000800D78009F
:101AB0008C0078000D0078009AAC02000000000055
:101AC0001F0037000400E000160032000500E000AF
:101AD00014003200F1002000958F10001100360034
:101AE00008509000DA4502000000000090407800A5
:101AF000C144980090409000D1449800A0409000CC
:101B0000E1449800B0409000F1449800A048900053
:101B1000A144980030489000B04498000001200093
:101B2000800D78008001EB000C0178008D007800BA
:101B30000A4078007DFF0700010037000000EB003D
:101B40004F06BE004F05BE004F04BE000000060059
:101B5000889FBE00800478000004EB00E381200031
:101B600002C2B30068C07900824F50000500320005
:101B70000004E000030032000804E800F00F540005
:101B8000F8FF3A000800E8000081EB00810F5000E8
:101B900008003C0008017800E1812000090078007D
:101BA00010120200000000000040EB0000F47C0076
